:1000000000800020691B0000311B0000511B000014
:1000100000000000000000000000000000000000E0
:10002000000000000000000000000000511B000064
:100030000000000000000000511B0000BD1B00007C
:10004000511B0000511B0000511B0000511B000000
:10005000F51A0000511B0000AD180000551B0000F0
:10006000511B0000511B0000511B000079070000CC
:10007000511B0000F5180000511B0000511B00002F
:10008000511B0000511B0000511B0000511B0000C0
:1000900000000000511B0000511B0000511B00001C
:1000A000511B0000511B0000511B0000511B0000A0
:1000B0000000000010B5064C2378002B07D1054B3B
:1000C000002B02D0044800E000BF0123237010BDC4
:1000D000800200200000000070D10000044B10B529
:1000E000002B03D00349044800E000BF10BDC04608
:1000F000000000008402002070D1000010B5002133
:100100000D2001F06DFF074B01211A88064B0D20D1
:100110001A800022054B5A809A80054B197001F015
:100120005FFF10BD9C030020C00300209C02002044
:10013000BE03002070B5144D144C2B78002B20D03A
:10014000134B236010220021206808F098F8122336
:10015000226813700F4B1B78002B0DD003220E4B1F
:1001600021689A568A705A882168CA7005212268C7
:10017000595611719B88537101232A7853402B7073
:1001800070BD064BDDE7C04602000020980300204A
:100190009E030020BE0300209C020020AE0300202E
:1001A00070B51E491E4801F0E3F91E4905F04AFDED
:1001B00006F03EF81C4B00B218801C4B1C4C1B88F0
:1001C000C01A0422A35E00B26080834200DAA080DD
:1001D000184B1B78002B08D1174A1388013B1BB220
:1001E0001380002B01DCFFF789FFFFF7A3FF134DFE
:1001F0001349280001F0C3FF0223E15E0A22280010
:1002000002F01BF828000F4901F0B9FF2800042371
:10021000E15E0A2202F015F870BDC04600507D4430
:10022000A8020020000020419C030020C003002001
:100230009C020020BE030020000000207009002066
:10024000D6C80000DCC8000010B5054C05492000E8
:1002500000F055F900221221200000F029F910BD0C
:10026000C40300208903000012221D4B70B51A80C0
:1002700000221C4C5A809A8077211B4A200001F0F2
:10028000C7F81A4D002815D128001949FA2401F0A1
:1002900087FF0D25A4000021280001F0A1FE200009
:1002A00001F0CAFC2800012101F09AFE200001F0B3
:1002B000C3FCF0E70121200001F086F904212000B1
:1002C00001F091F90321200001F09CF901212000A7
:1002D00001F0A7F92800074901F062FF70BDC04690
:1002E0009C020020A8020020C40300207009002006
:1002F00098C80000C8C80000E12110B5174C490299
:10030000200002F061FB01210D2001F039FE0121E6
:10031000032001F035FE0021022001F031FE012111
:10032000032001F05DFE00210D2001F059FEFFF7D2
:100330008BFFFFF799FF03220949022001F022FBFE
:100340000849200001F02CFF0021032001F048FEA5
:1003500001210D2001F044FE10BDC04670090020AF
:10036000FD000000E4C8000010B5FFF719FF1420DD
:1003700001F062FC10BD000010B50121014801F040
:1003800033F810BDA802002010B5074C07482378A9
:1003900010220749002B00D1064900F00FF8217800
:1003A0000D2001F01DFE10BD02000020C40300203E
:1003B000AE0300209E03002000207047F8B5050022
:1003C0000E0017000024BC4208D02B68315D1B686A
:1003D00028009847002801D00134F4E72000F8BD38
:1003E00070470300FC33196ADA69914203D01B6A33
:1003F000C018007E704701204042FBE70300FC3339
:10040000D8691B6AC01A01D50130FF30704700005F
:10041000F7B50193FA238026002504009B00836032
:10042000124B760008330F004560290000920360EC
:100430003200183007F023FF23002000FC33213066
:10044000DD6132001D622900FF3007F018FF8723AD
:100450009B00E3185D609D606B461B7827612375E8
:100460006B461B79A57520006375FEBDF8C80000BA
:1004700070B5060018250C49006902F0D1F9306901
:1004800002F01AF82B000821307D084C4343E31892
:10049000595601F0E9FD0821707D45436419615604
:1004A00001F0E2FD70BDC046A086010034CA000024
:1004B00070B506001825006902F08DF9306901F069
:1004C000FBFF2B000821307D064C4343E3185956AF
:1004D00001F0CAFD0821707D45436419615601F0A1
:1004E000C3FD70BD34CA00008A2300229B00C154A2
:1004F0000C3BC3185A609A600123837570478B23A5
:100500009B00C1507047020010B5FC3253689468DC
:100510000133DBB29C4202D054680155536010BDD8
:10052000F7B500240500170001932000A24227D050
:100530002B00FC33DC611C620122286901F0FAFF08
:10054000A0421CD02E001836286902F062F801344F
:1005500001003000FFF7D7FF2869A74206D001F05D
:10056000C9FF0221286901F0CFFFEDE701F0B9FFD3
:10057000019B002B03D00321286901F0C5FFE0B2E5
:10058000FEBD10B50123FFF7CBFF10BD002210B553
:10059000837D93420DD087239B00C4186368A468B1
:1005A0000133DBB2A34204D02130FF30FFF7ABFFB1
:1005B0000122100010BD0300FC3399685A68914273
:1005C00006D09A68805C9A680132D2B29A6070470D
:1005D00001204042FBE700228A2370B59B00827510
:1005E00005000E00C15C006901F0A4FF002806D1DF
:1005F0000321286901F088FF0224200070BD8723B1
:1006000028009B00EA18536894682130FF301C1BB7
:1006100001D50134FF34002C0ED02C69FFF7CBFF3D
:10062000C1B2200001F0B3FF0028E8D103212869FE
:1006300001F06AFF0324E0E7002EDED003212869E1
:1006400001F062FFD9E710B50121FFF7C4FF10BD2B
:1006500010B51830FFF7AFFF10BD70B5040000698A
:1006600001F0B5FF002814D0206901F0BEFF00287A
:1006700010D0206901F03EFF0321206901F044FF02
:100680008C239B00E558002D39D10023FC34E36115
:10069000236270BD206901F0B2FF002809D02069F3
:1006A00001F0A8FF002804D0206901F0ADFF002868
:1006B000DFD0206901F0A3FF002826D1206901F0D6
:1006C0008FFF0028E5D0206901F09EFF002837D079
:1006D00087239B00E218536892689B1A01D5013367
:1006E000FF33FF21002B05D020002130FF30FFF722
:1006F00062FFC1B2206901F05CFFA075C9E7236801
:1007000020001B699847A847BFE7206901F0F2FE67
:100710002069032101F0F8FE206901F075FF00282F
:10072000B7D0872300229B00E3185A609A60012308
:10073000A3758B239B00E3589342AAD09847A8E760
:100740002200FC32D369126A0133DBB22069934282
:1007500006D101F0C6FE0321206901F0D5FE98E71D
:1007600001F057FF010020001830FFF7CCFE206990
:1007700001F0C0FEEFE7000010B50248FFF76DFF83
:1007800010BDC046C403002010B505230422024951
:100790000248FFF73DFE10BDC8080020C40300203A
:1007A00070B5040092B048222B49684607F05EFD00
:1007B00023000025A9331B78AB4216D0230000206C
:1007C000AB331D782549002D37D10022244B06F08C
:1007D00075FC0022234B05F04BFD04F069FFFA2164
:1007E00080B2890004F098FD85B22300AA331B78FB
:1007F000002B17D023000020AC331E781749002EA1
:1008000022D107F025FB184905F01CFA174904F01E
:100810006DFF04F035FFFA2180B2890004F07CFD01
:100820002D18ADB26A46AE34237800209B00D35811
:10083000AB4200D8033812B070BD02000B00013D7E
:1008400005F016FDEDB2BEE702000B00013E05F01B
:100850000FFDF6B2D3E7C0461CC900000000F03F10
:1008600000409F40008078400000FA4400809C4394
:1008700000280AD04368002B07D08368002B04D0DF
:10088000C06843425841404270470120FBE7F0B541
:100890008FB005000C0005921E00002A00D1D0E0A8
:1008A000002E00D1CDE0830723D0486807F04CFA32
:1008B0003268736806F074FE02000B00009001912C
:1008C00006F0FCFB3269736906F0F8FBB268F36866
:1008D000029003910098019906F0F0FB0B000200D2
:1008E0000298039905F0C4FC059B30677167186096
:1008F000596000231F00EB0700D49FE0326F736F35
:10090000100019000092019306F0D8FB02000B00C2
:10091000069007910098019906F0D0FB0890099184
:10092000206807F011FA02000B000290039106F014
:10093000C5FB326A736A0A900B910098019906F020
:10094000BDFBB269F36905F093FCB26AF36A040077
:100950000D000698079906F0B1FB02000B0020007D
:10096000290005F085FC326B736B04000D000898BC
:10097000099906F0A3FB02000B002000290005F0F6
:1009800077FC029A039B06F099FB326C736C0C9017
:100990000D910098019906F091FBB26BF36B05F095
:1009A00067FCB26CF36C04000D000698079906F022
:1009B00085FB02000B002000290005F059FC326D78
:1009C000736D04000D000898099906F077FB02008A
:1009D0000B002000290005F04BFC02000B000C98D6
:1009E0000D9905F045FC326E736E069007910098E4
:1009F000019906F063FBB26DF36D05F039FC0A9ABC
:100A00000B9B06F05BFB0A9A0B9B04000D000298FF
:100A1000039906F053FBB26EF36E06F04FFB020033
:100A20000B002000290005F023FC0B0002000698B3
:100A3000079905F01DFC059B9860D96038000FB040
:100A4000F0BD01235B421F00F8E7F0B585B000AFB1
:100A5000F860B960DD78160055196A461C00EB1D78
:100A6000DB08DB00D31A9D4620007B60FFF700FF08
:100A7000002815D1636860789C46A378012B1AD0B2
:100A80008021FA68ABB20A43110065466A46A8475E
:100A900000239AB2B24206D3002801D00720404278
:100AA000BD4605B0F0BD7968E278C9188A5CB968BE
:100AB000CA540133EDE73300BA68F9686446A047C9
:100AC000EAE7F0B585B01E00150053006A4600AF96
:100AD0007B600733DB08DB00D31A04009D4630003F
:100AE000B960FB60FFF7C4FE002830D1002C2ED087
:100AF000BB68002B2BD0002D2ED01B78FA6813700A
:100B0000B378002B04D1230029197F308B4219D1EF
:100B10000123012D0DD9FB685A1C0123E15C1170E2
:100B2000B968C95C01335170D9B202328D42F5D82F
:100B3000BB8821787078B468FA68A047002808D08C
:100B4000072005E01A7802401A700133DEE7012021
:100B50004042BD4605B0F0BD0620F9E7F7B50500F7
:100B60006B461B209E1D98712B00A8331F786B4687
:100B7000DC1D01222B002100FFF767FF00280CD1AC
:100B8000302223783F01934317403B4323702F3A91
:100B90002B0021003000FFF794FFFEBDF0B50500EB
:100BA00085B008000C00FFF763FE002800D014E1B8
:100BB00006231D4227D002AB1B3003AE1870012262
:100BC00023003100FFF741FF00281CD1AB0708D5F7
:100BD00022000121A932337812788B430A40134353
:100BE00033706B0709D523000221AA331B783278B2
:100BF0005B000B408A431343337023000122310012
:100C000002A8FFF75EFFF0231D4266D0002864D1E2
:100C10000100032202A803AF07F031FB23000422E6
:100C200039001C20FFF711FF002856D130230600A1
:100C30001D421AD02300AC331A78EB0608D52300E6
:100C4000AB3339781B78073081430340194339703F
:100C5000AB0606D538213B78D2008B430A401343BC
:100C60003B701C23012602AA13702B0614D5230007
:100C7000AB33DA78112A01D91122DA7022001F2150
:100C8000AB32D2787B780A408B431343BB551D238C
:100C900002AA93550136F6B26B060ED523000E213B
:100CA000AD331B78FA785B008A430B401343BB5586
:100CB0001F2302AA93550136F6B22300A8331B78EE
:100CC000032B04D12000FFF76BFD002805D1230082
:100CD0003200390002A8FFF7F4FEE123DB001D42D9
:100CE0004BD0002849D103AE19302300012202A9BC
:100CF0003070FFF7AAFE00283FD123002200B03356
:100D0000B1321B781178013201931278EB050CD5C2
:100D10000127BC4602A800786346B8432700AF37D6
:100D20003F781F40384302AB1870AB0509D5022746
:100D300002AB1878019BB8435B003B40034302A819
:100D400003706B0508D5042002AB1B7889000140B5
:100D500083430B4302A90B702B0708D5402102AB3C
:100D60001B7892010A408B43134302AA137023009D
:100D7000012202A93000FFF7A4FEC0235B011D423F
:100D80002BD0002829D12300B3331F7801331B78DF
:100D90001A30019303AE02AB187001222300310018
:100DA000FFF753FE002818D12B0506D50222337811
:100DB0007F00934317401F433770EB0407D504218E
:100DC000019A337892008B430A4013433370230017
:100DD0000122310002A8FFF774FE05B0F0BD7E23AA
:100DE000F7B501AD2B706B465E1DB6230400337062
:100DF000FFF73EFD002826D16B469F1D01222300F0
:100E000039000330FFF721FE3B78DB0619D50028B7
:100E100017D12300012231002800FFF752FE0028DD
:100E200011D10230E36898476B46DD1D0122230093
:100E300029000220FFF709FE2B789B0701D4002828
:100E400001D004204042FEBDF0B589B06B46DD1DE7
:100E5000002304002B70FFF70BFD071E00D0D8E025
:100E6000A378012B00D1D7E00123E37023000122F6
:100E700029000020FFF7E9FD071E00D0C9E02B780C
:100E8000502B00D0CAE023702000FFF7A8FF071EF8
:100E900000D0BEE002AD01001522280007F0EFF9F6
:100EA0001522230029003120FFF7CFFD26006B78A3
:100EB000070028781B0288361843308006F044FF6C
:100EC0000022584B06F0FAF8EB7820616161A878AF
:100ED0001B021843708006F037FF0022524B06F0C9
:100EE000EDF8A061E16104202856307106F0F2FEB1
:100EF00000224E4B06F0E2F8AB792062616268791D
:100F00001B0218434A4B00B2F080C01806F0E2FE04
:100F10000022484B06F0D2F82B7AA062E162E87911
:100F20001B021843424B00B23081C01806F0D2FEBB
:100F30000022414B06F0C2F8206361630920285665
:100F4000B07206F0C7FE00223C4B06F0B7F8A06373
:100F5000E1630A202856F07206F0BCFE0022384BEE
:100F600006F0ACF82B7B20646164E87A1B0218431E
:100F7000B08106F0E9FE0022324B06F09FF8AB7B11
:100F8000A064E164687B1B021843F08106F0DCFE7C
:100F900000222D4B06F092F8206561650F2028563F
:100FA000307406F097FE0022284B06F087F8A06503
:100FB000E16510202856707406F08CFEFC23002298
:100FC0009B0506F07BF8AB7C20666166687C1B02A3
:100FD000184300B2708206F07DFE0022134B06F02B
:100FE0006DF8A066E16613202856307506F072FE93
:100FF00000220E4B06F062F8206761671420285625
:10100000707506F067FE0022114B06F057F8A067D6
:10101000E167380009B0F0BDE07027E702277F42A2
:10102000F7E7C046000070400000103E0000F03CB2
:1010300000C0FFFF0000B03E0000203E0000F03D79
:101040000000A03D000020400000903F0000703FE5
:101050000000E03B70B5040008000D00FFF708FC3D
:10106000002809D12B00012221001B30FFF7EDFCE5
:1010700023789B069B0F237070BDF0B585B00500EB
:10108000FFF7F6FB041E5ED12B00A8331B78290066
:10109000019302AB9E1C3000FFF7DCFF33780400A5
:1010A000002B19D01B2002AB03AED870DF1C01222D
:1010B0002B003100FFF7C9FC041E0AD1302233781F
:1010C0003100934333702F3A2B003800FFF7F9FCBF
:1010D00004000520EB689847002C34D1019B032BBA
:1010E00034D103AE2B00042231001C20FFF7ADFCED
:1010F0003278072104002B001000AB330840187031
:101100001F20D2100A405A7072780240DA70F278CA
:1011100052100A409A70002C15D12800FFF740FBAE
:10112000041E10D12800FFF719FD041E0BD12B005F
:10113000012231000220FFF788FC041E03D133781E
:101140005B0700D5053C200005B0F0BD019B012BDD
:10115000F9D12800FFF702FD0400F4E77FB5140081
:10116000060006220D006846002107F088F80822D4
:10117000002102A807F083F82000FFF779FB002880
:1011800027D1002D25D02300062269460430FFF721
:101190005CFC00281BD16B466A465B7892781B0288
:1011A000120413436A46127802A9134302936B4652
:1011B0001A795B7912021B041A436B46DB78300004
:1011C0001A432300039210332A00FFF760FB04B098
:1011D00070BD01204042FAE710B500F02DFD10BDB2
:1011E000F8B50F000D4E010030681C001500FFF728
:1011F0007BF93068390003681B689847013C084B4D
:10120000A4B230689C4205D0036829781B689847CF
:101210000135F3E7FFF717FA0020F8BDFC050020C1
:10122000FFFF0000F8B50023164E0700F356013308
:1012300006D10100144800F0B5FA04002000F8BD02
:101240000725002400200021305600F0C9FE0121AE
:101250000020A9400D4B3940185600F0C1FE002077
:101260000121305600F0BCFE0020094B64001856E6
:10127000E4B200F0E1FE002801D001231C43013D4F
:10128000E0D2DBE7FA05002000060020F905002087
:10129000F8050020F0B51C00002385B0174F019120
:1012A000FB5606001500013308D1002302AA537132
:1012B00013711349039A134800F044FA30000021D7
:1012C00000F08EFE0198FFF7ADFF013C0E4BA4B27B
:1012D0009C4204D02878FFF7A5FF0135F5E70121EE
:1012E000300000F07DFE0023FB56013302D105489B
:1012F00000F044FA002005B0F0BDC046FA05002019
:1013000040420F0000060020FFFF0000F0B51C0067
:10131000002385B0194E0191F356070015000133E3
:1013200008D1002302AA537113711549039A154875
:1013300000F008FA3800002100F052FE8020019BE6
:1013400003431800FFF76EFF013C0F4BA4B29C4211
:1013500005D00020FFF766FF28700135F4E7012172
:10136000380000F03DFE0023F356013302D105485A
:1013700000F004FA002005B0F0BDC046FA050020D8
:1013800040420F0000060020FFFF0000F7B51C00E0
:101390000700134D0191010028681600FFF7A4F81B
:1013A0002868019903681B6898472868FFF74BF97C
:1013B000E2B239002868FFF7E4F883B20120A342C3
:1013C0000CD1013C074BA4B29C4206D028680368AC
:1013D0005B69984730700136F3E70020FEBDC046D8
:1013E000FC050020FFFF0000FF22002301770549D4
:1013F00003620A70044983740A70044943740A70D2
:1014000003747047F9050020F8050020FA05002054
:10141000F8B504001C2026002500217520560F0079
:1014200029362A35431C22D1254B10001A60FFF7BC
:101430001FF8012337702B70224BE362224B2000F0
:101440002363224B28306363FFF7FEFC0300002078
:1014500083420BD12300D4331870013B60741870A1
:10146000A07498702074D03401302070F8BD012130
:1014700000F0B6FD1C200121205600F081FD002067
:10148000134B1856431C0AD1124800F033F9237F3E
:10149000337000232B70104BE362104BCFE7012118
:1014A00000F06EFD00200E4B0121185600F068FD83
:1014B00000200C4B0021185600F062FDE7E7C04603
:1014C000FC0500208D130000E1110000D91100007F
:1014D000FA050020000600200D1300009512000000
:1014E000F9050020F80500200200012330B5D232B2
:1014F0001370427C040085B00420002A00D0203004
:101500002200D1321370A37C002B15D10233184373
:10151000237C002B01D040231843E37C002B01D017
:1015200080231843250028352900FFF737FB0028C2
:1015300004D0002005B030BD1223E8E723000122CB
:10154000D0331A702800FFF798FD0028F1D12A0047
:1015500069460330FFF702FE009A019B2260636038
:10156000029A039BA260E36043425841C0B2E1E7A4
:1015700070B504000D1CFFF7B7FFA068E16806F026
:1015800067FC0C4904F04CFA291C04F049FA06F0F7
:101590000DFC094A094B02F0A7FD02000B000020D8
:1015A000074905F0FDFF0022064B05F087FD06F018
:1015B0004FFC70BD0000C842EBE2361AC05BC83F6A
:1015C0000000F03F40A5E5400023052907D80200B0
:1015D000D43211700122994203D1437413001800D0
:1015E00070474274FAE70023052907D80200D33276
:1015F00011700122994203D18374130018007047BF
:101600008274FAE70023072907D80200D532117047
:101610000122994203D10374130018007047027429
:10162000FAE702000020112904D813000130D63354
:101630001970D07470470000F0B5040085B01E002A
:101640000AAB1B78103001930BAB1B781700029389
:101650000CAB1B780D00039300F0F4F8200024304D
:1016600000F0F0F8220000234032A363E36313701C
:1016700063729D4205D10A4B0A4A22210A4806F0AC
:1016800089FD6B461B79200063716B461B7A2560D0
:10169000E3716B461B7B2771A671237205B0F0BD09
:1016A00069C90000DEC900007AC90000437A002B36
:1016B00004D18372C372C36001334372704730B583
:1016C000040085B002AD00680291039200F0B0FE04
:1016D0006B79227AE17900932068002301F052F8B7
:1016E0002979029A206800F0C7FE206800F096FE73
:1016F00005B030BD70B518260400FFF7D7FF3300E2
:10170000082120790D4D4343EB18595600F0ACFCED
:1017100033000821A0794343EB18595600F0A4FC8C
:10172000082160794643AD19695600F09DFC044BD1
:10173000200006CBFFF7C3FF70BDC04634CA0000CF
:101740004406002007B5837A00910192002B07D050
:101750009A070AD5EFF310835A425341C37272B607
:101760000099019AFFF7ABFF07BDDB07F8D5C36807
:10177000014A9BB29360F3E700180040837A002B84
:1017800005D09A0704D5C37A002B00D062B6704703
:10179000DB07FCD5C368024A9BB2D360F7E7C046BB
:1017A0000018004010B5006800F04BFE10BD0000AE
:1017B0001FB5094B094A0A491A6000225A711A7169
:1017C000012302930193093300930932023B054838
:1017D000FFF732FF05B000BD4406002000093D00C0
:1017E000C008002000060020094B1868002809D115
:1017F000EFF310820749002A08D172B6BFF35F8F5A
:1018000001320A701A6801321A6070470870F9E7ED
:10181000500600204C060020084B1A68002A0CD005
:101820001A68013A1A601B68002B06D1044B1B781A
:10183000002B02D0BFF35F8F62B6704750060020C6
:101840004C060020FF23002110B504000370FC3B70
:1018500041708170C170017143710C22083006F033
:101860000EFD200010BD000001220B0010B513403A
:1018700008D00D4B1A70042343708368002B00D0EE
:10188000984710BD0222114204D007490A704370E4
:10189000C368F3E704231942F3D0034A13700333F8
:1018A00043700369EAE7C0464E48004110B5FFF7B0
:1018B0009BFF0C4B1B8C1B071B0F0B2B0FD80A4AD3
:1018C0009900885800280AD00F2408490A78A243B2
:1018D00013430B70064B1978C9B2FFF7C5FFFFF72A
:1018E0009BFF10BD00480041540600203F480041C6
:1018F0004E48004110B5024802F03FFA10BDC04604
:101900008406002013B51249124800F0F1FC124978
:10191000124800F0EDFC1249124800F0E9FC1249AF
:10192000124800F0E5FC124C1249200000F0E0FCE7
:101930001149124800F0DCFC0023019301330093AD
:101940000722053321000E4802F086F913BDC04678
:1019500000080042C0080020000C0042C40800201B
:1019600000100042C808002000140042CC080020EB
:10197000D008002000180042001C0042D4080020BB
:1019800084060020F7B500921822162542434F4BDB
:1019900007009B185D5701916B1C4ED04C4B4D4C72
:1019A0001E68002E27D1310044224B4806F067FC08
:1019B00031004422494806F062FC1022484B494954
:1019C0001E60CA67C021C120474B49005A508000A1
:1019D0001958FF36B14319501A60444B444A5A8093
:1019E00002232278134323706378DB09012BFBD099
:1019F0000122374B1A6001231E00AE406269324358
:101A00006261019A002A18D0102D1FD1E278134389
:101A1000E370009B042B0BD818000723A2789A438D
:101A200003F070FC030C0E10120005231343A37087
:101A30002A4B019A1A64B6B2E660F7BD0423F5E7B3
:101A40000323F3E70223F1E70123EFE73800002740
:101A5000002100F009FB224B1F499C461B68BA007D
:101A6000BB421DD16046013303608E501B4B019970
:101A70009950072D19DD0123083DAD000721A9402C
:101A8000144A9B009B189A698A439A61009A042A17
:101A9000D1D81000996903F035FC0B101214160010
:101AA0008858B042E1D00137D9E7AD000023E5E71F
:101AB0000522AA400A439A61BDE70422F9E70322FE
:101AC000F7E70222F5E70122F3E7C04634CA000037
:101AD00060090020001800401C090020D8080020E0
:101AE0006409002004E100E000E100E0000C004097
:101AF00005400000F8B50024094B1B68A34200D83C
:101B0000F8BD084E084FA5003369EA591A4204D0BF
:101B1000064BEB589847EB5933610134ECE7C0466C
:101B200064090020001800401C090020D80800208B
:101B3000054B10B51B6C002B00D098470123034ABE
:101B4000D1780B43D37010BDD80800200018004096
:101B5000FEE70000034B10B51B68002B00D0984730
:101B600010BDC0466809002070B50F490F4CA14256
:101B700004D100F087F802F0D7F9FEE70C4D0023FE
:101B80008D42F6D0CA18E818A24205D3094B82420A
:101B9000EFD00949002204E0006804331060F1E747
:101BA00004C38B42FCD3E4E7000000207C02002049
:101BB00074D1000080020020640F002010B500F0F6
:101BC0005EF8002801D100F04FF810BD014B1860FD
:101BD0007047C04668090020F7B5134801228446C3
:101BE0001249134C8E68636805689B0E134001927E
:101BF00088686268019F920E3A4067463F68934248
:101C00000ED1BD420CD186420AD35B19FA25486831
:101C1000AD00861B07486B437043000DC018FEBD26
:101C20003D0013000600E3E76C09002010E000E02F
:101C300000ED00E05555000070B5041E10D0FFF710
:101C4000CBFF050000F01AF8FFF7C6FF054B401B5D
:101C50009842F7D9FA23013C9B00ED18002CF3D1F0
:101C600070BDC046E703000010B5034A1368013396
:101C7000136000F0FFFA10BD6C09002070470020CF
:101C8000704700001E22F0B5504851494368514D3D
:101C900093431A0002231343436008238A691343C2
:101CA000FE228B612B68D2039B0213404A4A1343E6
:101CB0004A4A936113000422DC681442FCD00124D8
:101CC000474A14701678264203D0567876B2002E12
:101CD000F8DB01249460547864B2002CFBDB414CA7
:101CE0005460547864B2002CFBDB8224E4015480FD
:101CF000547864B2002CFBDB02249C840E34DE6832
:101D00002642FCD0384CDC621024DE682642FCD02F
:101D10002C68A40E3F2C00D1203C9E6A334FA402B5
:101D20003E4034439C629C6A314EA40AA402344370
:101D30009C62304CDC6200249C841034DE682642B5
:101D4000FCD02D4C9C841024DE682642FCD002245A
:101D50009E8C34439C841024DE682642FCD00024F0
:101D60009460547864B2002CFBDB244C54605478AB
:101D700064B2002CFBDB1C6A214E344080261C62BE
:101D80001C6AB4431C62032393601E4B5360537858
:101D90005BB2002BFBDB0023FF240B721A4A4B7251
:101DA0008B72CB72194B1A60194A2B6811689A060C
:101DB0005B01C90E2340520F12020B431343154A15
:101DC00013858023426813434360F0BD0040004107
:101DD0000004004024608000060600000008004067
:101DE000000C004001040100B905FF7DFF03FFFF67
:101DF000FF01000080BB0A1C24050000000703004F
:101E0000FFFCFFFF03060100006CDC020400002061
:101E10002060800000400042FA212D4B10B5186868
:101E2000890003F079FA2B4B013898424FD82A49A0
:101E30002A4A4860C020136A00061B021B0A03439B
:101E4000136200238B6007330B608021136A09063D
:101E50001B021B0A0B431362FC22214B196A0A4323
:101E60001A62FF22196A12020A431A62A022196A30
:101E7000D2020A431A621B4B1C005A7852B2002A43
:101E8000FBDB194A5A80194B1A00597EC9090129EE
:101E9000FBD0C821890099800521D970537EDB09C8
:101EA000012BFBD0C02300205B011361907000F078
:101EB00023F863785BB2002BFBDB0D4B0D4A63808C
:101EC000D379DB09012BFBD04123537010BDFEE712
:101ED00004000020FFFFFF0010E000E000ED00E044
:101EE00000040040000C00401E4000000040004282
:101EF00021400000004800421F4900B50B004A7E07
:101F0000D209012AFBD001380A282FD803F0FAF9A8
:101F10001B2E2E2E2E2E062E2E2411001A69174946
:101F20000A400F211A615A788A43110001220A439C
:101F300010E01A6911490A400F211A615A788A4340
:101F400011000322F3E71A690C490A400F211A61B4
:101F50005A788A435A7000BD1A6908490A400F210D
:101F60001A615A788A4311000222E0E7F0221969C7
:101F700012050A43F3E7C04600400042FFFFFFF0AE
:101F8000182310B508244343134AD01804570134CA
:101F900012D001249A5643689C4003290CD80800AB
:101FA0000E49D2015218D318403303F0ABF9021096
:101FB000060B02211970546010BD0621197054607F
:101FC0009461F9E70621197054605461F4E7022125
:101FD00019709460F0E7C04634CA00000044004124
:101FE0001823F0B508245843114A13181C5701341C
:101FF0001BD0012635005F688356BD400D4ADB01CA
:102000009A18906805420BD10C00601E8441D219C9
:102010004032107834400336A400B043204310709F
:10202000044A9B18002901D15D61F0BD9D61FCE768
:1020300034CA000000440041182310B5082443436B
:1020400007490020CA181457013408D05B560549C7
:10205000DB015B18186A5368D8400123184010BD93
:1020600034CA0000004400411822424370B52D4E8E
:102070000300B218127A52B2140001320ED0481C7A
:1020800000240C280AD803F03DF9071F1F1F1F1F4B
:102090001F1F1F0B0B0B0B0001246442200070BD9F
:1020A000092905D100211800FFF76AFF0024F5E790
:1020B0000A2901D10839F6E700240B29EED10A39A3
:1020C0001800FFF75DFFE9E7182201205343F218DB
:1020D000F3565568144ADB016C089B18C9B22840B6
:1020E0001C1900280ED00F2030342278090102403C
:1020F00011434122C9B25B192170403319780A4358
:102100001A70D3E722000F26303214785B19B443DB
:102110002143117041224033197804000A431A7098
:10212000BCE7C04634CA000000440041F7B50600D1
:102130000D000C008B180193019B671B9C4207D07C
:10214000336821781B683000984701340028F3D1A8
:102150003800FEBD70B5040008000D0007F010F94E
:102160002368020029005B682000984770BD10B505
:102170000B1E02D0FFF7EEFF0300180010BD10B5D4
:10218000FFF7F5FF10BD10B503681B68984710BD39
:1021900010B50249FFF7DEFF10BDC046CCCB0000F2
:1021A00070B50400FFF7E3FF05002000FFF7F0FF24
:1021B000401970BDF0B58BB06B4615000022053399
:1021C0000600DA770800012D00D80A2509AC29009D
:1021D00003F028F9CAB2130037330700DBB209292C
:1021E00002D813003033DBB2013C2370002FEED154
:1021F00021003000FFF7BBFF0BB0F0BDF8B50600C3
:102200000C00151E04D10368C9B21B689847F8BDBD
:102210000A2A0CD100290BDA2D21FFF7B4FF614205
:1022200007002A003000FFF7C5FF3818EFE7D2B2E9
:1022300021003000FFF7BEFFE9E710B5FFF7DEFF32
:1022400010BD70B50400FFF7D9FF05002000FFF7AF
:102250009FFF401970BD0000014B18607047C046D9
:10226000080000200122024B52421A607047C0460B
:1022700008000020164A10B51368591C26D0013BEF
:102280001360002B22D172B6124B134A04339342CF
:1022900013D9124A01211000147D0C42FCD02021D8
:1022A000148BFF319B085B0021431183D3610C4BDE
:1022B00013800123027D1A42FCD0BFF34F8F094BDC
:1022C000094ADA60BFF34F8FC046FDE710BDC04634
:1022D0000800002000000000030200000040004150
:1022E00002A5FFFF00ED00E00400FA0510007047B2
:1022F000016070479446F0B59E1E721E964162467C
:10230000056892072F6836063A4332432A6007254C
:1023100005AC24780068A4012940214342680024C8
:10232000022B00D05C03114321434160F0BD30B566
:10233000C0250368AD031C6812052A402243C0244F
:102340000904A40221401143196003685A68144328
:102350005C6030BD0123026811680B4313600368A1
:102360001A68D207FCD4DA69D207F9D4704702237D
:10237000026811680B4313600268D3699B07FCD4A1
:10238000704703681A7ED20702D41A7E9207FCD5E2
:102390007047002203685A8370470368187E40071D
:1023A000C00F70470368187EC00970478023026819
:1023B0005B42117E0B43137670470368588B80078E
:1023C000C00F704702230268518B0B435383704741
:1023D0000368187EC007C00F70470368188DC0B22D
:1023E000704703681A7ED207FCD589B2012019858F
:1023F0007047012203689A757047012203681A75B5
:1024000070470123026811680B43136003681A6860
:10241000D207FCD4DA69D207F9D4704702230268E4
:1024200011680B4313600268D3699B07FCD47047A3
:102430000368DA699207FCD402211A688A431A6099
:1024400070470268936A5B0A5B02194391620368F2
:102450001A7E5207FCD5986AC0B2704710B5490081
:10246000044802F059FF80B2002801D0013880B240
:10247000C0B210BD006CDC0270B54B080C0001212D
:1024800005680B400C402E6824075B072343334349
:102490002B6011000468FFF7E1FF207370BD01237A
:1024A000026811680B43136003681A68D207FCD4F2
:1024B000DA69D207F9D470470223026811680B4326
:1024C00013600368DA699207FCD430215A8B8A437F
:1024D000110010220A435A830268D3695B07FCD4B7
:1024E000704780230268DB02116851680B43536018
:1024F00070470000036803491A685A680A405A6026
:102500007047C046FFFFFBFF032230B50368114050
:102510001C68074D5A6809042A40E4061143640FF9
:102520005960052C03D10268D3695B07FCD430BD28
:10253000FFFFFCFF490010B511430468CBB2618B6B
:102540008906890F012904D0618B8906890F022928
:10255000F5D1616AC90AC902194361620368002A98
:1025600008D11A7ED207FCD5588B4007C30F012033
:1025700058400BE0187E8007C00FF5D11A7ED207B5
:10258000F8D5C022596892020A435A6010BD036808
:10259000283319700368187EC007C00F03D15A8B07
:1025A000D207F8D57047588B4007C30F0120584019
:1025B000F8E7036828331970036800201A7E520771
:1025C00004D5588B01234007C00F5840704703685B
:1025D0001868C006400F043843425841C0B27047E3
:1025E0000368187E4007C00F70470368187EC00755
:1025F000C00F70470368588BC006C00F7047036850
:10260000187E8007C00F70470368588B0007C00F03
:10261000704703681A68D206520F052A02D11A7E43
:102620009207FCD528331878C0B270470368104A67
:10263000934213D00F4A934212D00F4A934211D0C3
:102640000E4A934210D00E4A93420FD001200D4AF9
:102650004042934201D1063040B270470020FBE770
:102660000120F9E70220F7E70320F5E70420F3E76C
:1026700000080042000C004200100042001400421A
:1026800000180042001C0042F8B5FFF7CFFF0028F9
:102690002EDBC3001C481F22C01805230579C35632
:1026A00001201A4090400326C022184952001E40C3
:1026B000F6008850813AB240C024D243B440002B87
:1026C00017DA0F263340083B114E9B089B009B19DD
:1026D000DE6932401443DC613F231D408023DB016F
:1026E0001D430C4B08605D805A7852B2002AFBDB18
:1026F000F8BD064E9B089B009B19C026B6009F594B
:102700003A4014439C51E7E7D0CB000000E100E0E1
:1027100000ED00E0000C0040F8B504000F001600CA
:102720001D00FFF7B1FF2000FFF714FE1C21BB00C6
:102730000B4071072268090C0B4313608423226845
:102740009375012F1AD11021012E00D008390C4B9E
:1027500069431868C00002F0DFFD072221680240CB
:102760008B895203DB04DB0C13438B812268030447
:102770009089DB0C400B400318439081F8BDC046A4
:1027800004000020F7B50400019308AB0D0016000B
:102790001F78FFF736FE2000FFF776FFC0223605D0
:1027A000920332400C261643C0222D04920215409B
:1027B000072223683543BF072F431F60019B216811
:1027C00013401A0080239B0213434B602268D36995
:1027D0005B07FCD4F7BD70B504000D001600FFF7D1
:1027E00053FF2000FFF75BFE1C2221686D000B6881
:1027F00093431A0010231343FF220B6023681540F4
:102800005D62002E04D001232268516A0B4353629B
:102810000723226893752268D3695B07FCD470BDD7
:10282000F8B504000F00FFF72FFF2000FFF737FE79
:102830001422236879001A600C4B25681E6830004A
:1028400002F06AFD0A490400300002F065FD7D23B4
:10285000FA215843C90002F05FFDFF23241AE868FB
:10286000053C1C4098430443EC60F8BD0400002084
:1028700040420F003F20704713B56B460268D97184
:102880000733546819000122A04716BD10B5022174
:10289000006900F009FD034B1B6801335A1E934188
:1028A000181810BD5C00002010B50321006900F06D
:1028B00011FD10BD10B50321006900F0D9FC10BD59
:1028C00010B5054C23685A1C04D103685B6998470E
:1028D00003002060180010BD5C000020074B0200C0
:1028E000186810B5411C03D0012252421A6010BD75
:1028F0000221106900F0D8FDF9E7C0465C00002015
:1029000010B51300094A0400D079C0B2002805D1DF
:10291000627E002A02D00123636006E00A0020697B
:10292000032100F0CFFD0028F5D010BD10000020DD
:1029300010B503784222023303700249024800F0C6
:102940006DFE10BD180000208C09002010B5017824
:10295000020043780020A12908D1212B05D10722AC
:102960001649174800F05AFE012010BD2129FCD15C
:10297000202B13D107221149114800F0EFFC9622B9
:102980000E4BD200196891420ED10124D87904402F
:102990000AD1FA20FFF760FC0020E6E7222B06D1DF
:1029A0009278064BDA71EAE7FFF75CFCF4E7232B39
:1029B000DBD15288034B1A60D7E7C04610000020D5
:1029C0008C0900200C000020012343767047000092
:1029D000FA220021054B92009A60054A596008329C
:1029E0001A60044A19761A617047C04670090020BF
:1029F00000CC00008C0900207047704770B50F268E
:102A0000CB1D013902003240D5B22C000009303410
:102A1000092A00DD07341C70013B8B42F2D170BDE6
:102A2000A02110B50400490001F05AFB200010BDA0
:102A3000F8B5032908D1304B8000C058002802D0D7
:102A400003689B689847F8BD822919D1C3B22B4D02
:102A50005A01AA1891692A4C80010C40C0218905AD
:102A6000214391612749083340187021506128683B
:102A70005B011A5C8A43110030220A431A54E2E7D0
:102A80000029E0D1C026C1B21C4C4B01E3189A6862
:102A90001B4DB6052A4032439A601B4A80018218BA
:102AA0005A600A000727246808325201115DB943B1
:102AB0000F000121394311559F6912493D404018CB
:102AC0002E439E6158617020115D814308001021E2
:102AD0000143115599680D48A21808408021490307
:102AE000014399609968890B8903996040231179A2
:102AF0000B431371A7E7C04690090020440E002045
:102B0000FFFFFF8FB8090020780B0020FF3F00F087
:102B1000EFF3108303600123436072B670470368CC
:102B2000002B02D162B6BFF36F8F7047F7B5050077
:102B3000FC35EB690600002B18D196277F00C45D99
:102B40006846FFF7E5FF019BE4B2013B02D3F45D69
:102B5000E4B2FAE768460193FFF7E1FF002C01D1E8
:102B60000020FEBDE86AAB6AC01AFAE76846FFF7C4
:102B7000CFFF9E220024019B5200013B02D3B45C94
:102B8000E4B2FAE768460193FFF7C9FF002CE7D0EB
:102B9000E86BAB6BE8E7000030B54468FC30436994
:102BA0008069DBB25A01A2189168094D800429405E
:102BB00000090143916091680833890B8903916092
:102BC00022685B01D318402219790A431A7130BD7B
:102BD000FF3F00F0F7B50500FF21FC356A69436847
:102BE0000A401B68083252019A18D3790400DB07A7
:102BF00054D50126D6716B6962680B405B01D3180E
:102C0000286A9A689204920C002822D1EA62EA6A41
:102C1000002A40D06A6B2E6268465A60FFF778FF40
:102C20009E273E21019B7F00013BFF315A1C2ED085
:102C300096225200A654E25D581ED2B2002A05D058
:102C4000665468460193FFF76AFFF7BD62540300BC
:102C5000ECE7EA63EA6B002A1DD000222A626A6A66
:102C600068465A60FFF754FF96273E21019B7F007C
:102C7000013BFF315A1C0AD09E225200A654E25D4D
:102C8000581ED2B2002ADBD162540300F2E7684634
:102C90000193FFF744FF2000FFF77EFF63681A6887
:102CA0006B69DBB208335B01D3187F22DA71CCE7A2
:102CB000F7B5070068463C00FFF72AFF0026FF2211
:102CC000019BFC34013B0DD3E0682169884204DBA1
:102CD000E6682069961B3618F4E72669E168761ADB
:102CE000013EEFE768460193FFF719FFE369684685
:102CF000002B52D1FFF70CFF9621019B4900013BAD
:102D00005A1C0CD07D5C5A1EEDB2002D05D16846D0
:102D10000193FFF704FF2800FEBD1300F0E76846AB
:102D200001930025FFF7FBFEFF21A36AB54214D0F3
:102D3000E26A9A4211D95A1CA262626AD3181878C0
:102D4000E36822690133C0B20B40934203D0E268CA
:102D5000BA181072E3600135E7E7E26A9A42DAD105
:102D60000023A3620133E36168469624FFF7D0FE97
:102D700064003E220021019BFF32013B581CC6D05B
:102D80003955B85C5E1E002805D0B954380001934F
:102D9000FFF702FFEDE73300F0E7FFF7B9FE9E21F2
:102DA000019B4900013B5A1C06D07D5C5A1EEDB2C6
:102DB000002DACD01300F6E7684601930025FFF71D
:102DC000AEFEFF21A36BB54202D0E26B9A421DD842
:102DD000E26B9A429FD100236846A363E3619E247D
:102DE000FFF796FE64003E220021019BFF32013B6B
:102DF000581C00D18BE73955B85C5E1E002817D0EF
:102E0000B95438000193FFF7C7FEECE75A1CA263E0
:102E1000626BD3181878E36822690133C0B20B40A3
:102E2000934203D0E268BA181072E3600135C9E733
:102E30003300DDE710B50400FFF73AFF2300FC3351
:102E40001969DA68914203D01B69E418207A10BD31
:102E500001204042FBE710B50400FC34FFF728FFD7
:102E6000E0682369C01A01D50130FF3010BDF0B50C
:102E700085B0019200910500FFF71AFF02A8FFF745
:102E800047FE01200024FF26039B40425A1E531C8C
:102E90001FD02B00FC3301998C4218D2D9681F69CE
:102EA000C91B01D50131FF31002910D01969DF6834
:102EB0008C460100BC4506D019691F6969180137A5
:102EC0003740097A1F61009F39550134E3E7013A21
:102ED000DDE702A80392FFF722FE200005B0F0BD57
:102EE00037B56B46DC1D00230D0020002370FFF773
:102EF0001FFD2B681818286001F098F8210001F0D8
:102F000051F82B681818286020783EBD02220B006B
:102F100010B593430C00012B0BD10D4B08341B68EB
:102F200064011C19802321795B420B432371E271F8
:102F300010BD01F07BF8210001F068F80028F7D0FF
:102F4000034B08341B6864011C197F23E371EFE70E
:102F5000440E002070B50024364B012105000B20E3
:102F60001C70FFF70DF801210B20FFF739F8324BE9
:102F700001210C201C70FFF703F801210C20FFF742
:102F80002FF820232D4A0F20D1690B43D361012252
:102F90002B490B7813430B702A4B19788143197016
:102FA00006211C782143197027490C7822430A70A6
:102FB0001A7802401A70602219780A431A70234B5B
:102FC000234A5A805A78D209FCD12248FEF7FEFDE6
:102FD000214C7F26200001F03BF8200001F050F842
:102FE0000C2008232168CA7882431343CB70032145
:102FF0002268D3788B4301390B43D370226813784E
:103000003340137004232268167833431370226808
:10301000C1241389A40083431048138103591B0260
:103020001B0A035180230360137819430123117095
:103030002B7070BDAD090020AC09002000040040D9
:10304000584400413C44004159440041000C0040B8
:10305000064000008D3A0000440E002000E100E030
:103060000078002810D00121084B1B681A898A4378
:103070001A810822198B0A431A830422198B0A43E6
:103080001A830022024B1A607047C046440E00208B
:103090003C0E002010B50F4A93699B0B9B03936174
:1030A00013680222FF331A729879823A02439A71A6
:1030B0001A7A9207FCD57F24074A2140937A0800A8
:1030C000A3431900802301439172917A5B420B4321
:1030D000937210BD440E00200050004110B50B79D2
:1030E0000C00002B0CD10800FFF730FC002801D0A9
:1030F000012010BD094A93699B0B9B039361F7E77D
:1031000000F094FF210000F071FF0028F0D1034A85
:1031100093699B0B9B039361EBE7C046440E002031
:10312000F8B50D00832A19D1CBB2434C5A01A2182D
:1031300091694248AD010840C02189050143916170
:103140003F4920686D187021083355615B011A5C96
:103150008A43110040220A431A54F8BD022A65D15D
:10316000384B8A00D058002802D003689B699847E2
:10317000A020400000F0F0FE80270600324B7F00C8
:1031800003602D4B002143603A00083005F077F8CA
:10319000340096220023FC345200E360A3622361D2
:1031A0006561E361A7612362E362B3541032A363F4
:1031B000E363B3543E223800FF32B35405F042F8C3
:1031C0006062380005F03EF82B006063FF201A496A
:1031D00003405A018A189168184F08330F40C021E4
:1031E0008905394307279160134A5B011168AD00D7
:1031F0005A5CBA43170003223A435A546169736810
:10320000014049015918636A4B60736862691B6821
:10321000024052019B1801221B18997A30000A4380
:103220009A72FFF7B9FC074BEE5096E711002800A1
:10323000FFF7FEFB91E7C046440E0020FFFFFF8F23
:10324000B80900209009002030CC000070B50500BE
:103250000124064BA200D258002A06D021002800E3
:103260000134FFF75DFF0A2CF3D170BD6000002030
:103270000B4BCAB20B488901C9185301C3185961D5
:1032800099690832890B89039961036852019A1878
:103290000223D3715179823B0B4353717047C0466F
:1032A000B8090020440E0020084B8A00D05810B501
:1032B000002803D00368DB68984710BDC9B2044BEF
:1032C0004901591888688004800CF6E790090020AD
:1032D000440E002010B50C00FFF7E6FF00280CD0CC
:1032E000064BE4B21B68083464011C198023627920
:1032F0005B42134363710223E37110BD440E00204F
:1033000070B5CBB2124A13485C01890189180219C1
:1033100051609168104D08330D4080218902294386
:10332000402591609168890B8903916001685A0179
:103330008A1816793543157195796D06FCD55B01B0
:10334000C918CB79DB07FCD500198068C0B270BD05
:10335000780B0020440E0020FF3F00F070B51400F1
:1033600040220B4B0D001B68FF3359790A435A71F9
:103370000021FFF7C5FFA04200D920000023054926
:10338000A34203D0CA5CEA540133F9E770BDC046DA
:10339000440E0020780B002010B5C9B20B4849013B
:1033A000421893689B049B0C3F2B0BD99468403BBD
:1033B0009B04A40B9B0CA4032343936041188868CF
:1033C000C0B210BD93689B0B9B03F6E7440E002030
:1033D000F0B51C002F4B85B01B6806000D00019254
:1033E000002B54D02C4F3978C9B2002902D10C20BF
:1033F000FEF7F6FD64233B70284BAA00D058002846
:1034000008D0036822005B680199984704002000F7
:1034100005B0F0BD29003000FFF746FF844204D913
:1034200029003000FFF740FF040029003000FFF7BB
:10343000B3FF0121EBB21A4F03935B010293029A8F
:103440003B6801989B18FF335A7A0A435A72154B0E
:10345000A901C918220004F009FF002CD7D02900C7
:103460003000FFF721FF0028D1D14021039B3A68AB
:1034700008335B01D3181879014319710121D971FF
:10348000029BD318FF339A7A0A439A72BFE701244A
:103490006442BCE73C0E0020AC09002090090020EB
:1034A000440E0020780B002013B56B46DC1D220073
:1034B0000123FFF78DFF012801D1207816BD0120DF
:1034C0004042FBE7F0B51E003A4B85B01B680F0089
:1034D0000192002B3FD08023DB019E423BD8364C2B
:1034E0002178C9B2002902D10B20FEF779FD6423AF
:1034F00000252370314BBA01D3180293002E2CD033
:103500002F4B1B680393FF233B401C0000930834A0
:10351000039B64011C19A379DB0921D0294B2A499B
:10352000186801F0F9FE294B1721584301F0F4FE09
:10353000274BE279920713D4DA5D002A01D10138D2
:10354000F7D20122DA55009B5A011D4B9B189A694C
:10355000920B92039A6101256D42280005B0F0BDDF
:1035600000221B4B3400DA55402E00D940242200A3
:103570000199029804F07AFE009BA1045A01104BB5
:10358000890C9B18029A2D195A619A69361B920B65
:1035900092030A439A61009B039A08335B01D31894
:1035A0000222DA715979823A0A435A71019B1B1936
:1035B0000193A3E73C0E0020AD090020B8090020CC
:1035C000440E00200400002040420F007011010052
:1035D000AF09002070B50D001C000D4BAE01F618B0
:1035E00011003000220004F041FEEDB209496D01E6
:1035F0004D196E61AB69084A20001340AB61AB699D
:10360000A2049B0B920C9B031343AB6170BDC0469D
:10361000B8090020440E0020FF3F00F0F7B5104B22
:1036200001901B780F001500002B0CD10D4B1600DC
:103630001C78002C09D00C4E0C48348820186419D2
:1036400004F014FE34802800FEBD002EFBD03A1991
:10365000330000210198FFF7BDFF2418361AF4E764
:10366000380D0020390E00203A0E0020390D0020C0
:10367000F8B5002000AF0E001500012A27D9D31D90
:103680006A46DB08DB00D31A9D46080005F078FE89
:103690006C46032302220021013040002070637039
:1036A000AA420DD2307800280AD0531CDBB2013672
:1036B000A0549D4203D00232E154D2B2F0E72A0076
:1036C00021000448FFF7AAFF431E9841C0B2BD463F
:1036D000F8BDC0468C090020F0B50024012685B055
:1036E000184B0F0069461E7005000094FFF7F8FBA9
:1036F000154B01A90B806A3BFF3BCB716E3B0B72F4
:10370000009B8C7109334B800E4B4E7108711C70FD
:103710003A00092F0FD00D4F09223E700C4E2800A1
:1037200000943480FFF77AFF69462800FFF7D8FB42
:10373000328808493C702800FFF770FF012005B06F
:10374000F0BDC046380D002009020000390E0020EF
:103750003A0E0020390D0020F0B5CF7893B0050067
:103760000E00022F09D1C9882D48FFF7B5FF441E6E
:10377000A041C4B2200013B0F0BD00F057FC3100EE
:1037800000F024FC002803D0C417241AE40FF1E74A
:10379000012F0FD1F288082A0AD02249112A13D802
:1037A000D2B2002A10D02800FFF738FF0124E1E749
:1037B0001D49F5E70400032FDCD1B378002B05D1B8
:1037C000F2881A49032AEBD90A78ECE7022B06D1D2
:1037D000B27917492800FFF74BFF0400CAE7012B15
:1037E00002D1B2791349F5E7032BC3D1124B01A9DA
:1037F0001868FFF703F9114B03A91868FFF7FEF8E3
:103800000F4B05A91868FFF7F9F80E4B07A91868C0
:10381000FFF7F4F86B460533DC77B27901A9D9E7F5
:103820008C09002068CC00007ACC00005ECC00003F
:1038300050CC000062CC00000CA0800040A08000B2
:1038400044A0800048A0800037B5040048780D00EF
:103850000B2810D801F056FD061B0F2B0F40456DAD
:10386000494C6669097801AA002906D10223118012
:103870002000FFF7AFFE01203EBD002313802E4B3A
:103880001B78012B00D1137002230021F0E78A7806
:103890000023012A03D101AA1380284BF0E7264A0E
:1038A0001370274A93699B0B9B039361E3E78D7821
:1038B000012D06D10021214B01AA1D7011702B0092
:1038C000D6E70120002DD7D11B4B1D4A18709369F4
:1038D0009B0B9B039361CFE789782000FFF7DAFB0E
:1038E000C9E72000FFF738FFC6E70123154ACCE7F8
:1038F0000B780020DB06BFD12000FFF7A7FC2A20B1
:10390000AA78104BFF301A6002230D4A11680C5C34
:1039100023434A240B54FF340B5D2938FF380343FB
:103920000B55D4E70123084AAFE78A78064B1A60A3
:10393000B7E70020A0E7C046AE090020B609002086
:10394000440E00203C0E0020400E0020474BF7B5EF
:103950001C780600002C7CD1454D2B689B8B1B07E7
:103960000ED521002000FFF763F82A68102311000C
:10397000FF31887A03438B723E4B1C60082393838C
:103980002B689A8B52071FD504229A833A4A1378E0
:10399000002B0AD01378013BDBB213701378002B95
:1039A00003D101210B20FEF71BFB344A1378002BB7
:1039B0000AD01378013BDBB213701378002B03D1CC
:1039C00001210C20FEF70CFB2B68FF331A7AD2067C
:1039D0001ED510221A72597930320A435A71602367
:1039E000274930000A781A4234D1FFF72DFF2B689F
:1039F000FF33002831D08022997952420A439A71CC
:103A00001A7A520604D540221A72597A0A435A7217
:103A1000012427002B681B8CA343DBB20193019B7D
:103A200023413B4212D023002A6808335B01D3189C
:103A3000DA79D20702D4DB799B0707D5114BA200B4
:103A4000D05800280DD003681B6898470134082C13
:103A5000E5D1F7BDFFF742FBC9E720210A4A917182
:103A6000CEE7E1B23000FFF751FAEFE7390E002060
:103A7000440E00203C0E0020AD090020AC090020BF
:103A8000780B002090090020FF50004110B502483B
:103A9000FFF75CFF10BDC0468C090020014B024AB5
:103AA0001A607047440E002000500041012070470A
:103AB00010B50368014A1B6A984710BD1304000043
:103AC0000300FC33D9699A69914203D0DB69C018BD
:103AD000007D704701204042FBE710B504000069FB
:103AE000FEF738FC22000023FC329361D36186226A
:103AF0009200A4186360A36010BDF020014030392B
:103B0000484248417047F0231B011940802306209A
:103B10009B0099420AD00133FF330130994205D00E
:103B2000802302385B00994200D0002070470F20AC
:103B300001400020012903D00239481E8141481C60
:103B4000704700008923F0B5182685B002919B00CC
:103B50000400C05C330008214343324D1700EB18CA
:103B60005956FEF781FA304B0821E05C330043439D
:103B7000EB185956FEF778FA2C4BE25C0393022AB5
:103B800009D11133E05CFF2805D008214643AE1966
:103B90007156FEF769FA8A26B600A05DFF2819D093
:103BA0000121FEF7EDF91822A35D21495A43AB56D6
:103BB000AD18DB0158188B21890060501D49012286
:103BC0005B188C218900635069688A408D218900C7
:103BD00062501A600122029B11002069FEF79CFDD1
:103BE00039002000FFF78FFF390005002000FFF7A4
:103BF0009EFF390006002000FFF77FFF3300009092
:103C0000290020690122FEF775FB0B4B2069E25C5D
:103C1000039BE15CFEF78BFB2069FEF7A8FB05B078
:103C2000F0BDC04634CA0000250200002702000093
:103C3000184400411444004126020000802210B5BF
:103C400004005200002104F01AFB23000022FC3380
:103C50005A6020009A6010BDF7B51D0008AB1B78B4
:103C60000400009309AB1B78160001930023436006
:103C7000FA239B008360114B0F000833036014305C
:103C8000FFF7DCFF20001D30FF30FFF7D7FF89234F
:103C90006A469B002761E654094B1278E554094BAC
:103CA0002000E2546A46084B1279E2548A22293BEA
:103CB000FF3B9200A3541032A354FEBD8CCC0000F5
:103CC0002502000026020000270200000300FC334A
:103CD00059689A68914204DB5A689868801AFF30E4
:103CE000704798685B68C01A0138F9E710B51D3055
:103CF000FF30FFF7EBFF10BD030070B5FC33D9694F
:103D00009A69040091421AD0DA698218157DDA693D
:103D10000132D2B2DA618A239B00E35CFF2B0CD024
:103D200020001430FFF7D2FF0A2806DD8C238D22F5
:103D30009B009200E358A2581A60280070BD01252C
:103D40006D42E8E70300FC3358689B68C01A01D550
:103D50000130FF30704710B5040020001D30FF30E7
:103D6000FFF7F0FF0028F8D12069FEF70AFB10BD2D
:103D700010B51430FFF7E6FF10BD10B50400006960
:103D8000FEF71BFB002805D02069FEF726FB206903
:103D9000FEF718FB2069FEF700FB002820D0206901
:103DA000FEF71BFB2200FC329369D1690133DBB2C1
:103DB0008B4203D091696118087593618A239B0037
:103DC000E35CFF2B0CD020001430FFF77FFF0928A5
:103DD00006DC8B238D229B009200E358A2581A60C8
:103DE0002069FEF7F5FA00281AD020001D30FF30B8
:103DF000FFF7A8FF002822D086239B00E3189968CC
:103E00005A68914218D08E219A684900A218515CD4
:103E10009A680132D2B29A60C9B22069FEF7E1FA1B
:103E20002069FEF7BFFA002805D02069FEF7BEFA28
:103E30002069FEF7AEFA10BD01214942ECE7206986
:103E4000FEF7DBFAECE7000070B5040000690D0036
:103E5000FEF7BEFA00283ED1FF2686239B00E3181A
:103E60005A689968013232408A4223D1EFF31083B5
:103E7000DB0710D41E4B5B68DB05DB0DEDD0103B80
:103E80005BB2002B10DA0F221340083B9B08194A43
:103E90009B009B181B682069FEF79AFA0028DCD06B
:103EA0002000FFF76AFFD8E79B08C033124A9B0047
:103EB0009B58F0E75A68013216409A68964205D03E
:103EC0008E215A684900A21855545E602069FEF799
:103ED00090FA012070BD20001D30FF30FFF732FF47
:103EE0000028B9D129002069FEF77BFAF1E7C04626
:103EF00000ED00E01CED00E000E100E07047000094
:103F000010B5FCF7F9F9FCF72FFAFDF7B7FE034BF4
:103F1000002BF8D000E000BFF5E7C046000000002D
:103F200010B5FFF7EDFF000010B5FDF775FF04F0C9
:103F300065F9FFF7E3FF0120FDF77EFE054C200049
:103F4000FFF708F82000FFF78BF8FFF7E9FF0020E4
:103F500010BDC0468C09002010B504F073F910BDE7
:103F600010B504F079F910BD10B50200EFF310811F
:103F700072B60A4B1868002801D109481860186801
:103F80008218EFF30884A24204D21A60002900D1FB
:103F900062B610BD01204042F8E7C046480F00203D
:103FA000640F002070B50E0000254468002C0BD073
:103FB000236831005B6820009847002802DB2D1839
:103FC000E468F3E701256D42280070BD70B50D006F
:103FD0004468002C08D0236829009B68200098477B
:103FE000002802D1E468F4E7200070BD70B50D0030
:103FF0004468002C08D0236829001B6820009847DB
:10400000002802D1E468F4E7200070BD70B50D000F
:104010004468002C08D023682900DB6820009847FA
:10402000002802D1E468F4E7200070BD0121054AB0
:1040300010B5136804480B4003D1044C436004805E
:10404000116010BD4C0F0020500F00200204000032
:1040500070B50400012304CC0500117820000B4347
:10406000137080220021520004F009F92B689A781D
:10407000D207FCD49A789207F9D45C6270BD000034
:104080001F22144BF0B51B68590B9C0C9B0111406F
:1040900014405B0F914200D105211F2C00D1023C3E
:1040A000072B00D1043B02688F01158D0A491F269A
:1040B00029403943118505683440298D0A00B243EF
:1040C00022432A8500681903028D044B13400B43D9
:1040D0000385F0BD246080003FF8FFFFFF8FFFFFE6
:1040E00010B5FFF73DFF10BDF0B557464E46DE4612
:1040F0004546E0B58FB01D0006000F00140000F02B
:10410000ADF9CE4B009001919A461B785BB299466F
:1041100001333ED022002B002000290003F088FD4F
:104120008346002835D132003B003000390003F0CF
:104130007FFD00220390002800D06FE000233000B4
:10414000390001F06FFA00282CD000220023200053
:10415000290001F067FA8346002800D192E004AB01
:104160009846012342460493B54B53604346039A55
:104170001C615D611A629E60DF604246002300247C
:104180009361D4614B46002B67D00023AD4C009364
:104190000194009801990FB03CBC90469946A24604
:1041A000AB46F0BD0098019900F09AFF81460028C7
:1041B00000D19AE0009801990022002301F032FA20
:1041C0000028E6D03000390000F08AFF0028E0D057
:1041D0002000290000F084FF0028DAD004AB9846C4
:1041E000042342460493964B1461556153600023A7
:1041F0000024136200239361D46153461B789660B8
:10420000D7605BB2022B04D0404600F073FF002859
:1042100029D103F0DDFF2223036024E000232000E6
:10422000290001F0FFF90028B3D004AB9846012320
:1042300042460493824B4146536043465A461A62B3
:1042400000229E60DF601C615D617E4B8A61CB61F4
:10425000009201934B46022B9BD0404600F04AFF50
:10426000002800D18AE043461B6A002B04D003F0EB
:10427000AFFF43461B6A03604346DC699B690093BA
:10428000019486E72000290000F02AFF002800D1D1
:104290007FE7002200232000290001F0C9F900284F
:1042A00000D176E704AB9846012342460493644B61
:1042B000536043465A469E60DF601A621C615D612E
:1042C00053461B785BB2002B5DD0002042465E490E
:1042D0009061D161022B5BD103F07AFF212303604F
:1042E00043461B6A002BC7D0C1E73000390000F0FD
:1042F000F7FE002800D15DE72000290000F0F0FE65
:10430000002800D156E70098019953461B78020017
:104310005BB29B460B0003F08BFC04AB9846002875
:1043200062D1032342460493454B146155615360A7
:1043300010629660D760454B20002900002202F0F1
:10434000BDFE5B4604000D00002B27D1E022414654
:104350003F4B12068A61CB613000002200233900F6
:1043600001F066F900282AD1404600F0C3FE00287B
:10437000B6D103F02DFF22230360B1E703F028FF3D
:10438000212303606FE74246002300249361D46138
:10439000404600F0AFFE0028A2D19DE70022414632
:1043A0002C4B30008A61CB6100220023390001F0E0
:1043B0003FF9002835D15B46022BDAD0D4E7200044
:1043C000290000F09FFE22002B0001F02BF90028AD
:1043D00005D1E022204B120641468A61CB6153464B
:1043E0001B785BB29B46E6E7012342460493144BDD
:1043F000536043464A469E60DF601A621C615D61FD
:104400005B46002BBFD0002300221900100002F0F1
:104410004BFA43469861D9615B46022B00D15BE7BA
:10442000B6E72000290000F06DFE22002B0001F00D
:10443000F9F80028D3D10022034BCDE788000020F3
:10444000C0CC00000000F03F0000F0FF0000E03FA3
:10445000FFFFEF470000F07FFFFFEFC7F0B55746C3
:10446000DE464E4645465C006408E0B598461F00AF
:10447000230093B083468A46160013430CD07D4B2D
:104480004D00029181466D089D4212DD7A4B9C469B
:104490005B4665441D4361D10023784C0093019431
:1044A0000098019913B03CBC90469946A246AB4691
:1044B000F0BD9D4250D09C42E8DC6E4B9C426BD0DC
:1044C000002304935346002B69DB002A10D1694B6B
:1044D0009C424CD0694B9C4200D1A3E08023DB0579
:1044E000984500D1BCE0664B984501D100F0D6FB61
:1044F0005846514600F0F0FD4B4600900191002BCC
:1045000007D1002D67D053465C4A9B009B0893421D
:1045100061D05346DB0F013B99464A46049B134347
:1045200000D190E0574B9C4200DCBBE0564B9C42D4
:1045300001DC00F010FC554B9D4201DC00F004FC56
:104540004346002B23DD524A524B1000190002F063
:10455000B5FD00900191A3E7002805D04E4800F07A
:10456000CBFD009001919BE7AC42F7DCA5E75A46F2
:10457000414BEB18134300D18EE7444B9D4200DCC6
:1045800099E3434600960197002B00DB88E7002360
:1045900000240093019483E7002A91D076E73F4BF3
:1045A0009C423CDC394B9C428FDD3D4923158C46B7
:1045B0006344142B00DCB2E33421CB1A3100D94020
:1045C00008009840904200D07FE701231940013352
:1045D0005B1A049379E74346002B07DA009A019BA4
:1045E0000020264902F060F900900191029B002B07
:1045F00000DB55E7204B9C46049B65441D4301D1DD
:1046000000F00EFC049B012B00D049E7009C019DAB
:104610008021220009066B180092019340E70223D3
:10462000049352E758465146434600900191002BAF
:1046300000DB35E75A4653460020104902F034F9B2
:10464000009001912CE75A4653465846514602F0D5
:10465000A7FF02000B0002F027F9009001911FE76D
:104660005A4653465846514602F028FD00900191A3
:1046700016E7C0460000F07F000010C00000F03FC9
:104680000000E03F0000E0410000F043FFFFEF3F8B
:104690009C7500883CE4377EC4CC0000FFFF3F439C
:1046A00001FCFFFFE44B00229D420ADC00980199C7
:1046B0000022E24B02F002FD35220D000090019134
:1046C0005242DF492B158C46634498462D03DD4C3E
:1046D000DD4B2D0B90442C439D420ADDDB4B9D426C
:1046E00001DC00F001FC01239C46D94BE0449C46D0
:1046F0006444002200230E920F9310921193002223
:104700000025D04B0692079300980199069A079BC3
:1047100021000890099102F043FF069A079B0A9036
:104720000B910898099901F0A3FD02000B000020ED
:10473000C44902F0B9F80A00010013000C910D926F
:1047400002000A980B9902F0B9FC0A00010013005C
:1047500002910392002200920193802364109B0532
:10476000234380242403A4460020634459190400F1
:104770000D0002000B000098019902F09FFC02005E
:104780000B000A980B9902F00BFF069A079B0A9000
:104790000B912000290002F003FF02000B00089893
:1047A000099902F0FDFE009A019B02F087FC0200CD
:1047B0000B000A980B9902F0F3FE0C9A0D9B02F085
:1047C0007DFC029C039D0890099122002B00200093
:1047D000290002F073FC04000D009E4A9E4B02F07B
:1047E0006DFC9E4A9E4B01F043FD22002B0002F01F
:1047F00065FC9C4A9C4B01F03BFD22002B0002F023
:104800005DFC9A4A9A4B01F033FD22002B0002F026
:1048100055FC984A984B01F02BFD22002B0002F02A
:104820004DFC964A964B01F023FD2200069007911D
:104830002B002000290002F041FC02000B0006982A
:10484000079902F03BFC009A019B04000D000298BE
:10485000039901F00DFD089A099B02F02FFC22003C
:104860002B0001F005FD009C019D0A900B91220098
:104870002B002000290002F021FC0022814B0400C3
:104880000D0001F0F5FC0A9A0B9B01F0F1FC0022EF
:104890000B0011001A00069107920A000098019976
:1048A00002F00CFC00220C900D9106980799754BB4
:1048B00002F076FE22002B0002F072FE02000B00D6
:1048C0000A980B9902F06CFE029A039B02F0F6FB29
:1048D000069A079B04000D000898099902F0EEFB68
:1048E00002000B002000290001F0C2FC04000D00B2
:1048F00002000B000C980D9901F0BAFC0022100088
:10490000E022614B12060090019102F0D7FB0C9A55
:104910000D9B029003910098019902F041FE020064
:104920000B002000290002F03BFE584A564B02F0D3
:10493000C5FB574A04000D0000980199554B02F041
:10494000BDFB02000B002000290001F091FC109A31
:10495000119B01F08DFC06900791404603F0BAF9D7
:10496000069A079B04000D000298039901F080FC51
:104970000E9A0F9B01F07CFC22002B0001F078FCCA
:10498000002022002B000090019102F009FE0E9AF7
:104990000F9B02F005FE029A039B02F001FE02004B
:1049A0000B000698079902F0FBFD069007914A4616
:1049B000049B013B134300D188E10023214C029367
:1049C000039400223B0030003900140002F0E8FD9F
:1049D000009A019B02F072FB32003B0004900591AB
:1049E0000698079902F06AFB02000B0004980599EB
:1049F00001F03EFC3D0006000F00009801992200E6
:104A00002B000496059702F059FB02000B003000C2
:104A100039000092019301F02BFC1F4B04000D00A4
:104A20008B460200994200DC55E11C4BCB18034336
:104A300000D0FBE134E0C046FFFF0F000000404320
:104A400001FCFFFF0000F03F8E98030079B60B00D9
:104A50000000F0FFEF4E454A287ECA3F65DBC99350
:104A60004A86CD3F01411DA96074D13F4D268F512B
:104A70005555D53FFFAB6FDBB66DDB3F03333333AB
:104A80003333E33F0000084009C7EE3FFD033ADC43
:104A9000F5015B14E02F3EBEFFFF8F40000070BFAA
:104AA00004980599E84AE94B01F0E2FB009A019B62
:104AB00006000F002000290002F072FD02000B002A
:104AC0003000390000F0C8FDAA46002800D0ADE152
:104AD0008024DF4A53469446640322001B15634436
:104AE0001A411300DB495B445A001E001B038C462D
:104AF0001B0B23431424520DD74D62441541A21AB7
:104B0000134199465B46AE4300203100002B02DA88
:104B10004B465B42994602000B000098019902F057
:104B20003FFD4B461B0500900191020098460B008B
:104B30000498059901F09CFB0D0000240022C74B4E
:104B40002000290002F0BAFA009A019B0690079112
:104B50002000290002F024FD02000B0004980599B2
:104B600002F01EFDBE4ABF4B02F0A8FABE4A060084
:104B70000F00BE4B2000290002F0A0FA02000B003B
:104B80003000390001F074FB04000D0002000B003E
:104B90000698079901F06CFB069A079B06000F0028
:104BA00002F0FEFC02000B002000290002F0F8FCDD
:104BB0003200009001913B003000390002F07EFA93
:104BC00004000D00AA4AAB4B02F078FAAA4AAB4B9C
:104BD00002F0E6FC22002B0002F070FAA84AA94B72
:104BE00001F046FB22002B0002F068FAA64AA74B10
:104BF00002F0D6FC22002B0002F060FAA44AA54B7A
:104C000001F036FB22002B0002F058FA02000B00E4
:104C10003000390002F0C4FC04000D0002000B005B
:104C20003000390002F04AFA8023049005910022F6
:104C3000DB052000290002F0B3FC02000B00049801
:104C4000059901F031FE009A019B04000D0030002F
:104C5000390002F033FA009A019B01F009FB0200CF
:104C60000B002000290002F09BFC32003B0002F008
:104C700097FC02000B000020874902F091FC43469C
:104C80005B181A15002A00DC3FE11900029A039B09
:104C900002F014FA00900191FFF702FC5346002B3A
:104CA00001DAFFF725FC5846514600F03DF9009027
:104CB0000191FFF7F5FB4346002B00DB67E48023FF
:104CC0001B06FB1800960193FFF7EAFB0023734CC9
:104CD0000293039475E64B005B089A46704B9A4525
:104CE00000DCF9E06F4B5B441A430AD1009A019B48
:104CF00002F056FC049A059B00F0B8FC002800D195
:104D0000E6E602980399684A684B02F0D7F9664ACA
:104D1000664B02F0D3F900900191FFF7C1FB002A26
:104D200001D0FFF7E5FB1432D31A22001A4111001B
:104D30009940A14201D0FFF7CDFB01231A40DB18B7
:104D40009B1A0493FFF7C6FB4346002B01DBFFF7DA
:104D50001EFCFFF7F8FB564B9D42F5DD4E4B9D4286
:104D600001DDFFF7EDFB0098019900224A4B02F0AC
:104D700017FCC0224F4BD20504000D0002F09EF933
:104D80004D4A029003914D4B2000290002F096F904
:104D90000022009001914A4B2000290002F08EF978
:104DA00002000B004748484902F0FAFB22002B00A2
:104DB00002F084F902000B000020444902F0F0FBED
:104DC0002200069007912B002000290002F076F9BE
:104DD00002000B000698079902F070F91A4A354B49
:104DE00002F06CF902000B000098019902F0D8FB68
:104DF00002000B0004000D000298039901F038FA3C
:104E0000029A039B00200090019102F0C9FB02006E
:104E10000B002000290002F0C3FB06900791C6E5B5
:104E20000098019902000B00FFF711FC284A294B5A
:104E30000298039902F042F9254A264B02F03EF906
:104E400000900191FFF72CFBFE822B654715973CE4
:104E500002FCFFFF01FCFFFFFFFF0F00432EE63FB8
:104E6000EF39FAFE422EE63F396CA80C615C20BE99
:104E7000D0A4BE726937663EF16BD2C541BDBB3E60
:104E80002CDE25AF6A56113F93BDBE166CC1663F3E
:104E90003E5555555555C53F0000F03F0000F0BF49
:104EA000FFCB904000346F3F59F3F8C21F6EA5014D
:104EB000FEFFEF3F4715F73F44DF5DF80BAE543E72
:104EC0000000D03F555555555555D53F0000E03FA2
:104ED0009C7500883CE4377E00220E4B904691463C
:104EE0009A4500DC29E6F3E580220B4BD2050E92B1
:104EF0000F930A4A0A4B8025109211930022094B06
:104F0000ED0206920793FFF7FFFB4A4600F08AF98D
:104F1000BCE6C0460000E03F03B8E23F06D0CF4306
:104F2000EBFD4C3E0000F83FF8B54746CE46674BD8
:104F300080B50A000F00190005003940994200D1E0
:104F40009BE004000100002F69DD3F1500D1B4E0B3
:104F50005F4B12039C468023120B5B0313435B00E1
:104F6000CA0F67449B184A00F80703D5D20F5B00AD
:104F70009B188A0079108C460021802016248946CF
:104F800080030D189D4202DC29185B1B8144D50F5C
:104F90005B00013C5B1952004008002CF1D100205D
:104FA0008046802020250027000609E08B425CD047
:104FB000D40F5B00013DE31852004008002D16D0CD
:104FC000C4198B42F2DD27180E00002C49DB5B1A56
:104FD000A242894149425B1A121BD40F5B00013D7A
:104FE00080443100E31852004008002DE8D11343FB
:104FF0004ED143465B0837494A46884649465210D7
:105000004244C90702D5802109060B4361460F05BA
:10501000BD18180029000CBC90469946F8BD7B00CD
:105020005B0803433900002BF5D0002F3CD1E30A85
:10503000153A6405002BFAD08020400303423FD18B
:10504000002700E00F005B00791C0342FAD0250026
:1050500020208D40401A2900D71B2200C2401A434D
:1050600076E7FE43F60F8E19B1E79442A0D82718D1
:10507000002CF6DB1E000023AEE702003B002800F8
:10508000390002F01BF82A003B0001F0F1F8C2E7FA
:105090004346013303D0434601335B08ABE70123AA
:1050A00098460023C144A6E73B00020002F078FACC
:1050B00002000B0001F0F8FBADE713000022BBE794
:1050C0000127210020207F42C6E7C0460000F07F74
:1050D00001FCFFFF0000E03F49004B08190070474A
:1050E000034B48009C4640086044C00F7047C046D0
:1050F0000000108000207047002001497047C04622
:105100000000F87FF0B5C64600B5CB0F9846404A80
:105110004B005B0D9A1882B00D000400132A2FDC9F
:10512000002A49DB3B4F17413E000E40064323D087
:105130007F08390029400C430AD03749BD438C46CB
:1051400063445C425C418023DB021341E4071D435E
:105150004146CE0031492B008E1922003468756813
:105160002000290001F084F8009001910098019935
:1051700022002B0002F014FA02B004BC9046F0BDED
:10518000332A08DD8023DB009A42F5D102000B00B0
:1051900001F06EF8F0E7224A94460122634452423D
:1051A000DA400242E8D052080242D1D09443802231
:1051B000D2051A411443CBE74B005B080343DBD015
:1051C0000B031B0B1C436342234380244D0C24031D
:1051D0001B0B23406D042B4319004346DA000F4B91
:1051E0009B181C685D6802000B002000290001F07C
:1051F0003FF8009001910098019922002B0002F0E5
:10520000CFF942464B005B08D60733431900B3E79A
:1052100001FCFFFFFFFF0F00EEFBFFFFC8CC00000B
:10522000EDFBFFFF4B0070B55B0D14000A00002B77
:105230001AD14B005B08034315D0234B002201F029
:105240003DFF224B9C422DDB0A004B005B0D363BA1
:105250001F4DE318AB422ADC002B0DDD1D4C1B0556
:1052600022401A43110070BD1B4DAB42F0D1020029
:105270000B0000F0FDFFF6E71D00353519DA174B7E
:1052800002009C4209DD0B001548164900F032F877
:10529000134A144B01F012FFE5E70B0012481349C3
:1052A00000F028F8104A114B01F008FFDBE702007C
:1052B000E9E7084C363322401B051343190000224E
:1052C0000B4B01F0FBFECEE700005043B03CFFFF6C
:1052D000FE070000FFFF0F80FF07000050C3000023
:1052E0009C7500883CE4377E59F3F8C21F6EA50117
:1052F0000000903C30B54A00DB0FDB0752081A4330
:10530000110030BD02B4714649084900095C4900EA
:105310008E4402BC7047C046002243088B4274D3BF
:1053200003098B425FD3030A8B4244D3030B8B42A6
:1053300028D3030C8B420DD3FF22090212BA030CAF
:105340008B4202D31212090265D0030B8B4219D390
:1053500000E0090AC30B8B4201D3CB03C01A5241B0
:10536000830B8B4201D38B03C01A5241430B8B42F8
:1053700001D34B03C01A5241030B8B4201D30B03E1
:10538000C01A5241C30A8B4201D3CB02C01A524108
:10539000830A8B4201D38B02C01A5241430A8B42CB
:1053A00001D34B02C01A5241030A8B4201D30B02B4
:1053B000C01A5241CDD2C3098B4201D3CB01C01ACE
:1053C000524183098B4201D38B01C01A52414309D8
:1053D0008B4201D34B01C01A524103098B4201D3C6
:1053E0000B01C01A5241C3088B4201D3CB00C01A33
:1053F000524183088B4201D38B00C01A52414308AB
:105400008B4201D34B00C01A5241411A00D20146CF
:10541000524110467047FFE701B5002000F0F0F858
:1054200002BDC0460029F7D076E7704703460B431C
:105430007FD4002243088B4274D303098B425FD38D
:10544000030A8B4244D3030B8B4228D3030C8B42B9
:105450000DD3FF22090212BA030C8B4202D312129F
:10546000090265D0030B8B4219D300E0090AC30B74
:105470008B4201D3CB03C01A5241830B8B4201D321
:105480008B03C01A5241430B8B4201D34B03C01A0A
:105490005241030B8B4201D30B03C01A5241C30A82
:1054A0008B4201D3CB02C01A5241830A8B4201D3F3
:1054B0008B02C01A5241430A8B4201D34B02C01ADD
:1054C0005241030A8B4201D30B02C01A5241CDD282
:1054D000C3098B4201D3CB01C01A524183098B42CD
:1054E00001D38B01C01A524143098B4201D34B01B6
:1054F000C01A524103098B4201D30B01C01A524119
:10550000C3088B4201D3CB00C01A524183088B429F
:1055100001D38B00C01A524143088B4201D34B0088
:10552000C01A5241411A00D20146524110467047FA
:105530005DE0CA0F00D04942031000D340425340FF
:1055400000229C4603098B422DD3030A8B4212D3BF
:10555000FC22890112BA030A8B420CD389019211F1
:105560008B4208D3890192118B4204D389013AD02E
:10557000921100E08909C3098B4201D3CB01C01A03
:10558000524183098B4201D38B01C01A5241430916
:105590008B4201D34B01C01A524103098B4201D304
:1055A0000B01C01A5241C3088B4201D3CB00C01A71
:1055B000524183088B4201D38B00C01A5241D9D289
:1055C00043088B4201D34B00C01A5241411A00D20A
:1055D0000146634652415B10104601D34042002B06
:1055E00000D54942704763465B1000D3404201B585
:1055F000002000F005F802BD0029F8D016E770473A
:105600007047C0468446101C62468C46191C63468F
:1056100000E0C0461FB501F0E9FC002801D40021DC
:10562000C8421FBD10B501F041FC4042013010BD21
:1056300010B501F0DBFC002801DB002010BD0120CB
:1056400010BDC04610B501F0D1FC002801DD0020DE
:1056500010BD012010BDC04610B501F063FC00284C
:1056600001DC002010BD012010BDC04610B501F0C6
:1056700059FC002801DA002010BD012010BDC046F1
:105680009E2110B5C905041C02F096FC002803D128
:10569000201C00F0CDFD10BD9E21201CC90500F08E
:1056A00003FC00F0C5FD80231B069C466044F2E726
:1056B00070B500220C4B04000D00FFF7D7FF002847
:1056C00004D12000290002F0CFFA70BD064B002261
:1056D0002000290001F064FF02F0C6FA80231B06B7
:1056E0009C466044F1E7C0460000E041F8B54746FB
:1056F000CE4643025B0A4400C20F9C464800DD00D0
:105700004B02240E5B0A000E80B598462600914697
:10571000C90FDB00271A8A4229D0002F15DD002887
:105720004AD1002B00D095E0ED08FF2C00D188E095
:105730006B025B0AE6B25B02F605580A3043D207F9
:1057400010430CBC90469946F8BD002F00D087E06E
:10575000601CC0B2012800DCB6E0EE1A720100D570
:10576000C5E0002E3DD1002200260023E3E7002FF4
:1057700000DC96E000285DD0FF2C60D08022D204AF
:1057800013431B2F00DDECE02022D21B18009340B6
:10579000F8405A1E93410343ED186B017BD5013449
:1057A000FF2C00D1B7E0012207262A406B089A4D52
:1057B0001D4015432E4029E0FF2CB5D08022D20495
:1057C00013431B2F00DDB2E02022D21B19009340AF
:1057D000F9405A1E93410B43ED1A6B015BD5AD01A5
:1057E000AE09300002F0F2FB05388640844265DCE9
:1057F000041B330020200134E340041BA640751E27
:10580000AE41334307261D0000241E4001224B46B3
:105810001A40002E04D00F232B40042B00D0043557
:105820006B0100D480E70134E6B2FF2C2FD1FF26B4
:10583000002380E7002B52D1FF2C00D074E70A0030
:10584000ED08002DF3D08023DB032B435B025B0AC2
:10585000FF2670E7013F002FBED0FF2CB1D163E7D8
:10586000002C47D0FF2869D08024E4047A422543E5
:105870001B2A00DDC5E02C002026D440B21A95403A
:105880006A1E954125435D1B04008946A5E7AB01CF
:105890005B0A50E7002401224B461A406B07BAD13D
:1058A00042E7002F3BD10134E0B201284ADDFF2C52
:1058B000BDD00726ED186D082E40A7E70723574DEA
:1058C000241A35401E40A1E7002C1BD1002D6ED1BB
:1058D000002B00D19AE00A001D003C0024E7013FA4
:1058E000002F00D158E7FF2C00D04AE7A7E75E1B46
:1058F000894676E7002D1CD10A00FF281FD004003E
:105900001D0011E7002D5DD1002B17D1802300224F
:10591000DB03FF260FE70A00FF2600230BE7002C1E
:1059200021D1002D66D1FF28E9D11D0087E7012391
:1059300052E77A1CA7D0FA43FF2899D10A001D002C
:10594000FF24F1E6002E21D1002D4FD0002B4CD0AA
:10595000ED186B019ED5314B07362E4001241D40BA
:1059600054E7012318E7FF28DFD08024E4047F42B6
:1059700025431B2F4DDC2026F61B2C00B540FC4098
:105980006A1E95412543ED18040006E7002DCCD092
:10599000002B00D153E780216046C903084203D0A1
:1059A0004046084200D11D000121114047E7002B6D
:1059B00000D1B9E6EA1A500125D507265D1B2E4015
:1059C000894623E7FF24002B00D1ADE68022604604
:1059D000D203104204D04046104201D11D00894636
:1059E00001224B46FF241A409EE62B00DD080A00E8
:1059F00000249DE67A1CC6D0FF43FF28B9D11D00C4
:105A00001DE701253FE7151E00D044E700220023D3
:105A100091E60125B7E7C046FFFFFF7DFFFFFFFBD3
:105A2000F8B557464E464546DE464402E0B54600C8
:105A30008846640A360EC70F002E63D0FF2E24D08E
:105A40008023E400DB041C43002399469B467F3EF1
:105A5000434642465D02D20F5B006D0A1B0E904624
:105A6000924665D0FF2B55D080220021ED00D20454
:105A70007F3B1543F61A43464A467B400F2A00D91E
:105A80008DE06D48920082589746002C54D108232F
:105A90009946063BFF269B46DAE700255346022936
:105AA0001BD0032900D1BFE0012928D030007F306E
:105AB000002820DD6A0704D00F222A40042A00D0E3
:105AC00004352A0103D530005C4A80301540FE2899
:105AD00003DCAC01640AC2B201E0FF2200246402CC
:105AE000D205600ADB07104318433CBC9046994638
:105AF000A246AB46F8BD0122101A1B287CDD00220D
:105B00000024ECE7002C1DD104239946033B00261A
:105B10009B469DE7FF3E002D20D1022143464A4689
:105B20007B400A430F2AD8D84548920082589746AE
:105B3000002D19D10121F1E70C239946093BFF26DD
:105B40009B4685E7200002F041FA7626431F9C40E1
:105B500000237642361A99469B4679E74A46032344
:105B60001A439146032186E7280002F02FFA431FCB
:105B700036189D40763600217DE780240023E4031B
:105B8000FF22ACE700258023DB031C4228D01D4206
:105B900026D12B435C02640A4346FF229FE7620141
:105BA0006C01A24224D21B210025013E01271000D6
:105BB0006D005200002801DB944201D8121B3D43C6
:105BC00001390029F3D11400621E944125436DE789
:105BD000BA46594625005346022900D061E77CE7C2
:105BE0008023DB031C436402640A3B00FF2276E748
:105BF000121B1A210125D9E79E362A00B5402C0038
:105C0000C240651EAC411443620704D00F222240FB
:105C1000042A00D00434620103D4A401640A0022DF
:105C20005DE7012200245AE78024E4032C43640248
:105C3000640AFF2253E7C046D8CC0000FFFFFFF7FD
:105C400018CD0000F0B54E4657464546DE46E0B555
:105C500043025B0A450083B00F1C99462D0EC60F08
:105C6000002D57D0FF2D24D08020DB00C004184326
:105C7000002381469A469B467F3D7C027A00FB0FBB
:105C8000640A120E984623D0FF2A4BD0E3008024EA
:105C90000020E4047F3A1C43AD186B1C4746019377
:105CA000534677403A000F2B48D87D499B00CB588C
:105CB0009F46002B00D085E008339A46063B9B4662
:105CC0007C027A00FB0FFF25640A120E9846DBD196
:105CD000002C00D090E0524601231A439246012046
:105CE000DBE74C4658461700022824D0032800D191
:105CF000CFE00022002301284DD15802D205400AEE
:105D0000FF071043384303B03CBC90469946A24677
:105D1000AB46F0BD002B5BD104239A46033B002524
:105D20009B46AAE7FF35002C60D1524602231A4356
:105D300092460220B1E7FF220023DEE74B461B0C10
:105D40009C464B462604360C180461463300220C50
:105D50006446000C43434E435043544380191A0C8D
:105D60001218964203D9802149028C4664441B04D0
:105D70001B0C1004C01883015E1EB341800E184333
:105D8000130C1B199B0103431C00230179D501232C
:105D900062081C401443019A7F32002A4DDD6307DC
:105DA00004D00F232340042B00D00434230103D557
:105DB0003C4B019A1C408032FE2ABCDCA3015B0AEA
:105DC000D2B29AE70C239A46093BFF259B4654E73B
:105DD000180002F0FBF84A46431F76259A4000233C
:105DE0006D4291462D1A9A469B4646E7524603233A
:105DF0001A439246032050E7200002F0E7F8431FC1
:105E00002D1A9C40763D002047E780230027DB03C6
:105E1000FF2272E7424666E74C463200584662E788
:105E200080234A46DB031A4222D01C4220D123435E
:105E30005B025B0A4746FF225FE701239A1A1B2A8F
:105E400021DC23000199D3409E318C401A002300AD
:105E50005C1EA34113435A0704D00F221A40042AA0
:105E600000D004335A0111D49B015B0A002244E79D
:105E700080234A46DB0313435B025B0A3700FF22A1
:105E80003BE7019587E70022002336E70122002344
:105E900033E78023DB0323435B025B0AFF222CE70B
:105EA00058CD0000FFFFFFF7F8B54746CE46440047
:105EB000C20F80B547024802400A84466646480041
:105EC0007F0A240EF60025009046FB00000EC90F45
:105ED000B146FF2800D185E001267140261A914283
:105EE00057D0002E43DD002800D07FE0494600292E
:105EF00000D1AAE0013E002E00D0F7E05B1A5A0163
:105F000000D48BE09B019C09200002F05FF805386B
:105F10008440854200DDD3E0451B2300202001356D
:105F2000EB40451BAC40621E9441234307240025EF
:105F30001C40012241460A40002C04D00F21194088
:105F4000042900D00433590100D480E00135ECB2BB
:105F5000FF2D00D0A3E0FF2400235B02E405580AD4
:105F6000D207204310430CBC90469946F8BD002E42
:105F700074D1601CC0B2012800DCA7E04A469C1A1C
:105F8000620100D5B6E0002CBED10022002400231F
:105F9000E3E7002E00DC85E0002846D0FF2C49D046
:105FA00080224846D2041043814601221B2E09DC80
:105FB00020204C46801B84404A462000F240441E6C
:105FC000A04102439B185A0128D50135FF2D00D16D
:105FD000A8E00122072494491A405B080B401343B0
:105FE0001C40A6E7002E00D078E775E7FF2C54D0C0
:105FF00080224946D2041143894601221B2E09DC26
:1060000020214846891B88404A460100F240481E2C
:1060100081410A439B1A5A0100D573E70122414688
:106020000A40590700D089E711E04846002858D1B6
:10603000FF2C0CD1DB08002B00D18CE78020C003A3
:1060400003435B025B0AFF2487E7FF2C25D0DB08B4
:10605000FF2DF0D05B025B0AECB27EE7002C4DD046
:10606000FF2818D08024E404724223431B2A00DD59
:10607000C4E01C002025D440AA1A93405A1E934124
:1060800023434A460500D31A884638E7721CF8D0E5
:10609000F243FF28EAD10A004B46FF25D7E79B01D0
:1060A0005B0A5AE7002E41D1651CE9B2012945DDA2
:1060B000FF2D00D14FE707244B445B081C4038E715
:1060C00007225A4B2D1A2340144032E7002C1DD1D1
:1060D000002B7AD14B46002B00D191E00A0000251D
:1060E000B5E7013E002E19D14B446CE7FF2C84D15B
:1060F000FF25ACE74A468846D41A05E7002BC5D1F0
:106100000A00FF28C8D005004B46A0E7002B49D164
:106110004B46002B77D00A00FF2598E7FF2C00D0D4
:1061200043E787E70A00FF24002316E7002C15D178
:10613000002B57D1FF28E6D14B467BE7002C20D11E
:10614000002B57D04946002953D04B445A0168D5FB
:106150000724364A1C4001251340EAE6FF28EBD00D
:106160008022D204764213431B2E53DC2025AD1B24
:106170001A00AB40F2405C1EA34113434B440500A0
:1061800021E7002BD8D04946002900D152E78021D1
:10619000C9030F4200D14DE76046084200D049E7ED
:1061A0004B4647E74846FF25002800D14FE78022AD
:1061B000D203174204D06046104201D14B468846B4
:1061C00001224146FF250A4041E7484600281FD0EA
:1061D0001A1A500120D54A460724D31A1C40884673
:1061E0000025A6E6741CC9D0F643FF28BCD14B4657
:1061F00020E799464B460025DB082BE7012340E7C3
:1062000000220023A9E680230022DB03FF24A4E66A
:1062100000251CE70123B1E7002AF1D01300002577
:10622000FCE60025FAE6C046FFFFFF7DFFFFFFFB0F
:1062300041024200C30F490A120E00207E2A0DD9E6
:106240009D2A0CD8802000040143952A0ADC962060
:10625000821AD1404842002B00D108007047034AFF
:106260009818FBE7963A9140F4E7C046FFFFFF7F9E
:10627000F0B54F464646D6460C000903C0B5490A5C
:10628000470F5E0039431F03DB0F9C4665007B0A06
:10629000570F1F436D0DE40F760DA146C000B846A1
:1062A000D200AB1B64457BD0002B5FDD002E00D0FD
:1062B000A4E03E00164300D112E15E1E002E00D085
:1062C0009EE1871A4346B84280410125C91A4042DF
:1062D000091A0B0200D431E149024E0A002E00D106
:1062E0006EE1300001F072FE0300083B1F2B00DD61
:1062F00061E120223900D21A9E40D1409F400E43D6
:106300009D4200DD51E15D1B6B1C1F2B00DD7CE11C
:106310002021C91A3D0030008F408840DD40791EA1
:106320008F41310007222843D940002507433A40D6
:10633000002A09D00F233B40042B05D03B1DBB4254
:10634000BF417F42C9191F000B0200D426E26A1C1C
:10635000C64B55056D0D9A4200D106E1C44AFF08AF
:106360000A40530752023B43120B8EE0002B00D031
:10637000B8E06B1C5B055B0D012B00DC30E1871A7C
:106380004346B842B641CB1A76429E1B330200D533
:106390004CE13B003343A1D100220024002570E0F2
:1063A000002B00DCE5E0002E00D183E0AF4EB542CB
:1063B00060D0802636043743B846382B00DC3EE1F7
:1063C000434613431F007A1E97413F18874280417E
:1063D000404209180B0200D4B0E0A44B01359D42A5
:1063E00000D1C3E0A24A7B080A4001210F401F43AD
:1063F0005108D30707221F433A4099E79B4EB54205
:1064000038D0802636043743B846382B00DDDCE030
:106410001F2B00DC30E11E004746203EF740BC4603
:10642000202B04D04026F31A46469E4032431700E4
:1064300063467A1E97411F43CCE0002B00D104E253
:106440004346134300D159E14B07C008184380234A
:10645000C9081B03194208D04546ED081D4204D166
:106460004346D008590708432900420FC9007F4D11
:106470001143C0004B07CA087C49C00803438D4242
:1064800068D012036D05120B6D0D00211203180068
:10649000130B0A0D12051A43764B2D0513402B439F
:1064A0005B00E4075B08234319001CBC9046994637
:1064B000A246F0BD3E00164312D05E1E002E00D054
:1064C00000E1871887428041414440420918012574
:1064D0000B0233D5022585E76446330041461000A0
:1064E0001D00C7E7002D00D0DAE00C000443F3D014
:1064F0005C1C00D19FE15D4CA64200D12FE1DB4343
:10650000382B00DD66E11F2B00DD83E12024050030
:10651000E41A0F00DD40D940A0404346A7405B1A73
:10652000441EA04198462F433843171ABA4292415D
:1065300043465242991A64463500CAE607223A4059
:10654000002A00D0F6E64B07CA084849FF083B433B
:106550008D4296D11900114300D19EE1802109039B
:106560000A431203120B414D8FE71500002200234E
:106570008BE7002B00D0C7E06B1C5F057F0D012F60
:1065800000DCF1E0394DAB4200D1B9E085180A00DA
:10659000854289414244494251180722CF076D087C
:1065A0002F4349083A401D00C2E607223049ED1A40
:1065B00031403A40BCE63E002838864000279FE63E
:1065C000380001F003FD20308EE6434613431F00E0
:1065D0007A1E9741C71BB84280414042091A78E6AB
:1065E0000E003B0006431343002D61D1002E00D066
:1065F000F4E0002B00D11BE164463900100039E7BC
:106600001A4FBB427AD03300FFE630001F3DE8400E
:10661000202B03D04021CB1A9E4037437B1E9F4145
:10662000072207433A400021002589E7171A43460D
:10663000BA42B641591A76428E1B64464EE61F2B6B
:1066400000DDADE020264746F61AB740B9461700F0
:10665000B246DF404E463E4337005646B240561ED5
:10666000B24117434246DA408918AEE6FF07000000
:10667000FFFF7FFFFFFF0F8020264746F61AB74037
:10668000B9461700B246DF404E463E4337005646F5
:10669000B240561EB24117434246DA40891A99E782
:1066A0007F4CA6425BD0802424045B42214327E731
:1066B000002E0CD1002B00D1CBE064463900100035
:1066C000774DD7E6764FBB4218D0330075E6002BE6
:1066D00014D04B07C00818438023C9081B03194274
:1066E00007D0FC081C4204D17907D0080843E146D2
:1066F00021004C46420FC9001143C000684DB9E665
:106700001D0000220023C0E6002D5BD10D000543D3
:1067100000D1E2E65D1C00D1B0E0614DAE421FD079
:10672000DB43382B71DC1F2B00DD96E020250F00AA
:10673000ED1AAF40B9460700AA46DF404D463D433B
:106740002F005546A840D940451EA841884407431C
:10675000BF18974292415142414435003AE664469F
:1067600035004146100085E60B000343002D00D0A4
:1067700063E6002BF5D04346134300D17AE6871831
:106780008742804107224144404209183A400B02A7
:1067900000D4D5E6434B01351940C9E5380069E618
:1067A0001E004746203EF740BC46202B04D0402622
:1067B000F31A46469E403243170063467A1E9741BD
:1067C0001F4302E6364DAE42CAD080252D045B42FF
:1067D0002943A6E70843411E8841A6E6002B00D1C5
:1067E00048E6871A4346B842B641CB1A76429E1B0A
:1067F00033024BD5171A4346BA429241591A5242B4
:10680000891A072264463A4092E501430F00791E37
:106810008F419DE71C000F00203CE740202B03D058
:106820004024E31A99400843411E884138437CE6DE
:106830000022002425E6171A4346BA429241591A0B
:106840005242891A6446350043E541461000144D12
:1068500010E680220024120380E61D000F00203D78
:10686000EF40BC46202B03D04025EB1A994008434B
:1068700007006346781E87411F4369E787189742E0
:106880009B4141445B42C9183500A3E53B003343BB
:10689000CED0072231003A4052E600231A00F4E538
:1068A000FF070000FFFF7FFFF0B55746DE464E466C
:1068B0004546E0B5834607000E03480085B0924682
:1068C0001C00360B400DCD0F002800D19DE0954BEC
:1068D000984239D08023F6001B041E43924A7B0F56
:1068E00033439946944603006344009300230026F3
:1068F000FF00029323031B0B98466300E40F5246EC
:106900005B0D019400D1B3E086498B4200D19EE03B
:106910004246D100802212040A435146490F1143D6
:106920008B46814952468C4600996344CB1A00211C
:10693000D20000932B0063409A460F2E00D905E148
:106940007A4BB6009B599F465B463343994600D02D
:10695000B8E002230826002700900293CAE7CB463E
:106960003A0002990195019B9A46022927D00329F2
:1069700000D180E2012944D06D49009B8C466344DC
:106980001C00002C38DD530700D013E2D2085B4610
:10699000DB0109D55946674B19408B468021C90058
:1069A0008C46009B63441C00634B9C4207DC5B46A7
:1069B00064055F075B0217431B0B620D02E00023B7
:1069C0000027584A00211B031C0B0B0D1B052343FA
:1069D00014055A4A380013401C4353466400DB0731
:1069E00064081C43210005B03CBC90469946A24671
:1069F000AB46F0BD0122524201231B1B382B00DCA9
:106A0000ADE1002200230027DCE75B4633439946D3
:106A10005ED0002E00D18AE1300001F0D7FA0300E9
:106A20000B3B1C2B00DD7BE11D22D31A5A460100D3
:106A3000DA4008398E4013005F46334399468F4051
:106A40003F4B00261B1A00930023029352E7414656
:106A500053460B433B499B468C46009B6344009343
:106A60005B46002B3BD1022300221E43022161E73B
:106A7000434613439B4637D04346002B00D162E187
:106A8000404601F0A3FA03000B3B1C2B00DD53E151
:106A900002004146083A914088461D21CB1A5146D2
:106AA000D9400B0041460B439B46534693401A0086
:106AB000009B25499C46604403008C466344009338
:106AC000002137E70323B14600900C26029311E71B
:106AD0000023009301330426002702930AE70323CF
:106AE000C3461E43032125E701331E430022012133
:106AF00020E700239A46802300271B03094A61E709
:106B0000802349461B03194200D1E2E0594619424D
:106B100000D0DEE00B431B0317001B0BA246014A0B
:106B200050E7C046FF07000001FCFFFF98CD0000C2
:106B3000FF030000FFFFFFFEFE070000FFFF0F80C6
:106B40000DFCFFFF01F8FFFFF3030000D94500D95A
:106B5000CBE000D1C6E03C0048460027009B013B4B
:106B600000935B46160E1B021E4313029846330425
:106B70001B0C9946310C0191FEF754FC4A464243E6
:106B80000B04210C050019438A4207D98919013DDC
:106B90008E4203D88A4201D9851E8919881A019923
:106BA000FEF740FC09048C464A46210464464243F1
:106BB000090C030021438A4204D98919013B8E4202
:106BC00000D8F1E02D041D43AB464346891A4246E6
:106BD000280C12041D0C5B46140C22001B041B0C19
:106BE0005A4303946B434443029568431B19150CA5
:106BF000EB189C4203D980246402A44660441C0C18
:106C000015041B042D0C20185D19814277D373D015
:106C10000C1AA24A7D1BAF42BF419446009B7F42A3
:106C20006344E01B1C00864200D1DBE00199FEF7C3
:106C3000F9FB4A4642430B04290C070019438A42D8
:106C400007D98919013F8E4203D88A4201D9871E8C
:106C50008919881A0199FEF7E5FB09044A46894615
:106C600029044D464243090C030029438A4207D9AF
:106C70008919013B8E4203D88A4201D9831E8919A2
:106C80003F04891A3A00039F1A43380013041B0C6F
:106C9000584381460298150C6F4343434543484689
:106CA000000C8446DB1963449F4203D980204002D4
:106CB0008446654448461F0C00041B04000C7D19E3
:106CC0001818A94200D284E000D17FE001231A43C2
:106CD00057E680234A461B0313431B031B0BAA469C
:106CE0006F4A6FE6BA4200D935E74B46DC075808D1
:106CF0007B081C43FF0734E70024AF4289D2474496
:106D00004745A4415B466442A4196418013BA6426E
:106D10001ED2A0426DD800D1B6E0241A9B4678E777
:106D200003005A46283B9A400027914688E6584679
:106D300001F04CF9203072E603005246283B9A409D
:106D400093460022B4E6504601F040F920309AE61E
:106D5000A642E2D1B845DCD9341A9B4659E71F2B2D
:106D600065DC504C0099A4465C46614408008C40A8
:106D700011008240D940501E82410C4314435A46B0
:106D8000DA401300620709D00F222240042A05D0FE
:106D90002200141D9442894149425B181A0262D5AF
:106DA0000122002300270DE68A4200D80AE7831E4D
:106DB000891907E70F231340042B00D1E6E5171DBF
:106DC0009742924153429B44FA08E0E5002800D1E3
:106DD000D7E57118531EB14227D3A94215D358D015
:106DE0001A0073E7002B00DC04E6012300229B4419
:106DF000CDE502234744474589415B429C464942D1
:106E000089190C19E344241A03E743465F004745F8
:106E10009B41B8465B429E19023A8919A94200D0AB
:106E200054E7404500D051E7ABE51A00F6E71F21D3
:106E30005F4649420C1BE740202B07D01A49009BB4
:106E40008C46634418005B4683401A43501E8241BF
:106E50003A4307270023174009D00F210023114090
:106E60001400042995D122005F075B021B0BD20896
:106E700017430022A6E5802359461B030B431B033F
:106E800017001B0B064A9DE5BD42B2D89B46002465
:106E9000BFE68045B9D31A00C3E7C046FF03000030
:106EA000FF0700001E0400003E040000F0B54F463E
:106EB0004646D6468446C0B58046194E18030F0391
:106EC0004D00000B5C0082463F0B6D0DC90F9146D3
:106ED000640DDB0F0120B5420AD0B44203D0A542B5
:106EE00001D157450CD01CBC90469946A246F0BD36
:106EF00066463E43F7D1AC42F5D154461443F2D135
:106F00000120C845EFD1994207D0002DEBD163464F
:106F10001F433800471EB841E5E70020E3E7C046BD
:106F2000FF070000F0B54F464646D6464D00C0B5B7
:106F30000E03C90F8A462C491F035C008046360B9E
:106F40006D0D91463F0B640DDB0F8D421ED08C42C0
:106F500016D0002D1ED130438446002C01D13A4377
:106F600023D06246002A1AD09A4529D051460220E1
:106F70000139084001381CBC90469946A246F0BD34
:106F800039001143E5D002204042F4E73043FAD102
:106F9000AC420FD0002C0FD13A43E7D00CE00122D5
:106FA000013B934318000130E5E763460020002BC6
:106FB000E1D0DBE73A43E6D19A45D7D1A542D5DC0B
:106FC000A54205DBBE42D1D808D00020BE42D2D2B5
:106FD00050460123013898430130CCE7C845C5D855
:106FE0000020C845F4D3C6E7FF070000F0B54F46C0
:106FF0004646D6464D00C0B50E03C90F8A462E49F7
:107000001F035C008046360B6D0D91463F0B640DEF
:10701000DB0F8D4218D08C4211D0002D18D1304397
:107020008446002C1ED13A431CD163460020002B1D
:1070300030D0514602200139084001382AE0390099
:107040001143EAD0022025E03043FBD1AC4226D0E8
:10705000002C26D13A4324D1514602200139084060
:10706000013817E06246002A0FD09A45E1D1A542C7
:1070700005DBBE42DDD819D00020BE420AD2504600
:10708000012301389843013004E00122013B93437E
:10709000180001301CBC90469946A246F0BD3A4308
:1070A000D0D19A45C5D1A542C3DCE0E7C845C0D8D8
:1070B0000020C845E3D3EDE7FF070000F0B55746D1
:1070C000DE464E464546E0B5834606000F034800BF
:1070D00087B092461D003F0B400DCC0F002800D119
:1070E0006FE0DE4B984238D08023FF001B041F4323
:1070F000730F3B430193DA4B0027994600239B46CD
:10710000F60081442B0369001B0B52469846490D3B
:10711000ED0F002900D185E0D04B994200D173E0FA
:107120004346DA0080231B0413435246CC48520FD7
:1071300084461343524600206144D2008944210012
:10714000694000918C46012149448A460F2F00D99D
:1071500090E0C449BF00CF59BF465B463B43019313
:1071600000D06AE102230827002681469B46C9E732
:1071700032005846019B61460091022800D175E01B
:10718000032800D1FEE1012800D02CE100230027D4
:10719000002600253F032A0D3F0BB34812053A4352
:1071A00002401B051343009A5B00D1075B080B43A9
:1071B0003000190007B03CBC90469946A246AB4649
:1071C000F0BD5B463B43019300D12FE1002F00D17E
:1071D000A5E1380000F0FAFE03000B3B1C2B00DD9C
:1071E00096E11D22D31A5A460100DA405E4608395C
:1071F0008F4013008E403B4301939C4B00271B1A8A
:10720000994600239B467DE7414653460B439349ED
:107210008C46E144002B00D01AE1022202201743E1
:1072200000228CE7134300D10DE14346002B00D12F
:1072300081E1404600F0CAFE02000B3A1C2A00DD44
:1072400072E10100434608398B4098461D239A1A83
:107250005346D3401A004346134352468A40494698
:10726000081A824989468144002068E77B4B002741
:1072700000268EE7140C1204120C1100370C360491
:10728000350C794328008C462E00604360448346C9
:1072900056432100300C80465846794340440291C1
:1072A000844506D98846802149028C46E0444146FF
:1072B00002913604010C360C00048B4681191E0C19
:1072C0001B041B0C0391190079438C46280075435D
:1072D0006544A8465843050C45447743A94203D961
:1072E000802149028C466744290C8C4639000004F1
:1072F000000C2D042D186144AB44059159460491AE
:1073000001990F043F0C080C390051434243904649
:1073100002008C46090C8B4662437C4344445C4427
:10732000A04503D98021490288464244210C884661
:1073300061460904090C8C463900594343437043A4
:107340007E430F0CF6182404BE19644442448C4654
:10735000B34203D980235B0298464044029B6146B6
:107360009846049B370443449B46AB45AD416B4272
:107370000D0405992D0C8C467F196744FD18A8460D
:107380005D462D19A542A44193466442A446C344D8
:10739000DC448F42BF4198459B4193459241A445AF
:1073A000A4415B427F421F43360C52426442BF19E4
:1073B0002243BF18624638184302D20D0399134383
:1073C0006A020A43501E82416146ED0D2A434E0275
:1073D0003243D90100D4B3E00126500832400243C1
:1073E000DE0732435B08224C5444002C62DD510717
:1073F00009D00F201040042805D0101D9042924162
:1074000052429B180200D90104D580241948E40097
:10741000034054441848844200DD27E75E075B02BE
:10742000D2081F0B630516435B0DB2E60023994695
:107430000133042700269B4664E603230197814617
:107440000C279B465EE6012201201743002276E6C8
:10745000032303201F43434671E6C046FF07000095
:1074600001FCFFFFD8CD0000FFFF0F800DFCFFFFE8
:10747000FF030000FFFFFFFEFE0700000023802740
:1074800000933F030026434B83E6019B3200A44652
:10749000584670E6AC466EE6802701993F033942B4
:1074A0002DD03B422BD11F433F033F0B00951600CD
:1074B000384B6EE601252D1B382D00DD66E61F2DAD
:1074C00040DC35481C005044160082408440EE40A9
:1074D000501E824134431443EB40620709D00F220F
:1074E0002240042A05D02200141D944280414042CB
:1074F0001B181A023ED501230027002649E68027E3
:10750000019B3F031F433F033F0B0094214B40E689
:1075100003005A46283B9A40002601926DE65846E1
:1075200000F054FD203057E603005246283B9A40B5
:107530001300002293E6504600F048FD20307BE621
:10754000CA4650E71F201E004042041BE640202D83
:1075500003D0124C5444A3401A43501E824132437C
:1075600007260027164009D00F20002310401400E2
:107570000428B9D122005E075B021F0BD208164314
:10758000002306E680273F031F433F033F0B1600FF
:10759000004BFEE5FF0700001E0400003E04000053
:1075A000F8B557464E464546DE460C000903E0B5A1
:1075B000490A460F5F0031431E03DB0F760A9B46E4
:1075C000530F3343C84E6500C000E40FD2006D0D69
:1075D000A24681467F0D9C469046B74200D1B9E055
:1075E0005B46012673409B46EE1BA34500D183E01A
:1075F000002E63DD002F00D0B1E06346134300D1BD
:1076000023E1731E002B00D0BAE1861A6346B04214
:1076100080410125C91A4042091A0B0200D447E1F2
:1076200049024B0A98464346002B00D189E1404667
:1076300000F0CCFC0300083B1F2B00DD7CE1202286
:107640003000D21A4146D040994002009E400A4381
:107650009D4200DD6AE15D1B6B1C1F2B00DD94E188
:10766000202110003500C91A8E40DA408840DD40E4
:10767000711E8E4111000722284300250643324027
:10768000002A09D00F233340042B05D0331DB34209
:10769000B641764289191E000B0200D43DE26A1CF5
:1076A000914B55056D0D9A4200D119E18F4AF608AC
:1076B0000A40570752023743120B9BE0002E00D0BE
:1076C000C5E06E1C7605760D012E00DC48E16746AC
:1076D000861ACB1BB042BF417F42B8461F004346CB
:1076E000FF1A3B00B8461B0200D55FE137439AD131
:1076F00000220024002579E0002E00DCFAE0002FB3
:1077000000D18DE0784B9D4267D0802367461B04F3
:107710001F43BC46382E00DC52E1634613435A1E19
:1077200093411E1886428041404209180B0200D442
:10773000BEE06D4B01359D4200D1D2E06B4A73082B
:107740000A4001210E401E435108D30707221E4361
:10775000324095E71E00164300D045E740E7624BF4
:107760009D423AD0802367461B041F43BC46382EF7
:1077700000DDEBE01F2E00DC3AE133006746203BE2
:10778000DF403B00202E05D04027BF1B6646BE4091
:10779000324390464646721E96413343DAE0002B50
:1077A00000D114E26346134300D168E180234E0701
:1077B000C008C9081B030643194208D06046C00828
:1077C000184204D163460100D2085E071643F30055
:1077D0009946C900720F444D11434B46DE08424B97
:1077E0004F073743CA089D4200D16EE012036D0572
:1077F000120B6D0D00211203130B0A0D12051A4313
:107800003B4B2D0513402B435B00E4075B082343F0
:10781000380019003CBC90469946A246AB46F8BDDC
:107820006346134311D0731E002B00D007E1861866
:107830008642804161444042091801250B0237D538
:1078400002257BE73E00614691463500C5E75C4670
:10785000002D00D0E1E00B000343F3D0731C00D1F6
:10786000ACE1214B9F4200D13AE1F343382B00DDDC
:107870006FE11F2B00DD8CE120250E00ED1AAE40DC
:10788000B0460600AA46DE40454635432E00554622
:10789000D940A8406346451EA8415B1A9C46304328
:1078A000161AB242924163465242991A3D00B4E61A
:1078B00007223240002A00D0E4E60B4BF6084F07BF
:1078C0003743CA089D4200D090E73B00134300D1E4
:1078D000A6E180231B031A431203120B024D89E712
:1078E00015000022002785E7FF070000FFFF7FFF4C
:1078F000FFFF0F80002E00D0C7E06B1C5E05760DE9
:10790000012E00DCF0E0C84DAB4200D1B9E0851893
:107910000A00854289416244494251180722CE0734
:107920006D082E43490832401D00A9E6BF49ED1AF3
:10793000114007223240A3E6320028388240002658
:1079400086E6300000F042FB203073E663461343C6
:107950005A1E9341C61AB04280414042091A5CE661
:107960000E00674606431743002D5ED1002E00D05F
:10797000F3E0002F00D11EE15C46614691462CE702
:10798000A94FBE427BD01E00F1E610001F3DE8402B
:10799000202B03D04021CB1A9A401643731E9E41E0
:1079A0000722064332400021002583E7161A63466A
:1079B000B2428041591A40420B1A98465C4632E660
:1079C0001F2E00DDABE02027BB1B9A4663465746BF
:1079D000BB40994613004F46F3401F433B005746B8
:1079E000BA40571EBA4113436246F240891898E6DE
:1079F0002027BB1B9A4663465746BB409946130057
:107A00004F46F3401F433B005746BA40571EBA410A
:107A100013436246F240891A9CE7834B9F425FD032
:107A200080252D047342294320E7002E0CD1002F1E
:107A300000D1D0E05C46614691467B4DCDE67A4F61
:107A4000BE421CD01E0065E6002F18D0C0084E07AD
:107A500006438020C9080003014208D06346DC08C1
:107A6000044204D12100DA46D2085E071643F3002F
:107A7000994601245346C900720F11431C406A4DB8
:107A8000ABE61D0000220027B4E6002D59D10B0003
:107A9000034300D1D6E6731C00D1B2E0624B9F4293
:107AA0001ED0F343382B6FDC1F2B00DD97E0202521
:107AB0000E00ED1AAE40B0460600AA46DE4045462E
:107AC00035432E005546A840D940451EA8418C4458
:107AD0000643B61896429241514261443D0025E664
:107AE0003D006146914678E60B000343002D00D02F
:107AF00055E6002BF5D06346134300D16DE686189A
:107B00008642804161444042091800220B0200D4A1
:107B1000D0E6464B01351940B2E5B1465DE633008B
:107B20006746203BDF403B00202E05D04027BF1B8F
:107B30006646BE40324390464646721E96413343E7
:107B4000EFE5394B9F42CBD080252D04734229436A
:107B5000A8E70843411E8841A2E6002F00D13CE679
:107B60006346861ACF1AB0429B415B42FB1A984685
:107B70001B024ED5161A6346B2429241591A52421E
:107B8000891A5C4600227BE501430E00711E8E417E
:107B90009FE71D000E00203DEE40B046202B04D094
:107BA0004025EB1A99400843814648464346411E0A
:107BB0008841184374E60022002417E6161A63462B
:107BC000B2429241591A5242891A3D0025E5614656
:107BD0009146154D01E680220024120379E61D002E
:107BE0000E00203DEE40B046202B04D04025EB1A7D
:107BF0009940084381464E464346711E8E411E43BE
:107C000067E7861896429B4161445B42C9183D0074
:107C10008CE547463743CED007224146324049E6FD
:107C200000273A00E6E5C046FF070000FFFF7FFFA0
:107C300070B50C4E0D031C0349005B002D0B490D64
:107C4000240B5B0DB14208D0064900208B4203D1C2
:107C500014432000441EA04170BD05430120002DA7
:107C6000FAD1F1E7FF07000030B5144D0A034B00CD
:107C7000120B5B0DC90F0024AB4211DD104CA34267
:107C800010DC8024640322430E4CE41A1F2C0CDD0C
:107C90000D48C31ADA4013005C42002900D11C00D1
:107CA000200030BD094BCC18FAE7094DE040AC4646
:107CB00063449A4013000343EEE7C046FE0300000E
:107CC0001D0400003304000013040000FFFFFF7FC9
:107CD000EDFBFFFF70B500282DD0C317C5185D4020
:107CE000C40F280000F072F9154B1B1A5B055B0DE1
:107CF0000A2815DD0B38854000222D032D0B0021AD
:107D000010002D030A0D2D0B12052A430D4D1B05E6
:107D10002A4013435B00E4075B082343190070BD4E
:107D200002002900153291400A000B21081AC540B3
:107D30002D032D0BE3E70024002300250022DEE7BE
:107D40001E040000FFFF0F8010B5041E25D000F0B8
:107D50003DF9144B1B1A5B055B0D0A2812DD0B382D
:107D6000844000222403240B0021100024030A0D68
:107D7000240B120522430C4C1B05224013435B00CD
:107D8000590810BD02002100153291400A000B2154
:107D9000081AC4402403240BE6E700230024002231
:107DA000E2E7C0461E040000FFFF0F804100090EFD
:107DB0004B1C70B5DBB24602750AC40F012B14DDF3
:107DC000E0239B006D07360BCB1800210A0D28001D
:107DD00012051C4D32435B052A405B0813435B00D0
:107DE000E4075B082343190070BD002914D1002D5E
:107DF0001ED0280000F0EAF80A281CDC0B232A0019
:107E00001B1ADA40030015339D400F4B12031B1A57
:107E10005B05160B5B0DD8E7002D06D0320B8026D4
:107E200036036D071643094BCFE7084B0026CCE716
:107E300000230026C9E703002A000B3B9A400025D7
:107E4000E3E7C046FFFF0F8089030000FF07000043
:107E5000F0B54C00640D0B03621C5B0A460F520523
:107E6000C90F1E43C500520D012A29DD374BE71803
:107E7000FE2F1CDC002F3BDD8001431E98410722B2
:107E8000F3006D0F03432B431A40002A04D00F2246
:107E90001A40042A00D004338022D2041A4024D08D
:107EA0000137FAB2FF2F02D09B01580A01E0FF22EE
:107EB00000204002D205400AC90710430843F0BD24
:107EC0003543002C04D1002D0AD100220020F0E718
:107ED000002DECD08020C0033043FF22E9E70024CE
:107EE00000235B02580AE2B2E3E7DB083C00F8E754
:107EF0003B001733F3DB80231B0433431E26F61BA2
:107F00001F2E14DD02225242D71B1A00FA4017001E
:107F1000202E04D00E4A94466444A3401D432B00F7
:107F20005D1EAB4107223B431A400027ADE7094ADB
:107F30002800A218954093406C1EA541F0400722EE
:107F40002B4303431A4000279FE7C04680FCFFFFF6
:107F5000A2FCFFFF82FCFFFF8446081C6146FFE78E
:107F60001FB500F0C7F8002801D40021C8421FBD8A
:107F700010B500F049F84042013010BD10B500F0D6
:107F8000B9F8002801DB002010BD012010BDC0465B
:107F900010B500F0AFF8002801DD002010BD012071
:107FA00010BDC04610B500F057F8002801DC0020D5
:107FB00010BD012010BDC04610B500F04DF80028DE
:107FC00001DA002010BD012010BDC0461C21012394
:107FD0001B04984201D3000C10391B0A984201D3AC
:107FE000000A08391B09984201D30009043902A28A
:107FF000105C40187047C0460403020201010101F1
:10800000000000000000000070B542004E024C006D
:1080100045026D0A120EC30F760A240EC90FFF2AFD
:108020000FD0FF2C11D00120A24200D070BDB5426C
:10803000FCD18B420DD0002AF8D12800451EA84162
:10804000F4E70120002DF1D1EBE70120002EEDD166
:10805000E9E70020EAE7C04670B54A004E02450253
:1080600044006D0A240EC30F760A120EC90FFF2CAE
:1080700015D0FF2A0ED0002C15D1002A01D1002ED8
:108080001CD0002D14D08B4227D00220013B184079
:10809000013870BD002EEED002204042F9E7002DDD
:1080A000FAD1FF2A0ED0002A0ED1002EEDD00BE01F
:1080B00001230139994308000130EAE70020002D2F
:1080C000E7D0E2E7002EE7D18B42DED1944205DD16
:1080D0000221581E08400138DBE70024A24204DCDC
:1080E000B542D2D80020B542D3D2581E01239843BE
:1080F0000130CEE730B5420044024D02C30F4800C4
:10810000640A120E6D0A000EC90FFF2A12D0FF2852
:108110000CD0002A12D1002819D1002D17D1002C23
:108120002BD00220013B1840013826E0002DF0D072
:10813000022022E0002CFBD1FF281FD000281FD1F5
:10814000002D1DD10220013B1840013815E0002C04
:108150000ED08B42E5D10022904204DCAC42E0D844
:108160000020AC4209D2581E01239843013004E09C
:108170000123013999430800013030BD002DD7D1CA
:108180008B42CED18242E7DD0221581E08400138E1
:10819000F3E7C04630B51C00094B05001B6885B0ED
:1081A000D868084B002A01D1074B1A0002920193AC
:1081B00000912B002200054900F010F802F094F81D
:1081C0008C00002018CE0000CECB000025CE000091
:1081D000014B18687047C0468C0000200EB403B5F0
:1081E000010003AB044804CB0068019300F020F9C0
:1081F00002B008BC03B018478C00002070B5002600
:108200000C4D0D4C641BA410A64209D1002604F0AD
:1082100037FB0A4D0A4C641BA410A64205D170BD61
:10822000B300EB5898470136EEE7B300EB58984798
:108230000136F2E75C0200205C0200205C020020B4
:108240007802002010B5034B0100186800F06AF8AE
:1082500010BDC0468C00002010B5034B010018680B
:1082600000F016F810BDC0468C000020002310B5A9
:108270009A4200D110BDCC5CC4540133F8E703002E
:108280001218934200D1704719700133F9E70000CA
:1082900070B50500002910D00C1F2368002B00DAF0
:1082A000E418280003F0F8FB1D4A1368002B05D1E1
:1082B00063601460280003F0F0FB70BDA34209D98D
:1082C000216860188342F3D118685B684118216007
:1082D000EEE713005A68002A01D0A242F9D91968C2
:1082E0005818A0420BD1206809185818196082420A
:1082F000E0D110685268411819605A60DAE7A0426C
:1083000002D90C232B60D5E721686018824203D183
:10831000106852684118216062605C60CAE7C0461C
:10832000580F0020032370B5CD1C9D43083506006F
:108330000C2D1ED20C25A9421DD8300003F0ACFB39
:10834000254A14682100002919D1244C2368002BE8
:1083500003D1300000F0DEFF20602900300000F083
:10836000D9FF431C2BD10C233000336003F095FB65
:1083700003E0002DDFDA0C233360002070BD0B68B2
:108380005B1B19D40B2B03D90B60CC18256003E0C1
:108390004B688C420DD11360300003F07EFB20004F
:1083A00007220B30231D9043C31AE7D05A42E250F4
:1083B000E4E763600C00EFE70C004968C3E70323C0
:1083C000C41C9C43A042E1D0211A300000F0A2FF5F
:1083D000431CDBD1C7E7C046580F00205C0F0020CC
:1083E000936810B5013B9360002B04DA9469A342B3
:1083F00007DB0A2905D01368581C106019700800A3
:1084000010BD01F0A5FE0100F9E7F8B506000F0068
:108410001400D518AC4201D1002007E021783A00C1
:108420003000FFF7DDFF0134431CF3D1F8BD00003D
:10843000F0B59FB002900F0016000593002805D0FC
:1084400083690493002B01D102F0B4FE7B4B9F4261
:108450005BD1029B5F68BB891B0762D53B69002B20
:108460005FD0002306AC6361203363761033A376BC
:1084700035002B78002B01D0252B5CD1AB1B04934E
:108480000CD0320039000298FFF7BFFF431C00D127
:10849000C4E06269049B9446634463612B78002BBB
:1084A00000D1BBE0012200235242626002A9543293
:1084B00052186E1C2360E360A3601370A3653178CB
:1084C00005225F4803F0CAFA751C002835D12268DE
:1084D000D30604D5532302A95B1820211970130772
:1084E00004D5532302A95B182B21197033782A2B4A
:1084F0002CD0350000210A20E3682A786E1C303A1F
:10850000092A64D900292ED026E04E4B9F4202D181
:10851000029B9F689FE74C4B9F429CD1029BDF6868
:1085200099E73900029801F069FE002899D00120EE
:1085300040421FB0F0BD01359BE7414B2268C01A95
:1085400001238340134323602E00B8E7059B191DC8
:108550001B680591002B01DB099304E05B42E3609B
:108560000223134323602B782E2B0AD16B782A2BFE
:1085700035D1059B02351A1D1B680592002B2BDB9C
:108580000793324E29780322300003F067FA00285F
:1085900006D04023801B83402268013513432360AB
:1085A000297806222A486E1C217603F057FA002803
:1085B0003AD0284B002B25D10722059B0733934344
:1085C000083305936369039A9B18636150E743433B
:1085D00001219B18350090E701235B42D0E700237F
:1085E0000A201A000135636029786E1C3039092988
:1085F00003D9002BC5D00792C3E742430123521889
:108600003500F1E705AB00933A00134B21000298C7
:1086100000F0C0F80390039B0133D3D1BB895B0604
:1086200000D584E70B9884E705AB00933A000A4B2A
:108630002100029800F068FBECE7C04628CF00005C
:1086400058CE000048CF000008CF00005ECE0000EA
:1086500062CE0000958700000B840000F0B58BB05F
:1086600014001D1E129953DA802424061B191D00C4
:1086700014002D230B702023149E03229E43462EAC
:1086800007D03300453B59424B411099013ACB1872
:10869000109309AB049308AB0393139B00920293CE
:1086A000109B220001932B0001F0ACFE0700472E27
:1086B00002D1119BDB0724D5109BFB180793462E94
:1086C00014D13B78302B0CD100220023200029004C
:1086D000FCF7A8FF002804D10123109A9B1A139AD3
:1086E0001360139B079A1B68D3180793002200237B
:1086F00020002900FCF796FF302200280DD0079BB0
:1087000009933800099B159ADB1B13600BB0F0BD71
:108710000023AFE7591C09911A70099B07998B42F6
:10872000F8D3EEE7F0B5831C85B0019306000C008A
:1087300002702B23002901DA2D234C427370092C7F
:1087400022DD02ABDD1D20000A21FCF755FF6F1E64
:108750003031397020000A21FCF768FE0400092836
:108760000BDC023D3034019B2C7002AA073218004A
:10877000AA4204D8801B05B0F0BD3D00E3E72A788B
:1087800001351A700133F0E73023E418B370301D5F
:10879000F470EFE7F0B595B00C000A920B931A9DB8
:1087A000099003F0D1F8036818000C9300F0E8FD7D
:1087B0000023129323680E900D930D99277E2B684A
:1087C0000722C90545D59B1893431A0008322A6031
:1087D0001A685B68A264E3640122E56CA66C6B0016
:1087E0005B080F935242AC4B30000F99FFF720FA11
:1087F000002830D10122A84B524230000F99FCF7DB
:1088000021FF002827D10022002330002900FCF797
:108810000FFF002803D023002D2243331A709F4DF1
:10882000472F00D89E4D032300260D9A2361013364
:108830009A4322600B9B13AA009321000A9B09987C
:1088400000F0F4F9431C00D093E00120404215B041
:10885000F0BD0733B8E732002B0030002900FFF7E6
:10886000E7F9002804D08F4D472FDCD88E4DDAE78A
:1088700080230D996268DB000B43511C43D1073202
:10888000626012AA0021059211AA0392232223609A
:108890000691019308A9636852180292009332006E
:1088A0002B0004970998FFF7D9FE20233A00050012
:1088B0009A43472A07D1119BDA1C02DB6268934274
:1088C00045DD023FFFB21199652F25D820000139FF
:1088D0003A0050301191FFF725FF129A0600131845
:1088E0002361012A02DC2268D20701D5013323610A
:1088F000232308AA9B181B78002B9BD023002D2232
:1089000043331A7096E7672F00D176E1472FB8D12D
:10891000002AB6D10122B3E7662F19D16368002976
:108920000CDD2161002B02D12268D20702D5013370
:108930005B182361119B0026A365D9E7002B03D1A7
:1089400001222168114200D09A1C2261F2E76727B8
:10895000119B129A934205DB22682361D207E9D565
:108960000133E6E70121002B01DC4918C91A52182E
:10897000EBE72268530508D423692A000A9909986D
:108980000B9DA847431C29D15FE7652F00D8E0E085
:10899000A06CE16C00220023FCF744FE002834D0D8
:1089A0000123424A0A9909980B9DA847431C00D10C
:1089B0004BE7119B129A934202DB2368DB070DD52C
:1089C0000B9D0E9B0C9A0A990998A8470025431CF9
:1089D00000D13AE7129B013BAB420ADC23689B07BC
:1089E00000D508E1139BE068984200DB2FE71800F0
:1089F0002DE7220001231A320A9909980B9EB047ED
:108A0000431C00D121E70135E4E7119B002B2DDC4D
:108A10000123264A0A9909980B9EB047431C00D1AE
:108A200013E7119B002B05D1129B002B02D1236869
:108A3000DB07D3D50B9E0E9B0C9A0A990998B04779
:108A40000026431C00D100E7119B5B42B34201DCCE
:108A5000129B92E7220001231A320A9909980B9F70
:108A6000B847431C00D1F0E60136EDE7A36D129F35
:108A70009F4200DD1F00002F08DD3B002A000A99FD
:108A800009980B9EB047431C00D1DEE600230D93EE
:108A9000FB43DB170F9318E0FFFFEF7F6DCE000065
:108AA00069CE000075CE000071CE000079CE0000C6
:108AB000220001231A320A9909980B9EB047431CE1
:108AC00000D1C2E60D9B01330D930F9BA66D0D9A4D
:108AD0003B40F31A9342EBDC119B129AAD1993427F
:108AE00010DB2368DB070DD4129F119BBE1BFF1AFE
:108AF000B74200DD3700002F0DDCFE43F3170025E1
:108B00000C931CE00E9B0C9A0A9909980B9FB8478E
:108B1000431CE9D199E63B002A000A9909980B9D6C
:108B2000A847431CE9D190E6220001231A320A9992
:108B300009980B9EB047431C00D186E60135119A77
:108B4000129B0C999B1A3A000A409B1AAB42EBDC31
:108B500044E7129B012B02DC01231A4232D001238D
:108B60002A000A9909980B9FB847431C00D16CE66C
:108B70000E9B0C9A0A9909980B9F0135B847431C24
:108B800000D162E6A06CE16C129B00225F1E002304
:108B9000FCF748FD3B00002814D000250AE0220025
:108BA00001231A320A9909980B9FB847431C00D138
:108BB0004BE60135129B013BAB42F0DC2200330057
:108BC0005032DBE62A000A9909980B9DA847431CFE
:108BD000F4D13AE62200012319320A9909980B9E32
:108BE000B047431C00D130E60135E368139A9B1A65
:108BF000AB42EFDCF6E60025F7E7002A00D189E674
:108C00000021069112A9059111A90391232108A819
:108C100009182360019300922B00049702913200FF
:108C20000998FFF71BFD050045E6C046F7B515009E
:108C300001938A680B6900900C00934200DA1300DC
:108C400022002B6043321278002A01D001332B60BE
:108C500023689B0602D52B6802332B600627236806
:108C60001F4027D0230043331B785A1E93412268AC
:108C7000920630D42200019943320098089EB047F2
:108C8000431C25D0062320682A68E168034000259C
:108C9000042B03D18D1AEB43DB171D40A368226917
:108CA000934201DD9B1AED180027BD4220D1002020
:108CB00010E00137E3682A689B1ABB42D2DD22002C
:108CC0000123193201990098089EB047431CF0D146
:108CD00001204042FEBD3020E118433108702100E0
:108CE0005A1C45310978A218433202331170C1E78A
:108CF000220001231A3201990098089EB047431CB4
:108D0000E6D00137D1E70000F0B589B004920A003F
:108D100043320593039002920A7E0C000E9B6E2A4A
:108D200000D186E01FD8632A33D008D8002A00D1AA
:108D30008CE0582A4DD0250042352A7030E0642A54
:108D400001D0692AF7D1196825680A1D280629D596
:108D500008681A60002803DA2D23029A4042137033
:108D60006B4E0A274FE0732A74D008D86F2A1FD0A1
:108D7000702AE0D1202209680A43226003E0752AA4
:108D800016D0782AD7D12200782145321170614E51
:108D900022E025001A684235111D196013682B70F6
:108DA000012365E008681A606906D3D500B2D1E7EF
:108DB00019682568081D186008682E0605D5544EE8
:108DC00008276F2A1BD00A2719E06D06F7D580B255
:108DD000F5E745314E4E0A7018682268011D00689B
:108DE0001960150621D5D30702D520231A43226026
:108DF0001027002803D1202322689A4322602300F1
:108E0000002243331A706368A360002B58DB0422EE
:108E1000216891432160002854D1029D002B5AD033
:108E20002500337842352B7055E05506DBD580B2EE
:108E3000D9E71A680D68101D4969186013682E0675
:108E400001D5196002E06D06FBD519800023029D53
:108E500023614FE01A68111D1960156800216268CE
:108E6000280002F0FBFD002801D0401B6060636811
:108E700023610023029A13703CE023692A000499BD
:108E80000398059DA847431C3ED023689B0715D433
:108E9000079BE068984239DA180037E02200012386
:108EA000193204990398059EB047431C2CD0013514
:108EB000E368079A9B1AAB42F0DCE9E70025F7E785
:108EC0000028ADD0029D3900FCF7ACFA735C013D7F
:108ED0002B700028F7D1082F09D12368DB0706D5AE
:108EE00063682269934202DC3023013D2B70029BB0
:108EF0005B1B2361059B07AA00932100049B039839
:108F0000FFF794FE431CB8D10120404209B0F0BDE8
:108F10007BCE00008CCE0000F0B58BB002900092AA
:108F20000020AE2205938B680E00591E520004905B
:108F3000914205D95E3BFF3B04935E23FF33B36050
:108F4000F0233268DB0013433360330000271C3307
:108F50001D003C0003930897079701970697B26896
:108F6000002A13D0009B1B6809931B78492B00D162
:108F70007CE054D8392B47D8312B00D394E02D2BEB
:108F800000D19CE017D82B2B00D198E0019B002B3F
:108F900003D032689B4B13403360013C012C00D955
:108FA000EEE0BE246400039B9D4200D9DEE0012771
:108FB00038000BB0F0BD2E2B00D1A2E0302BE5D154
:108FC0003168C80570D580239943019B3160013316
:108FD0000193049B002B03D0013B01320493B26048
:108FE000B368009A013BB360336901333361009B7E
:108FF0005B680993013B5360002B00DCACE0136815
:10900000099301331360AAE7452B00D183E0462B77
:109010006DD0412BBAD1012CB8D102244CE0652B84
:1090200079D01BD8542B67D013D84E2BAED1002C3F
:109030004CD1019A002A4BD1E021E0203268C900CE
:109040001140C000814243D16F4901340A4032606F
:1090500032E0592B23D0612BDDD097E76E2BE6D081
:1090600018D8662B43D0692B00D08FE7002F37D15B
:10907000019A002A00D08CE7E021E0203268C90084
:109080001140C000814200D087E75F4901370A40A4
:10909000326011E0742B2FD0792B00D076E7072FA8
:1090A00000D073E7082707E0E219002A00D06DE737
:1090B000564A31680A4032602B70013590E78021B2
:1090C00032680A4200D161E78A43F4E7022C41D0BA
:1090D000012F02D0042F00D058E70137FFB2EBE791
:1090E0000221FA1E8A43D2B2002AF6D04EE7022F9E
:1090F00000D04BE70327DFE7062F00D046E707271E
:10910000DAE73268910500D440E741490A4032600D
:10911000019A0692D0E7A02180203268C900114050
:10912000C000814206D0024200D12FE701990029F8
:1091300000D132E7910504D4019906980895091ADF
:10914000079131490A40C02149000A433260002298
:109150000192B1E70324AFE7C0235B00F358009905
:1091600002989847002800D1F9E60FE7013D3359EE
:109170002978009A029898473369013B336112E7D6
:109180007B1E062B26D8022F39D8BE246400039BF1
:109190009D4200D80BE7013D33592978009A029887
:1091A00098473369013B3361F1E7049B009A013B27
:1091B00004931978BE235B00F358029809939847EB
:1091C0003369013B3361013CE4B2022CEDD1033F32
:1091D000FFB2ED1B3368DA0537D55B051AD5BE241F
:1091E0006400039B9D4200D8E1E6013D3359297894
:1091F000009A029898473369013B3361F1E73C00DC
:109200000495E0E7FFFEFFFF7FF8FFFF7FFEFFFF13
:109210007FFDFFFF33696C1E2178013B33616529B7
:109220000CD045290AD0BE235B00F358009A02985F
:1092300098473369AC1E013B21783361BE235B0044
:10924000F358009A029898472500102733681F406A
:109250005BD1C0232F703268DB0013408022D20024
:1092600093421BD1069A019B9B1A5A42002B22D192
:1092700000220399029800F0CBFE059B04003068A1
:109280000D001B68820723D51A1D05990A601B680B
:109290001C605D60F3680133F36089E6079B002B77
:1092A000E6D0089B3A00591C02980A2300F040FFC0
:1092B000079B089DC21A33007033FF339D4202D3CF
:1092C00035006F35FF351249280000F039F8CFE737
:1092D000042108401A1D01900028D6D105992000CC
:1092E0000A601B682200009329002B00FEF7A0FCF7
:1092F000002805D0019800F01FF8009B1860C9E70E
:1093000020002900FEF7A4FDF7E7002750E6C0463D
:109310009DCE0000002370B5064C050008002360B8
:10932000FAF722FE431C03D12368002B00D02B60E8
:1093300070BDC046600F0020004870470000C07F2D
:109340000EB400B50B499CB01DAB0290069007917E
:1093500004910948094904CB0591006802A90193C9
:1093600003F028F80023029A13701CB008BC03B065
:109370001847C046FFFFFF7F8C0000200802FFFF58
:109380000023C25C0133002AFBD1581E7047000045
:1093900070B516000D0002F051FE002E0DD06B23AB
:1093A0006A00520D9B1A002B07DD0024034A1B059F
:1093B0009D182B002200FDF781FE70BD0000F03FDC
:1093C000F0B5A7B007930023049007982293069165
:1093D0001D9202F0B6FA05000068FFF7D1FF0026E3
:1093E0000027069B05902193219B1A780D2A39D8D6
:1093F000092A3DD2002A44D0002313930022219C45
:109400000C922378302B00D07EE06378582B02D06A
:10941000782B00D06EE0079B964A0293139B21A9FC
:10942000019322AB0093049823AB01F09FFF072523
:109430000590054005D0062D2FD10023013421943D
:1094400013931D9B002B02D01D9B219A1A60139B26
:10945000002B1DD0802332001B06FB1810001900C2
:1094600027B0F0BD2B2A16D02D2A03D0202AC3D135
:109470000133B8E7012213925A1C21925B78002B2A
:10948000BCD1069B2193002313931D9B002BDBD1A2
:1094900032003B00E2E70022EDE7229A002A07D0E3
:1094A000352124A802F0B7FE2299049802F02EFB81
:1094B000681E042806D8FBF725FF0C0317190C00BB
:1094C000249E259F059B1B07BBD580231B061F439E
:1094D000B7E7259B684A69491A40239B249E5B187D
:1094E0001B051A431700EDE7654FEBE70126654FB3
:1094F0007642E7E7219B5A1C21925B78302BF9D00A
:10950000002B9ED001230C93219B0A22129300234F
:109510000B9308930A93219804782300303BD9B227
:10952000092934D9059A296803F0D8F8002840D0D1
:109530000020230084460A9A0790059220221900F1
:1095400091430A000021452A00D0BFE0059B0C9AF8
:10955000034313438B4294D0219B06930133219301
:10956000069B5B782B2B00D182E00C002D2B05D1C4
:109570000124069B02332193069B9B781A00303A04
:10958000092A00D884E0069A002121929EE00A99D7
:10959000082909DC08995143CB1808930A9B01302C
:1095A00001330A932190B6E70B995143CB180B93E3
:1095B000F4E7219A059B94460A9A634421931B7809
:1095C000002A36D0844605921A00303A092A12D968
:1095D00001220792B2E7219B01305A1C21925B784D
:1095E000302BF8D01A00313A082A3CD884460020A3
:1095F000219A05901292303B421C002B13D00A2175
:109600009444059A8518AA4215D10599059A013105
:10961000091812180591082A1BDC0A2208994A43E6
:109620009B1800220893219B1000591C21915B7804
:10963000CAE70A98D4E7541C082A04DC089A4A436B
:1096400008922200DFE7102CFBDC0B9A4A430B92B6
:10965000F7E7059900221029E5DC0A210B98414320
:109660005B180B93DFE70022944605920132B0E7C6
:109670000C007EE7A4CE0000FFFFEFFF33040000E4
:109680000000F07FFFFFFF7F219B5A1C21925B7837
:10969000302BF9D01A00313A0021082A16D8303B75
:1096A000219D0E93219B591C21915B781A00303A21
:1096B000092A32D94A1BAD4D2900082A03DC0E992C
:1096C000A94200DD2900002C00D04942059A002A59
:1096D00049D10C9A104300D0B3E6079A002A00D073
:1096E000CFE64E2B25D01FDC492B00D0C9E6A04980
:1096F00021A802F078F8002800D1C2E6219B9D49FC
:10970000013B21A8219302F06EF8002802D1219B91
:1097100001332193984F002693E60A220E994A437B
:10972000D218303A0E92BDE7692BE0D06E2B00D0F4
:10973000A7E6924921A802F056F8002800D1A0E639
:10974000219B1B78282B0CD124AA8D4921A802F03B
:109750005EF8052805D1259B874A249E1A431700E9
:109760006FE6884FD7E76346CB1A07930A9B002B17
:1097700001D1059B0A93059C102C00DD102408984C
:10978000FEF7E2FA059B06000F00092B15DC079B8C
:10979000002B00D155E6079B002B00DC7DE0162B4B
:1097A00062DCDC00784B320019193B00086849681C
:1097B000FDF784FC06000F0043E62200724B093AD5
:1097C000D2009B181A685B68FDF778FC06000B98BE
:1097D0000F00FEF7B9FA0B00020039003000FCF769
:1097E00047FD059B06000F000F2BD0DD059B1C1BC2
:1097F000079BE418002C00DC94E00F2323400AD0E0
:109800006149DB00C9183200086849683B00FDF770
:1098100055FC06000F000F239C436ED02633FF3308
:109820009C4248DD002405940B940A9422230026D0
:10983000049A514F13600B9BB34200D101E6229969
:10984000049802F063F90A99049802F05FF9059907
:10985000049802F05BF90B99049802F057F9210083
:10986000049802F053F9ECE52523059A9B1A079A10
:109870009342BBDB0F23059A434C9D1AE900611804
:109880003200086849683B00FDF718FC079B5E1B27
:10989000F600A619326873688AE7079B1633A5DBC2
:1098A000079B3000DA00384B39009B1A1A685B6856
:1098B000FCF7FAFF7EE70023300039001D00241179
:1098C000012C1DDC002B01D006000F002F4BED00FA
:1098D000FF182F4B32005D19286869683B00FDF7BF
:1098E000EDFB254B2B4A06000B4093429AD82A4A9F
:1098F000934213D90126294F7642002306937BE039
:109900000122144207D0224AEB009B181A685B68B8
:10991000FDF7D4FB012301356410D1E7D4239B0468
:10992000CF18EAE7002CE8D00F23644223400AD086
:10993000154ADB00D31830001A685B683900FCF761
:10994000B3FF06000F002411D7D01F2C28DD002400
:1099500005940B940A942223049A002613600B9B0F
:109960000027002B00D06AE76BE5C0461F4E0000C1
:109970006ECE0000FBCE00000000F07F76CE00002F
:10998000B8CE00000000F8FF98CF00000000B0FC47
:1099900070CF00000000A07C0000907CFFFFEF7FF4
:1099A00010232340069301D06A230693002330003E
:1099B00039001D00002C00DD0EE1002B01D0060057
:1099C0000F00069B002B0FD06B237900490D3A0046
:1099D0005B1A002B08DD1F2B00DC12E10026342B64
:1099E00000DC07E1DC27BF0400220023300039003F
:1099F000FBF718FE0028AAD1089B0A9A0093129937
:109A0000059B049802F0D9F80B90002800D109E7D3
:109A1000079B079ADB17524213401593079B0024BC
:109A2000DB43079ADB171A401C9205940B9B0498A2
:109A3000596802F033F80A90002800D1F6E60B9B33
:109A40000B991B690C319A1C92000C300893FEF79D
:109A50000DFC24AB019323AB009332003B00049830
:109A60000E960F9702F05CFB2290002800D1DDE6F5
:109A70000121049802F028F90590002800D1D5E6CC
:109A8000239B002B00DAC1E0159A9D181C9A94467E
:109A90000699249A5B1A36219B188A1AB249013B0F
:109AA00001208B4200DBBDE0C91A521A1F2900DDDC
:109AB000B1E08840002314901093AB180893130072
:109AC000069A6344D318089A0C932B00954200DD44
:109AD00013000C9A934200DD1300002B06DD089A58
:109AE000ED1AD21A08920C9AD21A0C92159B002BDE
:109AF00017D01A000599049802F07EF90590002805
:109B000000D193E60100229A049802F0E6F8129040
:109B1000002800D18AE62299049801F0F7FF129BF1
:109B20002293089B002B00DD7FE0079B002B08DDC4
:109B30001C9A0A99049802F05FF90A90002800D153
:109B400074E60C9B002B08DD1A000A99049802F0B9
:109B5000A5F90A90002800D168E6002D08DD2A004A
:109B60000599049802F09AF90590002800D15DE665
:109B70000A9A2299049802F0FDF9041E00D155E6D4
:109B80000025C3680599C560129302F0D9F9A8426F
:109B900055DA129BAB421BD1AE4219D13B03AB420B
:109BA00016D1D622714BD2043B40934210D963693F
:109BB000AB4202D12369012B0ADD21000122049866
:109BC00002F06CF90599040002F0BAF900286BDC88
:109BD000069B002B78D132E60122144207D0644A5A
:109BE000EB00D3181A685B68FDF768FA01230135AA
:109BF0006410DFE60121203B494299400A401700EA
:109C0000F2E6012252429A401640EDE61C9A159D5A
:109C1000D21A94463CE75749CB1A0100994010915B
:109C200014904AE700231093FAE7089A22990498BF
:109C300002F034F92290002800D076E7F6E50C9780
:109C4000002800D0A0E0129A3B031B0B002A27D06B
:109C5000494A934257D10122069B524231001000DB
:109C6000002B0BD0D425414BED043B401000AB4200
:109C700004D86C301B0DC31A9A401000814242D1A7
:109C80003E4B0C9A9A4202D14B1C00D1CEE5374B89
:109C90000C9A00261A401300802252039F1897E75F
:109CA000002B30D1002E2ED106993B002F4A0029DF
:109CB00020D01100D6203940C00481421ADCDC23B8
:109CC0009B04994200DC46E62D4B30001B93002399
:109CD0001A931A9A1B9B3900FDF7F0F906000F0042
:109CE0000B1E00D0ABE5002800D0A8E5049A223373
:109CF0001360A4E501261340224A76429B181E4AAF
:109D00001A43170064E7109B002B15D00C9B109A88
:109D1000134200D15CE7129B069A30003900002BF9
:109D20000FD0FFF735FB02000B000E980F99FCF7E0
:109D30009FFA06000F004BE7149B334200D147E720
:109D4000E9E7FFF725FB02000B000E980F99FDF7DE
:109D500027FC0022002306000F00FBF763FC00280D
:109D600000D0F8E534E7C04602FCFFFF0000F07FBA
:109D7000D0CE0000E2FBFFFFFFFF0F00FFFFEF7FF1
:109D8000000050390000F0FF0599200002F01CFA95
:109D900080230022DB0508900991FBF753FC002883
:109DA00000D17FE0129B002B4BD000228A4B1092F7
:109DB0001193894B0893894A0C9B13401493149A6E
:109DC000874B9A4200D0BAE00E9A0F9B1A921B93CF
:109DD000844A0C9B944663441F00109A119B3000E8
:109DE00039000C920D9302F029F902000B000C9837
:109DF0000D99FDF763F932003B00FCF739FA774A19
:109E0000794B06000A409A4264D90F9B774A9342E5
:109E100003D10E9B013300D108E50126734F764232
:109E20002299049801F072FE0A99049801F06EFEDE
:109E30000599049801F06AFE2100049801F066FE7D
:109E4000F4E5002E1ED10C9B1B0321D10898099923
:109E50000022614BFBF7ECFB00281FD10898099901
:109E60000022634BFDF72AF90500089180221206B3
:109E70009446089B1E9563441F931E9A1F9B109245
:109E8000119398E7012E03D10C9B002B00D162E5C2
:109E90000022584B0025109211938AE7544B129DD3
:109EA0000893E3E7524B089809990022FDF706F959
:109EB000129B05000891002B07D180231B06CB18AD
:109EC00016901793169A179BD9E70200089B1692D3
:109ED0001793F7E7D4239B04CF18069B002B9FD141
:109EE0003E4B149A0C973B409A4299D1089928000E
:109EF000FDF7BAFEFDF7EEFE0B0002000899280000
:109F0000FDF74EFB129B08900991002B04D1002E07
:109F100002D10C9B1B0358D008980999364A374B3D
:109F2000FBF786FB002800D089E408980999344A99
:109F30002F4BFBF791FB002800D171E77FE4069BD4
:109F4000002B2AD0D423149ADB049A4225D82D4A18
:109F50002D4B28000899FBF775FB002816D0280028
:109F60000899FBF7A5FB002800D10130FDF7ECFEB6
:109F7000129B05000891002B22D180231B06CB18D1
:109F800018901993189A199B10921193D622119B2D
:109F9000D2049B18149A9B1A11930E980F99109E35
:109FA000119F02F04BF802000B0030003900FDF762
:109FB00085F80E9A0F9BFCF75BF906000F008CE703
:109FC0000200089B18921993DCE70B4A0F4B089884
:109FD0000999FBF72DFBAEE70000F03F0000F07F92
:109FE0000000E07F0000B0FCFFFF9F7CFFFFEF7FE1
:109FF0000000E03F0000F0BF9535A094FFFFDF3F79
:10A0000035E5AF350000C0FFFFFFDF41FFFFCF3F69
:10A01000044B10B51B681B6A002B00D1024BFFF7E5
:10A02000CFF910BD8C000020F0000020F0B51F001B
:10A030000E0087B00590019102920C98347801F0DF
:10A040007DFC082200194378751C134036D12D2C55
:10A0500036D1B51C74780126002F62D0102F09D19B
:10A06000302C07D120222B789343582B54D1102722
:10A070006C7802352D4B3900F31818000393FBF769
:10A08000D1F9049101210023494202008C461800B5
:10A090002100303909291AD80C00A74223DD591CA8
:10A0A00009D06346824206D302D10499A14202DB61
:10A0B0000123784320182C780135E9E72E00BCE70E
:10A0C0002B2C01D01E00C7E7B51C7478FAE72100DD
:10A0D0004139192901D8373CDFE7210061391929B5
:10A0E00001D8573CD9E75A1C08D1059A233313608D
:10A0F000029B0398002B09D107B0F0BD002E00D0C1
:10A100004042029A002AF7D0002B01D06B1E019327
:10A11000029B019A1A60EFE73024002FAAD108278A
:10A12000A8E7302C9ED00A27A4E7C046FFFFFF7F98
:10A1300013B5054C2468246A002C00D1034C00940C
:10A14000FFF774FF16BDC0468C000020F000002011
:10A15000F8B505000E001400002804D08369002B18
:10A1600001D101F027F8224B9C422DD16C68A369E4
:10A17000A360A3891B0731D52369002B2ED0236848
:10A180002269F7B2981A6369F6B2834205DC2100AE
:10A19000280000F0A1FF002826D1A3680130013B70
:10A1A000A36023685A1C22601F706369834204D035
:10A1B000A389DB071AD50A2E18D12100280000F048
:10A1C0008BFF002812D00FE00A4B9C4201D1AC68F3
:10A1D000CDE7094B9C42CAD1EC68C8E721002800B2
:10A1E00000F00CF80028CAD0012676423000F8BDF5
:10A1F00028CF000048CF000008CF0000364B70B5D4
:10A200001D6806000C00002D05D0AB69002B02D1A3
:10A21000280000F0CFFF314B9C420FD16C680C231B
:10A22000E25E93B219072DD4D90611D40923012077
:10A23000336037331343A381404270BD284B9C42A7
:10A2400001D1AC68EBE7274B9C42E8D1EC68E6E72C
:10A250005B0713D5616B002908D023004433994272
:10A2600002D03000FEF714F8002363632422A38990
:10A270009343A38100236360236923600823A28999
:10A280001343A3812369002B0BD1A0218022A38932
:10A29000890092000B40934203D02100300001F06E
:10A2A00087FB0123A289134011D00023A3606369B7
:10A2B0005B42A361002023698342BED10C23E25E8E
:10A2C0001306BAD540231343A3810138B5E792079B
:10A2D00000D46369A360EDE78C00002028CF000064
:10A2E00048CF000008CF000010B5062002F08AF920
:10A2F000012002F0C3FAF0B503690C6989B00700C8
:10A3000005910026A34265DB0B00013C1433A50038
:10A3100003935B1904930300143302935D19049BA8
:10A3200028681B68591C0193FAF7F6FF0190B042A8
:10A3300029D0039B02989C460696624608CA94461A
:10A34000019A99B251431B0C534389190A0C9B186B
:10A3500007931E0C036889B29AB2069BD218036851
:10A36000521A190C6B469B8BCB1A11145B181914DB
:10A3700092B21B041A43049B069104C06345DCD2CD
:10A380002B68002B2DD00599380001F0D9FD00284D
:10A390001FDB0025019B029801330399019302689A
:10A3A00008C992B255199AB2AA1A05681B0C2D0C4D
:10A3B000EB1A15145B191D1492B21B04134308C049
:10A3C000049B8B42EBD2029AA300D3181A68002A8E
:10A3D00011D0019E300009B0F0BD2B68002B04D1D4
:10A3E000013C029B043DAB42F7D33C61CBE71A68CA
:10A3F000002A04D1013C029A043B9A42F7D33C6103
:10A40000E7E70000F0B516001F00446A9BB0029019
:10A41000239D06960797002C08D11020FDF712FF08
:10A42000029B5862446084600460C460029B5B6A63
:10A43000196800290BD05A68012393404A608B6049
:10A44000029801F063FB0022029B5B6A1A60002FF6
:10A4500020DA01232B607B005B080793079CB24B3B
:10A46000220017931A409A4217D1B04B229A1360D8
:10A47000069B002B03D1240301D100F087FDAC4BD8
:10A48000249A0893002A02D0AA4B249A13600898B1
:10A490001BB0F0BD00232B60E0E7069E079F002263
:10A4A000002330003900FBF7BDF8051E0BD0012357
:10A4B000229A1360A04B249A0893002AE7D09F4A5F
:10A4C00024990A60E3E718AB019319AB00933200BB
:10A4D0003B00029801F024FE630003905B0D74D0F2
:10A4E0003A03974C120B14432100964A30001695FC
:10A4F0009E180022944BFDF753F8944A944BFCF7B6
:10A50000DDFD944A944BFBF7B3FE040030000D00D0
:10A51000FDF7E0FB914A924BFCF7D0FD02000B00E7
:10A5200020002900FBF7A4FE04000D00FDF79CFBB2
:10A5300000220700002320002900FBF779F80028FB
:10A5400009D03800FDF7C6FB2B002200FBF76AF8A4
:10A55000434258413F1A01231493162F0DD88149C5
:10A56000FB00C91808684968069A079BFBF774F84E
:10A57000002846D00023013F1493189B9E1B002304
:10A580000A933300013B0B9304D501239B1B0A93D1
:10A5900000230B93002F36DB0B9B1197DB190B93DA
:10A5A00000230493209B0124092B00D984E0052B70
:10A5B00002DD0024043B2093209B981E032800D931
:10A5C00084E0FAF79FFE7577286A189B199A9E18FF
:10A5D000654BF218202A0FDD40239B1A9C40634BE9
:10A5E0000698F318D8402043FDF7AEFB0123604CDA
:10A5F000013E091916937CE7202306989B1A984080
:10A60000F2E71490B9E70A9BDB1B0A937B420493A1
:10A6100000231193C6E701230D93219B002B59DDE5
:10A620000C930993029A556A00226A600432100062
:10A6300014306968984252D9029801F02FFA029BAF
:10A6400028605B6A1B680893099B0E2B00D90AE1FE
:10A65000002C00D107E1069B079C12931394002F56
:10A6600000DC89E00F213A003E4B0A40D2009B18E3
:10A670001D685E6802233C110E93E3060BD53D4B2B
:10A680000C401A6A5B6A12981399FCF70DF90323C0
:10A69000069007910E9300233AE001230D93219B2E
:10A6A000FB180C9301330993002BBBDC0123B9E7A2
:10A6B0000023B1E70023F1E700230D942093013B31
:10A6C00000220C93099313332192ABE701230D93DE
:10A6D000023BF5E701230C9309931A00F4E70131DB
:10A6E00069605200A3E701231C420ED00E9B214A51
:10A6F00001330E93109B2800DB009B1831001A6871
:10A700005B68FCF7DBFC05000E00109B6410013356
:10A710001093002CE7D1069807992A003300FCF724
:10A72000C3F80690079142E00000F07F0F27000079
:10A7300001CF000004CF000079CE00007ACE0000E7
:10A740000000F03F01FCFFFF0000F83F61436F6332
:10A75000A787D23FB3C8608B288AC63FFB799F503A
:10A760001344D33F98CF00003204000012040000CD
:10A77000000010FE70CF000002230E93002F16D0B1
:10A78000129813997C420D332340CE4ADB00D31834
:10A790001A685B68FCF792FC002301261D000690F6
:10A7A00007912411002C00D08CE0002BB9D1149B10
:10A7B000002B00D196E0069C079D0022C24B200092
:10A7C0002900FAF735FF002800D18BE0099B002B08
:10A7D00000D187E00C9B002B41DDBC4B0022200008
:10A7E0002900FCF76BFC0E9B0690079101330E933A
:10A7F0000C9B7E1E0E981093FDF76CFA069A079B31
:10A80000FCF75CFC0022B24BFBF732FDB14A0E9024
:10A810000F910E9C0F9D94460F9B634415931D0052
:10A82000109B002B61D1069807990022AA4BFCF7D8
:10A83000B7FE2200159B06900791FAF70DFF00283E
:10A8400000D0A8E2A5480F99844661440B00069801
:10A8500007992200FAF7ECFE002800D095E2129B3F
:10A86000139C06930794199B002B00DA5CE10E2FD2
:10A8700000DD59E1934BFA009B185C681B68049358
:10A880000594219B002B00DBD8E0099B002B00DD09
:10A89000D4E000D07DE20498059900228E4BFCF7AD
:10A8A0000DFC069A079BFAF7E1FE099B04931E0034
:10A8B000002800D04FE2089B089A5D1C3123013725
:10A8C00013704BE234420AD00E9B854A01330E933B
:10A8D000EB009B181A685B68FCF7F0FB3300641010
:10A8E00001355FE73E00099B84E7109B0D995A1ED6
:10A8F000744BD2009B181A685B68002949D000206D
:10A900007849FBF7D1FF2B002200FCF749FE089B9A
:10A910000E900F91159306980799FDF7A5F904007D
:10A92000FDF7D8F902000B0006980799FCF738FEEE
:10A93000159B30345D1C1C700E9A0F9B069007917E
:10A94000FAF776FE00286CD1069A079B00205E4934
:10A95000FCF726FE0E9A0F9BFAF76AFE002800D03D
:10A96000C3E0089B109AEB1A9A4200DC77E70E9836
:10A970000F990022554BFCF7A1FB00220E900F917E
:10A9800006980799514BFCF799FB1595069007918E
:10A99000C1E720002900FCF791FB089C109A2300D6
:10A9A00094460E900F916344159306980799FDF70E
:10A9B0005BF90500FDF78EF90B0002000698079978
:10A9C000FCF7EEFD3035159B25700134069007919C
:10A9D000A3422AD10E980F99089A109B944663447B
:10A9E00000221D003F4BFBF743FC02000B000698C2
:10A9F0000799FAF731FE002800D076E00E9A0F9BF7
:10AA000000203849FCF7CCFD02000B00069807999E
:10AA1000FAF70EFE002800D121E76B1E1A78302AC3
:10AA200001D037003FE01D00F7E7069807990022A4
:10AA3000264BFCF743FB06900791B6E7089E049A65
:10AA4000059B06980799FBF72FFFFDF70DF904000A
:10AA5000FDF740F9049A059BFCF730FB02000B0060
:10AA600006980799FCF79CFD230030333370099A50
:10AA7000089B751CEB1A9A4248D102000B00FBF7A9
:10AA8000F7FB049A059B06900791FAF7E5FD00286D
:10AA90002AD1049A059B06980799FAF7C3FD002866
:10AAA00001D0E30720D40399029801F02FF8002386
:10AAB0002B70229B01371F60249B002B00D1E6E402
:10AAC0001D60E4E498CF00000000F03F0000244047
:10AAD00000001C400000C0FC000014400000C07CCE
:10AAE00070CF00000000E03F3E006B1E1A78392A4C
:10AAF00006D1089A9A4207D1302313701300013609
:10AB00001A7801321A708CE71D00EEE70022A44B80
:10AB1000FCF7D4FA00220023069007912E00FAF7E2
:10AB200081FD00288BD0BEE70D9A002A00D1DAE023
:10AB3000209A012A00DDBDE0169A002A00D1B5E076
:10AB4000984A9B18049D0A9C0A9A0121D2180A92DD
:10AB50000B9A0298D3180B9301F0B6F80600002C5C
:10AB60000EDD0B9B002B0BDD0B9A2300944200DDC6
:10AB700013000A9AE41AD21A0A920B9AD31A0B9368
:10AB8000049B002B1FD00D9B002B00D1AFE0002DAC
:10AB900011D031002A00029801F02EF9039A010029
:10ABA0000600029801F099F803991090029800F0BD
:10ABB000ADFF109B0393049B5A1B04D0039902988A
:10ABC00001F01AF903900121029801F07DF8119B20
:10ABD0000490002B00D1E3E11A000100029801F07B
:10ABE0000BF9209B0490012B00DD82E00025069BE1
:10ABF000AB420ED1079B1B03AB420AD1179B079AAE
:10AC0000134206D00A9B013501330A930B9B013393
:10AC10000B93119B0120002B6CD10B9B18181F2349
:10AC200018407ED001331B1A042B70DD1C23181A28
:10AC30000A9B24181B180A930B9B1B180B930A9B47
:10AC4000002B05DD1A000399029801F027F9039003
:10AC50000B9B002B05DD1A000499029801F01EF9E8
:10AC60000490149B002B5ED00499039801F068F9BE
:10AC7000002858DA00230A220399029800F05FFFA7
:10AC80000D9B013F0390002B00D190E10023310088
:10AC90000A22029800F053FF0C9B0600002B00DDF7
:10ACA00088E0209B022B00DC84E044E03623189AE5
:10ACB0009B1A47E7099B5D1E049BAB4208DB5D1BAB
:10ACC000099B002B0CDA0A9B099A9C1A00233BE78C
:10ACD000049B0495EA1A119B00259B181193EFE73A
:10ACE0000A9C099B30E7049D0A9C0D9E37E7049A55
:10ACF00064E70025049B049A1B69109303339B00AF
:10AD0000D318586800F097FF2023181A85E7042B02
:10AD100095D00A9A1C33D2180A920B9AE418D318C9
:10AD20008CE70300F5E7099B002B3DDC209B022B01
:10AD30003ADD099B0C930C9B002B0CD10499052246
:10AD4000029800F0FCFE04900100039801F0F8F86E
:10AD5000002800DDAFE5219B089DDF430023099318
:10AD60000499029800F0D2FE002E00D19BE6099BC8
:10AD7000002B05D0B34203D01900029800F0C6FEA4
:10AD80003100029800F0C2FE8DE6109B04931E0075
:10AD9000E1E70023FAE7109B370004931E008AE5E1
:10ADA00000002440330400000D9B002B00D1B2E0D2
:10ADB000099B0C93002C05DD31002200029801F064
:10ADC0006DF806003000002D11D07168029800F077
:10ADD00065FE3100040033690C319A1C92000C307E
:10ADE000FDF744FA01222100029801F057F8099674
:10ADF0000600089B0A9304990398FFF77CFA0999C7
:10AE00000D900400039801F09BF832001090049913
:10AE1000029801F0AFF801230B93C36830340500AA
:10AE2000002B04D10100039801F08AF80B9029004F
:10AE3000029800F06BFE0B9B209A13430ED1069AEA
:10AE4000013313420AD1392C26D0109B002B01DD8F
:10AE50000D9C31340A9B5D1C1C7081E7109B002BFC
:10AE600007DB1D00209B1D4322D10123069A1342BC
:10AE70001ED10B9B002BEDDD03990122029801F0FE
:10AE80000DF80499039001F05BF8002802DCE1D191
:10AE9000E307DFD5392CDBD10A9B0A9A5D1C3923E5
:10AEA00013706B1E1A78392A67D001321A7057E76F
:10AEB0000A9B5D1C0B9B002B04DD392CECD001346C
:10AEC0000A9BC9E70A9B0C9A1C70089BEB1A9342D9
:10AED0003ED000230A220399029800F030FE099B1D
:10AEE0000390B34209D100230A220999029800F085
:10AEF00026FE099006000A957DE7099900230A229B
:10AF0000029800F01CFE002309900A2231000298EA
:10AF100000F015FEEEE7099B0C93089B069304993D
:10AF20000398FFF7E8F9069B30305D1C18700C9A07
:10AF3000089B0400EB1A9A4208DD00230A220399B9
:10AF4000029800F0FCFD06950390E8E700230993C2
:10AF500003990122029800F0A1FF0499039000F0E8
:10AF6000EFFF00289DDC01D1E3079AD46B1E1A780D
:10AF7000302A00D0F4E61D00F8E7089A9A4203D17F
:10AF8000312301371370EBE61D008AE70B4B249A3F
:10AF900008930B4B002A01D0FFF777FAFFF777FAF7
:10AFA000209B012B00DC21E6119D012035E60C9B46
:10AFB000002BB2DC209B022BAFDDBCE6F8CE0000FC
:10AFC00000CF0000F7B58A8905000C00130760D494
:10AFD0004B68002B04DC0B6C002B01DC0020FEBD59
:10AFE000E76A002FFAD000232E682B6080235B01D4
:10AFF000216A1A4034D0606DA3895B0706D5636867
:10B00000C01A636B002B01D0236CC01A0200216AA6
:10B0100000232800E76AB847A189431C06D12B68A2
:10B020001D2B30D82B4ADA40D3072CD50023636080
:10B0300023692360CB0405D5431C02D12B68002B68
:10B0400000D16065616B2E600029C7D023004433B6
:10B05000994202D02800FDF71BF900206063BEE78B
:10B0600001232800B847431CC6D12B68002BC3D04E
:10B070001D2B01D0162B01D12E60AFE74023A289F2
:10B080001343A381ABE740230B430120A38140423C
:10B09000A5E70F69002FA1D00B680F60DB1B0193A0
:10B0A0000023920700D14B69A360019B002B00DCB9
:10B0B00094E7019B3A00216A2800A66AB04700285D
:10B0C00003DC4023A2891343DFE7019B3F181B1ACF
:10B0D0000193EAE7010040200B6970B505000C0000
:10B0E000002B01D1002070BD002804D08369002B03
:10B0F00001D100F05FF80B4B9C4209D16C680C2227
:10B10000A35E002BEED021002800FFF75BFFEAE7EB
:10B11000054B9C4201D1AC68F1E7044B9C42EED157
:10B12000EC68ECE728CF000048CF000008CF000013
:10B13000002310B50400036043608360818143668F
:10B14000C281036143618361190008225C30FDF70D
:10B1500096F8054B24626362044BA362044BE362DE
:10B16000044B236310BDC04645C600006DC60000F9
:10B17000A5C60000D1C6000010B5024900F08CF849
:10B1800010BDC046D9B0000070B568254A1E5543B1
:10B190000E0029007431FDF7C5F8041E08D0002107
:10B1A0002A00016046600C30A0606832FDF767F845
:10B1B000200070BD836913B50400002B28D183647F
:10B1C000C3640365134B144A1B688262019398425F
:10B1D00001D101238361200000F020F8606020008D
:10B1E00000F01CF8A060200000F018F80022E060D9
:10B1F00004216068FFF79CFF01220921A068FFF786
:10B2000097FF02221221E068FFF792FF0123A3615A
:10B2100013BDC04654CE000079B10000F8B51C4BF8
:10B2200007001E68B369002B02D13000FFF7C2FF90
:10B230004836B4687368013B04D53368002B07D0E7
:10B240003668F6E70C22A55E002D0DD06834F2E7D3
:10B2500004213800FFF798FF30600028F0D10C235C
:10B2600004003B602000F8BD20000A4B65662560A5
:10B270006560A560E36025616561A561082229001C
:10B280005C30FCF7FCFF6563A563A564E564E9E752
:10B2900054CE00000100FFFFF7B5040007000026B0
:10B2A00001914834002C01D13000FEBD6368A568CF
:10B2B0000093009B013B009301D52468F2E7AB8922
:10B2C000012B08D90E22AB5E013304D029003800CF
:10B2D000019B984706436835EBE7F0B50400056924
:10B2E00014344B1126009D4214DD1F22AD009B003B
:10B2F00011406519E318220000291ED004CB202735
:10B30000CA40A4467F1A66469D420BD83260002A86
:10B3100000D00436331B9B100361A64201D10023E9
:10B320004361F0BD1E68BE403243664604C604CB8E
:10B33000B446CA40E7E702CB02C216009D42FAD8E3
:10B34000E8E70300303B092B03D82038C3B21800CC
:10B3500070470300613B052B01D84738F6E7020030
:10B36000413A0023052AF2D82738EFE7F0B58DB02F
:10B3700005901498099102920A9300F0E2FA03688A
:10B3800018000793FDF7FCFF0222079B52421B188F
:10B39000013B1B7804900B93099B19688B1C521A74
:10B3A000D118019308910199013308783028F7D01A
:10B3B000FFF7C7FF071E00D06FE0049A07990198B6
:10B3C00001F08CF9002800D06DE0019B049A9C18D4
:10B3D0002078FFF7B6FF002869D00194019B187808
:10B3E000302809D0FFF7ADFF4342434103930123C7
:10B3F00026000893019C04E0019B01330193EDE7D3
:10B4000001342078FFF79DFF0028F9D1049A0799AD
:10B41000200001F063F9002809D1002E0AD1049B15
:10B42000E41826002078FFF78CFF002839D1002788
:10B43000BE4201D0371BBF002378502B01D0702BA8
:10B4400042D163782B2B34D02D2B36D00023661CB1
:10B4500006933078FFF775FF431EDBB2182B33D805
:10B460001038050001363078FFF76BFF431EDBB262
:10B47000182B24D9069B002B00D06D427F19099B05
:10B480001E60039B002B21D0089B06265A42534185
:10B490005B421E4030000DB0F0BD002303931E0040
:10B4A000A8E70134BEE7019C01230393C4E707002A
:10B4B000FAE700230693A61CCBE70123FAE70A2349
:10B4C0005D432D18103DCDE72600D8E7019B039979
:10B4D000E31A013B072B47DC059800F0DFFA030075
:10B4E000143303930893002305001E000693019B69
:10B4F000A3423CD3089C039B40C4E41AA4102C61D3
:10B50000300000F098FB029B64011B68261A01932F
:10B510009E425FDDF61A3100280000F092FE041E04
:10B520000FD001241F212000731E19408840010004
:10B530005A110398920012580A4202D0A34241DCE9
:10B54000022431002800FFF7C8FEBF19029B9B6848
:10B550000493BB424EDA2900059800F0D7FA002385
:10B56000129AA326136095E701315B10B2E7631EC0
:10B5700009930B9A1B78934215D0069B202B05D17B
:10B58000089B1E600026043308930696099B1878D2
:10B59000FFF7D7FE0F231840069B099C9840043301
:10B5A00006430693A3E70123049A9C1A099B1C19DE
:10B5B000019B9C42E1D30799200001F08FF80028FD
:10B5C000DBD194E7B11E280000F03BFE0028B7D085
:10B5D0000324B6E7019B00249E42B7DA9E1B290094
:10B5E0003200059800F05AFC030014330500BF1B1D
:10B5F0000393ABE7029B5E68BE426BDD019BF61BCB
:10B60000B34232DC029BDB68022B26D0032B28D00E
:10B61000012B19D1019BB34216D1012B0DDC029BEA
:10B6200062265B680193019A0A9B1A600123039AC0
:10B630002B611360129B1D602CE7019928000139D2
:10B6400000F0FFFD0028EAD12900059800F05EFA1D
:10B650000023129A502613601CE7139B002BDED0A8
:10B66000F2E7139B002BDAD1EEE7771E002C2FD1E7
:10B67000002F04D03900280000F0E3FD04001F2350
:10B680007A111F401E3BBB400399920052581A4248
:10B6900001D002231C43019B31009B1B0226280082
:10B6A0000193FFF71AFE029B5F68002C40D0029BBB
:10B6B000DB68022B10D0032B12D0012B06D1A2077E
:10B6C00004D5039A126814431C420CD110232EE0B7
:10B6D0000124D4E70126E8E70123139A9B1A139368
:10B6E000139B002BF2D02C69A30004932B00A20023
:10B6F00014339918002294461A68501C1DD0013248
:10B700001A602B001433022E3AD1029A0199126862
:10B71000013A8A420AD14A111F2101989200014040
:10B72000012004008C40D358234248D120231E43DB
:10B73000129B1D600A9B1F60ACE6624604C39942DF
:10B74000DAD8AB689C4212DB6B680598591C00F094
:10B75000A5F929002B6903909A1C92000C310C303A
:10B76000FCF784FD2900059800F0D0F9039D2B69B2
:10B770005A1C2A61012204339B00EB185A60C0E76F
:10B780002A69A2420ADD01212800FFF7A6FD029BDB
:10B7900001379B680126BB42C8DADCE61F24019A08
:10B7A00001262240141EC1D0049A9B18043B18683D
:10B7B00000F041FA20210C1BA042E4DBB6E70600B2
:10B7C000B4E7082370B520259A1A9200AD1A436891
:10B7D00006681C00AC40D34034430460436004302E
:10B7E0008842F4D370BD30B503680C780133002C67
:10B7F00002D10360012030BD1A781500413D192D9A
:10B8000000D820320131A242EFD00020F3E7F0B59A
:10B810008BB001920A68019953119B00CB180493D5
:10B820001F231A400890069202D0049B043304930D
:10B83000049B00251E1F37003400089B35601B68E1
:10B84000079505930295059B01330993059B5B784A
:10B850000393002B28D00398FFF773FD002845D1F0
:10B86000039B202B19D8029B079A934212DDBC42FE
:10B8700006D2072D04DC2A0039002000FFF7A1FFC3
:10B88000019B08259C4205D9271F00253C00029BEF
:10B890003D600793099B0593D5E7039B292B4AD16C
:10B8A000059B089A02331360029B002B43D0BC42D5
:10B8B00006D2072D04DC2A0039002000FFF781FFA3
:10B8C000019B9C4226D904CC1A600433A642FAD2CA
:10B8D000002204C39E42FCD23368002B04D1019B9A
:10B8E0009E4226D101233360052025E0029B0135CD
:10B8F00001330293082D06DD019B9C42CAD9002327
:10B900000125043C23600F22236810401B011843CB
:10B910002060BFE7069B002BDED02021069A049B07
:10B92000891A01225242CA40043B19680A401A602F
:10B93000D2E7043ED0E704200BB0F0BDEC30006845
:10B940007047F03070470000034B1B68186A0028EE
:10B9500000D10248F03070478C000020F000002039
:10B9600070B50E001D000E23C95E96B014000029AC
:10B9700007DA00232B60B3891B0611D48023DB0078
:10B980000FE06A4600F0EEFE0028F2DBF022019B99
:10B9900012021340054A9B185A4253412B60EDE7AF
:10B9A00040230020236016B070BDC04600E0FFFFBA
:10B9B000F7B502268B8905000C00334206D0230020
:10B9C00047332360236101236361F7BD01AB6A46FE
:10B9D000FFF7C6FF009907002800FCF7A3FC00282A
:10B9E00008D10C22A35E9A05EFD4032293431E4391
:10B9F000A681E4E70F4BAB628023A289206013434A
:10BA0000A381009B20616361019B002B0DD00E235D
:10BA1000E15E280000F0B8FE002806D00322A389CA
:10BA200093431A0001231343A381A0893843A081C3
:10BA3000CBE7C04679B1000082B0002900D101A94E
:10BA4000101E06D0002B06D013780B601078431E12
:10BA5000984102B0704702204042FAE7C9B282180A
:10BA6000904201D10020704703788B42FBD0013017
:10BA7000F6E710B5884202D98B18984203D3002309
:10BA800007E08B5C8354013AFBD210BDCC5CC454FC
:10BA900001339A42FAD1F8E77047704770B5466AA9
:10BAA00004000D00002E07D11020FCF7CBFB6062D4
:10BAB000466086600660C660666AF368002B13D035
:10BAC000636AAA00DB689B181868002818D1012156
:10BAD0000E00AE40721D9200200000F0D4FB002842
:10BAE0000CD0456086600DE021220421200000F08A
:10BAF000CAFB636AF060DB68002BE1D1002070BDF7
:10BB000002681A6000230361C360F8E770B5446AF5
:10BB100006000D00002C07D11020FCF793FB70628B
:10BB2000446084600460C460002D07D0736A6A6852
:10BB3000DB6892009B181A682A601D6070BDF7B51B
:10BB40001E0014239C4607000C0000200D698C4445
:10BB500063461B68013099B263461B6851431B0C56
:10BB6000534389190E0C9B1989B21E0C1B045B18D8
:10BB7000614608C18C468542EADC002E1BD0A368D2
:10BB8000AB4212DC63683800591CFFF787FF2100C5
:10BB9000236901909A1C92000C310C30FCF766FB73
:10BBA00021003800FFF7B2FF019C2B1D9B00E3181A
:10BBB00001355E6025612000FEBDF7B50600180066
:10BBC0000C000830092101931500F9F72FFC01231F
:10BBD000002183421FDB3000FFF760FF089B4361B9
:10BBE00001230361092D19DD230009331F00009390
:10BBF00064193B780100303B0A2230000137FFF71F
:10BC00009EFFA742F5D1009B5C19083C2F00019BC9
:10BC10009F4206DBFEBD5B000131DAE70A340925ED
:10BC2000F4E7631BDB5D0100303B0A223000FFF7C5
:10BC300086FF0137EBE70300020C0020824201D1AE
:10BC40001B0410301A0E01D108301B021A0F01D14B
:10BC500004301B019A0F01D102309B00002B03DB43
:10BC600001305B0000D4202070470722036810B524
:10BC700001001A400DD001240020234205D10230DA
:10BC8000034203D0E34020000B6010BD9B080B6013
:10BC9000FBE79CB21000002C01D110201B0CDAB283
:10BCA000002A01D108301B0A1A0701D104301B09F0
:10BCB0009A0701D102309B08DA07E8D45B0801D06B
:10BCC0000130E4E72020E0E710B50C000121FFF788
:10BCD000E5FE01234461036110BDF0B50B6914005A
:10BCE000126989B00D00934201DA25000C002F691A
:10BCF00026696968BB190293AB68BA19934200DAE6
:10BD00000131FFF7CBFE0200BB1914329B00D318A0
:10BD10009C4600211300049063451DD31435BF00D9
:10BD2000EB191434B6000593A319039501940793F6
:10BD3000079B0199994211D3029B002B06DD042336
:10BD40005B429C4463461B68002B51D0049B029AC3
:10BD500018001A6109B0F0BD02C3DDE7019B1B6842
:10BD600098B200281CD015000026039F02CF2C6833
:10BD70008BB24343090C4143A4B21B199B190E001B
:10BD800029680695090C71181E0C89190E0C9BB2B6
:10BD900009040B4308C5059BBB42E7D8069B5E60C0
:10BDA000019B1B681D0C1ED0100000271368039E0A
:10BDB0003168046889B26943240C0919C9190F0450
:10BDC0009BB23B43036080CE43683F0C6F439BB202
:10BDD000FB18090C5B18059906901F0C0430B14242
:10BDE000E6D806994B60019B0432043301939FE728
:10BDF000029B013B02939FE70323F7B51340050025
:10BE00000E001400002B08D02249013B9A00525822
:10BE100000233100FFF793FE0600A310019336D0F4
:10BE20006C6A002C07D11020FCF70CFA68624460A1
:10BE300084600460C4606F6ABC68002C07D1164936
:10BE40002800FFF741FF00230400B86003600122CF
:10BE5000019B13420AD0310022002800FFF73DFF6A
:10BE6000070031002800FFF751FE3E00019B5B10E8
:10BE700001930CD02068002807D12200210028005F
:10BE8000FFF72BFF0023206003600400DFE7300092
:10BE9000FEBDC04660D0000071020000F0B50D008C
:10BEA00017002B69541185B0E318019301330093F7
:10BEB0004968AB680290009A934235DB0298FFF71D
:10BEC000EDFD00230200060019001432A3422EDB10
:10BED000E343DB171C402B00A40014192A69143318
:10BEE00092009A1894461F22174024D00132D21B88
:10BEF0000392002219682000B9400A4304C404CB0D
:10BF00000399CA409C45F5D84260002A02D0019BA3
:10BF100002330093009B0298013B33612900FFF735
:10BF2000F5FD300005B0F0BD01315B00C3E79800BE
:10BF300011500133CAE704CB04C49C45FBD8E9E7A0
:10BF40000A69036930B59B1A0DD19200143014317F
:10BF500084188918043C043925680A68954204D07D
:10BF60000123954204D3180030BDA042F2D3FAE772
:10BF70005B42F8E7F0B50D0085B00700110028001E
:10BF80001400FFF7DDFF061E08D101003800FFF79F
:10BF900085FD01234661036105B0F0BD01230193D6
:10BFA000002804DB23002C001D000023019361689E
:10BFB0003800FFF773FD2F000022019B2669C36044
:10BFC0001434B300E31802932B6914379B00FB1859
:10BFD000039303009446143320CC04CF0192AAB2F9
:10BFE00094446A46614692882D0C8A1A0199090C7C
:10BFF000691A151449190D1492B209040A431A60FA
:10C00000039AAC460433BA42E6D802991A008C422D
:10C0100005D3043A1368002B0ED00661BCE704CCAC
:10C0200091B261440D14120C5219151489B2120404
:10C030000A43AC4604C3E8E7013EEAE70B001049B7
:10C0400010B519400F4BC918002904DD00220B0060
:10C050001000190010BD49420915002200231329C0
:10C0600004DC8020000308410300F1E714390120BB
:10C070001E2902DC1F24611A88400200E8E7C0463E
:10C080000000F07F0000C0FCF7B50600036914361D
:10C090009B00F3181D1F2C680F0020000193FFF771
:10C0A000CAFD20231B1A3B601C490A2816DC0B23FF
:10C0B00027001B1ADF4039439C460B000021AE428B
:10C0C00002D2019908390968153084406046C140A0
:10C0D0000C4322001000190003B0F0BD0027AE424F
:10C0E00002D2019D083D2F680B388446031E12D0F2
:10C0F0009C40202021433C00C01AC44021430B0037
:10C100000021B54201D9043D29686446C140A740D9
:10C110000F433A00DEE721430B00FAE70000F03F4F
:10C12000F7B51D0001211400089FFFF7B7FC2B0392
:10C130006D0006001B0B6D0D24D10193002C27D040
:10C1400068460094FFF791FD009C00281ED0019BDB
:10C1500020211A00091A8A40C340224372610193C8
:10C16000019CB461631E9C4101343461002D18D0E0
:10C17000124BED1835232D183D60181A099B1860D5
:10C180003000FEBD802252031343D6E77461E7E717
:10C1900001A8FFF76AFD0124019B3461736120301F
:10C1A000E4E7074BC018074B3860E3189B00F3180F
:10C1B0005869FFF740FD6401201ADFE7CDFBFFFF60
:10C1C000CEFBFFFFFFFFFF3FF0B585B00F0002A9D8
:10C1D0000600FFF759FF04000D00380003A9009482
:10C1E0000195FFF751FF36693F690200F71B7E0199
:10C1F000B446039F029E0B00F61B66443705002ED3
:10C2000007DD7919019100980199FAF74DFB05B006
:10C21000F0BDCB1BF7E71300013910B549111269C6
:10C22000013189001433920041189A189A4203D8B8
:10C230000023814203D810BD10CB10C0F6E708C020
:10C24000F7E70200006910B514324B11984212DB77
:10C250000BDD1F20014008D0980084582000C84002
:10C260008840010001208C4204D19B00D3189342E6
:10C2700003D8002010BD0300F7E7043B196800292C
:10C28000F5D00120F6E74A4370B511001400FCF721
:10C2900049F8051E03D022000021FBF7F0FF28001B
:10C2A00070BDF8B507000D001600002905D111007A
:10C2B000FCF738F804002000F8BD002A03D1FBF792
:10C2C000E7FF3400F7E700F085FA2C00B042F2D225
:10C2D00031003800FCF726F8041EECD029003200AB
:10C2E000FBF7C4FF29003800FBF7D2FFE3E70000AB
:10C2F000F0B58E6885B007000C00039201939E4252
:10C300003CD890238A89DB001A4234D0032509697E
:10C3100023685B1A0293636902985D43EB0F5D1912
:10C32000019B6D1001331B18AB4200D91D00530552
:10C3300032D529003800FBF7F5FF061E09D10C2382
:10C340003B6040230120A28940421343A38105B0F2
:10C35000F0BD029A2169FBF789FFA389144A1A40AC
:10C3600080231343A381029B2661F6182660656132
:10C37000019EED1AA560019B9E4200D9019E3200EC
:10C3800003992068FFF775FBA36800209B1BA3603F
:10C3900023689E192660DAE72A003800FFF781FF3C
:10C3A000061EE0D121693800FBF772FFC7E7C046DF
:10C3B0007FFBFFFFF0B59FB0029005938B890F00C4
:10C3C00016001B0611D50B69002B0ED14021FBF77F
:10C3D000A9FF38603861002805D10C23029A013882
:10C3E00013601FB0F0BD40237B61002306AC636186
:10C3F000203363761033A37635002B78002B01D0E1
:10C40000252B46D1AB1B04930CD032003900029887
:10C41000FFF76EFF431C00D1AEE06269049B9446B7
:10C42000634463612B78002B00D1A5E00122002337
:10C430005242626002A9543252186E1C2360E360BB
:10C44000A3601370A365317805225448FFF706FBFB
:10C45000751C00281FD12268D30604D5532302A9D6
:10C460005B1820211970130704D5532302A95B1808
:10C470002B21197033782A2B16D0350000210A2081
:10C48000E3682A786E1C303A092A4ED9002918D060
:10C4900010E00135B1E7414B2268C01A0123834007
:10C4A000134323602E00CEE7059B191D1B680591E1
:10C4B000002B01DB099304E05B42E360022313439A
:10C4C00023602B782E2B0AD16B782A2B35D1059B34
:10C4D00002351A1D1B680592002B2BDB0793304E8B
:10C4E000297803223000FFF7B9FA002806D040234C
:10C4F000801B83402268013513432360297806227C
:10C5000028486E1C2176FFF7A9FA00283CD0264B5C
:10C51000002B25D10722059B07339343083305934E
:10C520006369039A9B18636166E7434301219B1883
:10C530003500A6E701235B42D0E700230A201A005A
:10C540000135636029786E1C3039092903D9002B25
:10C55000C5D00792C3E74243012352183500F1E7E3
:10C5600005AB00933A00114B21000298FCF712F939
:10C570000390039B0133D3D1BB890B985B0600D496
:10C580002FE7012040422CE705AB00933A00074B10
:10C5900021000298FCF7B8FBEAE7C04658CE00003D
:10C5A0005ECE000062CE000095870000F1C2000060
:10C5B00070B504000D001F2904D916230360012063
:10C5C000404270BD436C002B04D08A009B181A684F
:10C5D000002A08D1200000F031F82A0001002000D4
:10C5E00000F01AF8EDE70020012AEAD0511C03D12F
:10C5F000162301302360E4E7002428001C609047E4
:10C600002000DEE710B5034B01001868FFF7D0FFEC
:10C6100010BDC0468C000020002370B5064C0500FC
:10C6200008001100236000F011F9431C03D12368B6
:10C63000002B00D02B6070BD600F002010B500F003
:10C64000F5F810BD70B50C000E25495F00F0CAF872
:10C65000002803DB636D1B18636570BDA389024A64
:10C660001340A381F9E7C046FFEFFFFFF8B51F00B5
:10C670008B8905000C001600DB0505D50E23C95E6D
:10C680000022022300F092F8A389054A28001340F3
:10C69000A38132000E23E15E3B0000F03DF8F8BDBF
:10C6A000FFEFFFFF70B50C000E25495F00F07EF82C
:10C6B000A389421C03D1054A1340A38170BD802287
:10C6C00052011343A3816065F8E7C046FFEFFFFF07
:10C6D00010B50E23C95E00F033F810BD002330B54D
:10C6E0009A420AD0013AC45CCD5CAC4204D1934278
:10C6F00002D00133002CF6D1631B180030BD0B1E95
:10C7000004D0FF2A04D98A2303608B3B18007047AA
:10C710000A700123FAE7000070B505000800110057
:10C720000022064C22601A00F5F7E0FD431C03D1FD
:10C730002368002B00D02B6070BDC046600F002026
:10C74000002370B5064C05000800236000F05EF879
:10C75000431C03D12368002B00D02B6070BDC04662
:10C76000600F0020002370B5064C05000800110082
:10C77000236000F053F8431C03D12368002B00D042
:10C780002B6070BD600F0020002370B5064C0500C3
:10C790000800236000F052F8431C03D12368002BEB
:10C7A00000D02B6070BDC046600F002070B5050042
:10C7B000080011000022064C22601A0000F04EF81A
:10C7C000431C03D12368002B00D02B6070BDC046F2
:10C7D000600F00200B1F1B68181F002B01DA0B587D
:10C7E000C018704770B50500080011000022064C03
:10C7F00022601A0000F03AF8431C03D12368002B92
:10C8000000D02B6070BDC046600F00205822012070
:10C81000014B40421A607047600F002058220120EF
:10C82000014B40421A607047600F002058220120DF
:10C83000014B40421A607047600F00205822024BA3
:10C8400000201A607047C046600F00205822012067
:10C85000014B40421A607047600F002058220120AF
:10C86000014B40421A607047600F0020582201209F
:10C87000014B40421A607047600F0020FEE7C0463F
:10C88000F8B5C046F8BC08BC9E467047F8B5C0462F
:10C89000F8BC08BC9E467047436F756C64206E6F91
:10C8A000742066696E642074686520424D50333888
:10C8B000382073656E736F722C20636865636B201C
:10C8C000776972696E672100424D503338382072A3
:10C8D000656164792E00416C743A20003B204D6103
:10C8E000783A20000A0A54656C656D6920726561AA
:10C8F00064792E2E2E0000000000000000000000D1
:10C900008D050000BD030000B9030000E103000035
:10C91000FD03000051060000E303000005000000D5
:10C920000A00000014000000280000005000000071
:10C93000A00000004001000080020000000500008F
:10C94000000A000000140000002800000050000051
:10C9500000A000000040010000800200000005006F
:10C9600000000A001718191516705F736572636F5F
:10C970006D20213D204E554C4C00433A5C5573656B
:10C9800072735C636F6479615C417070446174615F
:10C990005C4C6F63616C5C41726475696E6F3135BC
:10C9A0005C7061636B616765735C53656565647535
:10C9B000696E6F5C68617264776172655C73616DEA
:10C9C000645C312E372E375C6C6962726172696506
:10C9D000735C5350495C5350492E63707000535040
:10C9E00049436C6173733A3A535049436C617373B2
:10C9F00028534552434F4D2A2C2075696E74385F79
:10CA0000742C2075696E74385F742C2075696E748F
:10CA1000385F742C20536572636F6D53706954587E
:10CA20005061642C20536572636F6D52585061647D
:10CA300029000000000000000200000001000000CA
:10CA4000020000000000FFFFFFFF020000000000E6
:10CA500004000000010000001800000004000000B5
:10CA600000000400000000000A00000001000000B7
:10CA70001C0000001200000100010A00000000007C
:10CA80000B000000010000001C0000001300010169
:10CA900001010B000000000008000000030000007E
:10CAA0001C0000001000000000001000000000004A
:10CAB00009000000030000001C000000110001003C
:10CAC0000100090001000000080000000300000050
:10CAD000180000000200000400040800010000002B
:10CAE000090000000300000018000000030001041A
:10CAF000010409000000000007000000030000001E
:10CB00001C000000070001010101070000000000F7
:10CB100005000000030000001800000005000100EF
:10CB200001000500000000000600000003000000F6
:10CB30001C000000060000010001060000000000CB
:10CB400013000000050000002C000000FF0003009F
:10CB500003000300000000001200000004000000B9
:10CB60001C000000FF0000030003020000000000A2
:10CB700011000000040000001C000000FF00010282
:10CB800001020100000000001C000000060000007F
:10CB900000000000FF00FFFFFFFFFF00000000009B
:10CBA000180000000600000000000000FF00FFFF6A
:10CBB000FFFFFF0000000000190000000600000059
:10CBC00000000000FF00FFFFFFFFFF000D0A000054
:10CBD0000008004214090000000C0042150A000081
:10CBE00000100042160B000000140042170C000059
:10CBF00000180042180D0000001C0042190E000031
:10CC00000000000000000000792800000129000059
:10CC100075280000A92800008D280000DD280000EC
:10CC2000C1280000B528000000000000000000003E
:10CC3000D52B00006F2E0000FB290000572E0000AE
:10CC4000352E0000F9290000212A00002D2B0000BC
:10CC50005365656564205849414F204D30000403F9
:10CC6000090453656565640012010002000000407C
:10CC700086282F8004010102030112010002EF0245
:10CC8000014086282F8004010102030100000000FA
:10CC900000000000493E00002D210000ED3C000096
:10CCA000573D0000713D0000F93C0000C13A000012
:10CCB000B13A0000453B0000DB3A0000AD3A00000D
:10CCC000706F77000000000000000000000030439B
:10CCD00000000000000030C39E5B0000DA5A000034
:10CCE000FE5A00009C5A0000FE5A00007A5B0000C9
:10CCF000FE5A00009C5A0000DA5A0000DA5A00007E
:10CD00007A5B00009C5A0000D05B0000D05B000002
:10CD1000D05B0000865B0000DA5A0000DA5A00009F
:10CD2000FE5A00009A5A0000FE5A00007A5B00008A
:10CD3000FE5A00009A5A0000DA5A0000DA5A00003F
:10CD40007A5B00009A5A0000D05B0000D05B0000C4
:10CD5000D05B0000845B00003C5D0000E65C0000EE
:10CD6000E65C0000145E0000E25C0000E25C000093
:10CD70000A5E0000145E0000E25C00000A5E000033
:10CD8000E25C0000145E0000185E0000185E000007
:10CD9000185E0000205E00004C6B0000BE690000C1
:10CDA000026A000066690000026A0000F26A000080
:10CDB000026A000066690000BE690000BE690000EA
:10CDC000F26A0000666900005E6900005E690000AA
:10CDD0005E690000006B0000747200007671000054
:10CDE0007671000094740000707100007071000092
:10CDF0007C74000094740000707100007C7400006A
:10CE000070710000947400008A7400008A7400003D
:10CE10008A740000987400002C2066756E63746933
:10CE20006F6E3A2000617373657274696F6E2022B1
:10CE3000257322206661696C65643A2066696C65B9
:10CE400020222573222C206C696E652025642573B1
:10CE500025730A0090000020232D302B2000686CE1
:10CE60004C0065666745464700494E4600696E6658
:10CE7000004E414E006E616E00300030313233346E
:10CE80003536373839414243444546003031323334
:10CE90003435363738396162636465660065256C00
:10CEA0006400000035000000CEFBFFFFCB03000054
:10CEB000010000000000000034000000CEFBFFFF76
:10CEC000CB03000001000000000000000000000093
:10CED000BC89D897B2D29C3C33A7A8D523F6493950
:10CEE0003DA7F444FD0FA5329D978CCF08BA5B2572
:10CEF000436FAC6428066811496E66696E6974797F
:10CF0000004E614E00000000000000000000000024
:10CF10000000000000000000000000000000000011
:10CF20000000000000000000000000000000000001
:10CF300000000000000000000000000000000000F1
:10CF400000000000000000000000000000000000E1
:10CF500000000000000000000000000000000000D1
:10CF600000000000000000004300504F53495800EB
:10CF70000080E03779C34143176E05B5B5B89346D5
:10CF8000F5F93FE9034F384D321D30F94877825AA1
:10CF90003CBF737FDD4F1575000000000000F03FBF
:10CFA0000000000000002440000000000000594084
:10CFB0000000000000408F40000000000088C340D7
:10CFC00000000000006AF8400000000080842E414C
:10CFD00000000000D01263410000000084D7974198
:10CFE0000000000065CDCD41000000205FA002429E
:10CFF000000000E876483742000000A2941A6D4213
:10D00000000040E59C30A2420000901EC4BCD64205
:10D0100000003426F56B0C430080E03779C34143B0
:10D0200000A0D8855734764300C84E676DC1AB4326
:10D03000003D9160E458E143408CB5781DAF154444
:10D0400050EFE2D6E41A4B4492D54D06CFF080441F
:10D05000F64AE1C7022DB544B49DD9794378EA4434
:10D0600005000000190000007D00000000202020C5
:10D070002020202020202828282828202020202088
:10D080002020202020202020202020202088101058
:10D0900010101010101010101010101010040404B4
:10D0A0000404040404040410101010101010414172
:10D0B0004141414101010101010101010101010160
:10D0C0000101010101010101101010101010424274
:10D0D0004242424202020202020202020202020230
:10D0E00002020202020202021010101020000000D0
:10D0F0000000000000000000000000000000000030
:10D10000000000000000000000000000000000001F
:10D11000000000000000000000000000000000000F
:10D1200000000000000000000000000000000000FF
:10D1300000000000000000000000000000000000EF
:10D1400000000000000000000000000000000000DF
:10D1500000000000000000000000000000000000CF
:10D1600000000000000000000000000000000000BF
:04D1700000000000BB
:10D174006400010040420F00FFFFFFFFFFFFFFFFBD
:10D1840000C2010000000800080B000202020000B7
:10D194000904000001020200000524001001042417
:10D1A4000206052406000105240101010705810387
:10D1B40010001009040100020A0000000705020221
:10D1C400400000070583024000000000FFFFFFFF4E
:10D1D4000000000083000000020000008200000044
:10D1E400000000000000000000000000000000003B
:10D1F400000000000000000001000000900000207A
:10D204000000000028CF000048CF000008CF000035
:10D21400000000000000000000000000000000000A
:10D2240000000000000000000000000000000000FA
:10D2340000000000000000000000000000000000EA
:10D2440000000000000000000000000000000000DA
:10D2540000000000000000000000000000000000CA
:10D264004300000000000000000000000000000077
:10D2740000000000000000000000000000000000AA
:10D284004300000000000000000000000000000057
:10D29400000000000000000000000000000000008A
:10D2A4004300000000000000000000000000000037
:10D2B400000000000000000000000000000000006A
:10D2C4004300000000000000000000000000000017
:10D2D400000000000000000000000000000000004A
:10D2E40043000000000000000000000000000000F7
:10D2F400000000000000000000000000000000002A
:10D3040043000000000000000000000000000000D6
:10D314000000000000000000000000000000000009
:10D3240043000000000000000000000000000000B6
:10D3340000000000000000000000000000000000E9
:10D34400FFC6000039BA0000000000006CD00000E5
:10D35400F4C80000CECB0000CECB0000CECB000042
:10D36400CECB0000CECB0000CECB0000CECB000055
:10D37400CECB0000CECB0000FFFFFFFFFFFFFFFF7F
:10D38400FFFFFFFFFFFF0000010041534349490035
:10D394000000000000000000000000000000000089
:10D3A4000000000000000000000041534349490010
:10D3B4000000000000000000000000000000000069
:10D3C400000000000000000000000000DD0000007C
:10D3D4007903000089070000B11700000519000057
:0CD3E400D12900009D3A0000B5000000B7
:0400000300001B6975
:00000001FF
